:020000040801F1
:1000000000000220E9DD0108A5200108AD2001085B
:10001000B5200108BD200108C5200108000000002E
:10002000000000000000000000000000CD200108DA
:10003000DB20010800000000E9200108F72001088A
:1000400039DE010839DE010839DE010839DE010830
:1000500039DE010839DE010839DE010839DE010820
:1000600039DE010839DE010839DE01080521010801
:100070001921010839DE010839DE010839DE0108DD
:1000800039DE010839DE010839DE010839DE0108F0
:100090002D21010839DE010839DE010839DE0108A9
:1000A00039DE010839DE010839DE010839DE0108D0
:1000B00039DE010839DE010839DE010839DE0108C0
:1000C00039DE010839DE010839DE010839DE0108B0
:1000D00039DE010839DE010839DE010839DE0108A0
:1000E00039DE010839DE010839DE010839DE010890
:1000F00039DE010839DE010839DE010839DE010880
:1001000039DE010839DE010839DE010839DE01086F
:1001100039DE010839DE010839DE010839DE01085F
:1001200039DE010839DE010839DE010839DE01084F
:1001300039DE010839DE010839DE010839DE01083F
:1001400039DE010839DE010839DE0108000000004F
:10015000000000000000000000000000000000009F
:1001600000000000000000000000000039DE01086F
:1001700039DE010839DE010839DE010839DE0108FF
:1001800039DE010839DE010839DE010839DE0108EF
:1001900039DE01080000000039DE010839DE0108FF
:1001A00039DE010839DE010839DE010839DE0108CF
:1001B00039DE010839DE010839DE010839DE0108BF
:1001C00039DE010839DE010839DE010839DE0108AF
:0801D00039DE010839DE0108E7
:1001E00010B5054C237833B9044B13B10448AFF371
:1001F00000800123237010BDD40100200000000006
:1002000038E5010808B5034B1BB103490348AFF3B8
:10021000008008BD00000000D801002038E501087A
:1002200081F0004102E000BF83F0004330B54FEAA7
:1002300041044FEA430594EA050F08BF90EA020F14
:100240001FBF54EA000C55EA020C7FEA645C7FEAA7
:10025000655C00F0E2804FEA5454D4EB5555B8BFCA
:100260006D420CDD2C4480EA020281EA030382EA3B
:10027000000083EA010180EA020281EA0303362DCD
:1002800088BF30BD11F0004F4FEA01314FF4801CA0
:100290004CEA113102D0404261EB410113F0004FB2
:1002A0004FEA03334CEA133302D0524263EB430369
:1002B00094EA050F00F0A780A4F10104D5F1200E07
:1002C0000DDB02FA0EFC22FA05F2801841F1000162
:1002D00003FA0EF2801843FA05F359410EE0A5F136
:1002E00020050EF1200E012A03FA0EFC28BF4CF067
:1002F000020C43FA05F3C01851EBE37101F000451D
:1003000007D54FF0000EDCF1000C7EEB00006EEB29
:100310000101B1F5801F1BD3B1F5001F0CD34908B3
:100320005FEA30004FEA3C0C04F101044FEA44520A
:1003300012F5800F80F09A80BCF1004F08BF5FEA91
:10034000500C50F1000041EB045141EA050130BD71
:100350005FEA4C0C404141EB0101013C28BFB1F583
:10036000801FE9D291F0000F04BF01460020B1FACE
:1003700081F308BF2033A3F10B03B3F120020CDAA1
:100380000C3208DD02F1140CC2F10C0201FA0CF07F
:1003900021FA02F10CE002F11402D8BFC2F1200CE4
:1003A00001FA02F120FA0CFCDCBF41EA0C0190409A
:1003B000E41AA2BF01EB0451294330BD6FEA0404E3
:1003C0001F3C1CDA0C340EDC04F11404C4F12002CE
:1003D00020FA04F001FA02F340EA030021FA04F3E0
:1003E00045EA030130BDC4F10C04C4F1200220FA37
:1003F00002F001FA04F340EA0300294630BD21FA75
:1004000004F0294630BD94F0000F83F4801306BF3A
:1004100081F480110134013D4EE77FEA645C18BF2E
:100420007FEA655C29D094EA050F08BF90EA020FC5
:1004300005D054EA000C04BF1946104630BD91EABD
:10044000030F1EBF0021002030BD5FEA545C05D1C0
:100450004000494128BF41F0004130BD14F58004FF
:100460003CBF01F5801130BD01F0004545F0FE4173
:1004700041F470014FF0000030BD7FEA645C1ABFA8
:10048000194610467FEA655C1CBF0B46024650EADF
:10049000013406BF52EA033591EA030F41F400210B
:1004A00030BD00BF90F0000F04BF0021704730B591
:1004B0004FF4806404F132044FF000054FF0000166
:1004C00050E700BF90F0000F04BF0021704730B527
:1004D0004FF4806404F1320410F0004548BF4042FC
:1004E0004FF000013EE700BF42004FEAE2014FEA51
:1004F00031014FEA02701FBF12F07F4393F07F4F2C
:1005000081F06051704732F07F4208BF704793F02E
:100510007F4F04BF41F40021704730B54FF4607441
:1005200001F0004521F000411CE700BF50EA010244
:1005300008BF704730B54FF000050AE050EA0102ED
:1005400008BF704730B511F0004502D5404261EB5D
:1005500041014FF4806404F132045FEA915C3FF49E
:10056000D8AE4FF003025FEADC0C18BF03325FEA3B
:10057000DC0C18BF033202EBDC02C2F1200300FAEC
:1005800003FC20FA02F001FA03FE40EA0E0021FA11
:1005900002F11444BDE600BF53B94AB9002908BFAF
:1005A00000281CBF4FF0FF314FF0FF3000F06AB958
:1005B000ADF1080C6DE904CE00F006F8DDF804E0BA
:1005C000DDE9022304B070472DE9F047089D0C4691
:1005D000002B4ED194468C458646B2FA82F262D9FF
:1005E0004AB1C2F12003914020FA03F30CFA02FC55
:1005F000194300FA02FE4FEA1C471FFA8CF6B1FBC2
:10060000F7F44FEA1E4307FB141143EA014304FBCE
:1006100006F199420AD91CEB030304F1FF3080F084
:100620001281994240F20F81023C6344591A1FFA29
:100630008EF3B1FBF7F007FB101143EA014300FB17
:1006400006F69E420AD91CEB030300F1FF3180F04D
:10065000FC809E4240F2F980634402389B1B40EAD2
:10066000044000211DB1D3400022C5E90032BDE89D
:10067000F0878B4205D90DB1C5E90001002108467C
:10068000F5E7B3FA83F1002946D1A34202D39042A1
:10069000C0F0F080861A64EB03030120002DE6D041
:1006A000C5E90063E3E7002A40F09080A1EB0C0469
:1006B0004FEA1C481FFA8CF70121B4FBF8F64FEA09
:1006C0001E4308FB164443EA044307FB06F0984226
:1006D00008D91CEB030306F1FF3402D2984200F262
:1006E000CD8026461C1A1FFA8EF3B4FBF8F008FBE7
:1006F000104443EA044300FB07F79F4208D91CEB70
:10070000030300F1FF3402D29F4200F2B080204682
:10071000DB1B40EA0640A5E7C1F120068B4022FA28
:1007200006F71F4320FA06FC04FA01F343EA0C0320
:10073000F44000FA01F8380C4FEA1349B4FBF0FE1C
:100740001FFA87FC00FB1E4449EA04440EFB0CF927
:10075000A14502FA01F20AD93C190EF1FF3A80F0E4
:100760008480A14540F28180AEF1020E3C44A4EBAE
:1007700009041FFA83F9B4FBF0F300FB134449EAC0
:10078000044403FB0CFCA44507D93C1903F1FF30DA
:1007900067D2A44565D9023B3C4443EA0E40A0FB26
:1007A0000293A4EB0C049C42CE469C4651D34ED0FF
:1007B00055B1B8EB0E0364EB0C0404FA06F6CB401B
:1007C0001E43CC40C5E90064002150E7C2F120037C
:1007D00020FA03F10CFA02FC24FA03F394400C43D0
:1007E0004FEA1C4800FA02FE1FFA8CF7B3FBF8F040
:1007F00008FB1031230C43EA014300FB07F1994247
:1008000008D91CEB030300F1FF362CD299422AD9F8
:10081000023863445B1AA4B2B3FBF8F108FB11334E
:1008200044EA034401FB07F3A34208D91CEB040488
:1008300001F1FF3613D2A34211D902396444E41AFC
:1008400041EA004139E70446F0E6084606E7C845B4
:10085000AED2B9EB020E63EB070C0138A8E73146C4
:10086000EDE7034699E73046D4E7D6467FE7634491
:1008700002384DE70646234608460FE7023E63442A
:1008800030E700BF704700BF00000000000000001C
:1008900001F0FF01102A2BDB10F0070F08D010F831
:1008A000013B013A8B422DD010F0070F42B3F6D135
:1008B000F0B441EA012141EA014122F007047FF04E
:1008C00000070023F0E80256083C85EA010586EAA5
:1008D000010685FA47F5A3FA87F586FA47F6A5FAE1
:1008E00087F68EB9EED1F0BC01F0FF0102F00702ED
:1008F00032B110F8013B013A83EA010313B1F8D198
:100900000020704701387047002D06BF3546033878
:10091000073815F0010F07D1013015F4807F02BFB1
:10092000013015F4C03F0130F0BC0138704700BF02
:1009300002440346934200D1704703F8011BF9E7D4
:1009400070B50D4D0D4C641BA4100026A64209D1B4
:100950000B4D0C4C0DF0F0FD641BA4100026A642BC
:1009600005D170BD55F8043B98470136EEE755F8C0
:10097000043B98470136F2E770E6010870E601088B
:1009800070E6010874E601087047704738B50546FF
:10099000002941D051F8043C0C1F002BB8BFE418CB
:1009A00000F0E0F81D4A136833B96360146028460C
:1009B000BDE8384000F0DCB8A34208D9206821180F
:1009C0008B4201BF19685B6809182160EDE71A4680
:1009D0005B680BB1A342FAD911685018A0420BD141
:1009E00020680144501883421160E0D118685B68A8
:1009F000536008441060DAE702D90C232B60D6E775
:100A0000206821188B4204BF19685B68636004BFCB
:100A1000091821605460CAE738BD00BF34030020C4
:100A200070B50F4E0C463168054611B900F0A6F8B6
:100A300030602146284600F0A1F8431C03D14FF056
:100A4000FF34204670BDC41C24F00304A042F8D03B
:100A5000211A284600F092F80130F2D1EFE700BFEA
:100A6000300300202DE9F843CD1C25F0030508359F
:100A70000C2D38BF0C25002D064601DBA94204D9F8
:100A80000C2333600020BDE8F883DFF8D48000F049
:100A900069F8D8F800301C4644BB29463046FFF7B9
:100AA000BFFF431C044658D1D8F800402746002F0A
:100AB00043D1002C4BD023683946304604EB030960
:100AC00000F05CF8814542D121686D1A2946304614
:100AD000FFF7A6FF01303AD023682B442360D8F8F3
:100AE00000305A6862BBC8F800700FE02268521BE1
:100AF00020D40B2A17D96119A342256018BF596069
:100B0000636808BFC8F8001062514B60304600F0BF
:100B10002FF804F10B00231D20F00700C21A1CBFA0
:100B20001B1AA350AFE76268A3420CBFC8F80020AD
:100B30005A60EBE723466468AEE73C467F68B6E759
:100B40001A465B68A342FBD100235360DEE70C2307
:100B50003360304600F00CF894E70560D6E700BF3C
:100B6000340300200148FFF70FBF00BF2C03002013
:100B70000148FFF70ABF00BF2C03002038B5064D1F
:100B80000023044608462B600DF0F8F8431C02D100
:100B90002B6803B1236038BD280300202DE9F04FF6
:100BA00095B00AAF4FF47A737B6264233B6206F020
:100BB000A1F800F021FA00F01FFC00F0A1FE00F007
:100BC000D1FE00F069FF01F02FF801F0B9F800F054
:100BD00071FC00F019FD01F0C1F901F0D9FD00230D
:100BE000FB6116E04749FA6913465B0013449B001A
:100BF0000B44043300221A604249FA6913465B0031
:100C000013449B000B4408333F4A1A60FB690133CD
:100C1000FB61FB69052BE5D97F213C4809F026F9EA
:100C20007F213B4809F022F904223A49374808F06D
:100C300019FA02223849364808F014FA374B1B6873
:100C400000225A63354B1B6800229A63334B1B68A2
:100C50000022DA63324B1B6800225A63304B1B6858
:100C600000229A632E4B1B680022DA6300212B4876
:100C700009F0C2FC0421294809F0BEFC08212748DC
:100C800009F0BAFC0021264809F0B6FC04212448EA
:100C900009F0B2FC0821224809F0AEFC214809F015
:100CA000D9FB214B1B78002B75D0204B1B78002BD8
:100CB00071D00023BB611FE01249BA6913465B0083
:100CC00013449B000B44D3ED007A9FED192ADFED0E
:100CD000191A9FED191ADFED160AB0EE670A00F037
:100CE0003BFBF0EE407A154ABB699B001344C3ED11
:100CF000007ABB690133BB61BB69052BDCD90123D9
:100D00007B613DE0480300209A99993EAC050020A4
:100D10001806002038030020400300209C07002014
:100D2000E807002034080020440300204503002089
:100D30000000C8420000000000C07345900300207E
:100D4000A04A7B699B001344D3ED007A9D4B93ED41
:100D5000007AB0EE472ADFED9C1A9FED9C1ADFED7A
:100D60009A0AB0EE670A00F0F7FAF0EE407A954A78
:100D70007B699B001344C3ED007A7B6901337B617F
:100D80007B69052BDCD900F06BFA914B00221A70BD
:100D9000904B00221A7006F011F802467B6AD31AB3
:100DA000B3F57A7F5DD306F009F878628A4A4FF48A
:100DB00000718A480DF042F838613B69874A9E18F5
:100DC0003B69C3F50073FB607E4B1B681846FFF759
:100DD0008BFB04460D467B4B5B681846FFF784FB94
:100DE00080468946774B9B681846FFF77DFB824615
:100DF0008B46744BDB681846FFF776FBC7E90001AA
:100E0000704B1B691846FFF76FFB02460B46CDE996
:100E1000082397ED007B8DED067BCDE904ABCDE992
:100E20000289CDE900456E4AF96830460DF006F8B2
:100E300002463B6913443B613B69684A98183B6929
:100E4000C3F500731946674B674A0CF0F7FF02467B
:100E50003B6913443B613B699BB219465F4801F013
:100E600065FE05F0ABFF02463B6AD31A632B7FF6A3
:100E700018AF05F0A3FF38625C4B1B7823F0010428
:100E80004FF400615A4807F09FF8034623435AB2D3
:100E9000564B1B785BB213435BB2DAB2534B1A70FA
:100EA000524B1B7823F002044FF48051504807F056
:100EB0008BF803465B0023435AB24C4B1B785BB262
:100EC00013435BB2DAB2494B1A70484B1B7823F0DC
:100ED00004044FF40051464807F076F803469B009F
:100EE00023435AB2414B1B785BB213435BB2DAB275
:100EF0003E4B1A703D4B1B7823F008044FF48041A1
:100F00003B4807F061F80346DB0023435AB2374BF6
:100F10001B785BB213435BB2DAB2344B1A70334BBB
:100F20001B7823F010044FF40041314807F04CF8CF
:100F300003461B0123435AB22C4B1B785BB213436D
:100F40005BB2DAB2294B1A70284B1B7823F02004CD
:100F50004021284807F038F803465B0123435AB282
:100F6000224B1B785BB213435BB2DAB21F4B1A7091
:100F70001E4B1B7823F0400420211D4807F024F865
:100F800003469B0123435AB2184B1B785BB21343B1
:100F90005BB2DAB2154B1A70144B1B7823F0800445
:100FA0001021134807F010F80346DB0123435AB21F
:100FB0000E4B1B785BB213435BB2DAB20B4B1A7069
:100FC0006FE600BF90030020000000000000C84250
:100FD000440300204503002050E50108AC03002035
:100FE0006CE5010894E501089CE50108A8030020D0
:100FF000000400480008004880B594B000AF07F135
:101000001803382200211846FFF792FC3B1D0022EE
:101010001A605A609A60DA601A61002007F05EFA7E
:101020002123BB614FF48033FB6101233B63022327
:101030007B630323BB630423FB6355233B640223CD
:101040007B640423BB640223FB6407F11803184686
:1010500005F0C0FE0346002B01D000F0C7F90F23B6
:101060007B600323BB600023FB6000233B61002304
:101070007B613B1D0421184606F0BEF90346002B98
:1010800001D000F0B3F900BF5037BD4680BD00006D
:1010900080B582B000AF78607B681B68B3F1A04F69
:1010A00002D100F00FF806E07B681B68044A934207
:1010B00001D100F06DF800BF0837BD4680BD00BF0C
:1010C0000001005080B483B000AF00237B604FE08C
:1010D0002C4A7B6832F8133007EE903AB8EEE77A84
:1010E00029497A6813465B0013449B000B4408337C
:1010F000D3ED007A27EE277A23497A6813465B00FE
:1011000013449B000B440833D3ED007AF7EE006ADA
:1011100076EEE76A1C497A6813465B0013449B002D
:101120000B4404331B6807EE903AF8EE677A66EEDC
:10113000A77A77EE277A14497A6813465B0013443E
:101140009B000B44C3ED007A0E4A7B6832F81330E3
:1011500018460D497A6813465B0013449B000B4404
:1011600004331860094B01221A707B6801337B60DD
:101170007B68032BACD900BF00BF0C37BD465DF8C0
:10118000047B7047380300204803002044030020FC
:1011900080B483B000AF04237B6051E07B68043BE4
:1011A0002C4A32F8133007EE903AB8EEE77A2A4923
:1011B0007A6813465B0013449B000B440833D3ED5D
:1011C000007A27EE277A24497A6813465B00134495
:1011D0009B000B440833D3ED007AF7EE006A76EEFD
:1011E000E76A1D497A6813465B0013449B000B4471
:1011F00004331B6807EE903AF8EE677A66EEA77A3A
:1012000077EE277A14497A6813465B0013449B00F3
:101210000B44C3ED007A7B68043B0E4A32F813306E
:1012200018460D497A6813465B0013449B000B4433
:1012300004331860094B01221A707B6801337B600C
:101240007B68052BAAD900BF00BF0C37BD465DF8EF
:10125000047B704740030020480300204503002022
:1012600080B584B000AF364BD3ED017A9FED352ABF
:10127000DFED351A9FED351ADFED330AB0EE670A60
:1012800000F06AF887ED030A2D4BD3ED027A9FED4B
:101290002D2ADFED2D1A9FED2D1ADFED2B0AB0EE72
:1012A000670A00F059F887ED020A254BD3ED037A5F
:1012B0009FED242ADFED241A9FED241ADFED220A88
:1012C000B0EE670A00F048F887ED010A1C4BD3ED39
:1012D000047A9FED1C2ADFED1C1A9FED1C1ADFED2E
:1012E0001A0AB0EE670A00F037F887ED000A184BCB
:1012F0001B68D7ED037AFCEEE77A17EE902A5A6363
:10130000134B1B68D7ED027AFCEEE77A17EE902AB2
:101310009A630F4B1B68D7ED017AFCEEE77A17EE64
:10132000902ADA630B4B1B68D7ED007AFCEEE77A64
:1013300017EE902A5A6300BF1037BD4680BD00BF2C
:101340009003002000401C45000000000000C8423F
:101350009C070020E807002080B489B000AF87ED2B
:10136000050AC7ED040A87ED031AC7ED021A87EDD7
:10137000012A97ED057AD7ED047A37EE677AD7ED33
:10138000016AD7ED027A76EEE77A67EE276A97ED83
:10139000037AD7ED047A37EE677AC6EE877A97ED4F
:1013A000027A77EE277AC7ED077A97ED027AD7EDC2
:1013B000077AB4EEE77AF1EE10FA02DDBB68FB6162
:1013C0000AE097ED017AD7ED077AB4EEE77AF1EE0D
:1013D00010FA01D57B68FB61FB6907EE903AB0EE2D
:1013E000670A2437BD465DF8047B704780B400AFC0
:1013F00072B600BF00BFFDE780B58AB000AF07F14D
:10140000140300221A605A609A60DA601A61264B4F
:10141000DB6C254A43F02003D364234BDB6C03F0E1
:1014200020033B613B69204BDB6C1F4A43F0010307
:10143000D3641D4BDB6C03F00103FB60FB681A4BAC
:10144000DB6C194A43F00203D364174BDB6C03F0E7
:101450000203BB60BB68144BDB6C134A43F004030C
:10146000D364114BDB6C03F004037B607B684FF6A5
:1014700030037B610023BB610223FB6107F114038E
:1014800019460A4806F01EFC40237B610023BB611D
:101490000223FB6107F114031946054806F012FC0C
:1014A00000BF2837BD4680BD001002400004004840
:1014B0000008004880B58CB000AF07F1240300227B
:1014C0001A605A609A603B1D202200211846FFF7DF
:1014D0002FFA484B4FF0A0421A60464B4FF440326F
:1014E0005A60444B00229A60424B0022DA60414B22
:1014F00000221A613F4B01225A613E4B04229A613D
:101500003C4B00221A773B4B00225A77394B04227E
:101510001A62384B002283F82420364B4FF4906235
:10152000DA62344B4FF480621A63324B012283F843
:101530003820304B0022DA632E4B002283F8402003
:101540002C4807F0D3FB0346002B01D0FFF74EFFDA
:1015500000237B6207F124031946264808F0E8FCC3
:101560000346002B01D0FFF741FF234B7B6006238E
:10157000BB600223FB607F233B6104237B6100236C
:10158000BB613B1D19461B4807F054FE0346002B68
:1015900001D0FFF72BFF194B7B600C23BB603B1D79
:1015A0001946144807F046FE0346002B01D0FFF70A
:1015B0001DFF134B7B601223BB603B1D19460D487A
:1015C00007F038FE0346002B01D0FFF70FFF0D4B4D
:1015D0007B601823BB603B1D1946064807F02AFEB6
:1015E0000346002B01D0FFF701FF00BF3037BD4697
:1015F00080BD00BFAC05002002003004040060087C
:101600000800900C1000C01080B588B000AF3B46B9
:10161000202200211846FFF78BF9334B334A1A601A
:10162000314B4FF440325A602F4B00229A602E4BC0
:101630000022DA602C4B00221A612B4B01225A61E6
:10164000294B04229A61284B00221A77264B00224C
:101650005A77254B02221A62234B002283F824205A
:10166000214B4FF49062DA621F4B4FF480621A6391
:101670001D4B012283F838201B4B0022DA631A4BE2
:10168000002283F84020184807F030FB0346002B67
:1016900001D0FFF7ABFE164B3B6006237B600223B5
:1016A000BB607F23FB6004233B6100237B613B46DF
:1016B00019460D4807F0BEFD0346002B01D0FFF789
:1016C00095FE0C4B3B600C237B603B46194606485D
:1016D00007F0B0FD0346002B01D0FFF787FE00BFE7
:1016E0002037BD4680BD00BF180600200001005015
:1016F000000052470020903680B5A0B000AF78605F
:1017000007F16C0300221A605A609A60DA601A616D
:1017100007F11803542200211846FFF709F97B68E6
:101720001B68B3F1A04F6AD14FF40043BB614FF087
:101730000053FB6507F11803184606F075F80346D9
:10174000002B01D0FFF752FE664B1B680133654A40
:101750001360644B1B68012B0BD1634BDB6C624A3B
:1017600043F40053D364604BDB6C03F400537B61A0
:101770007B695D4BDB6C5C4A43F00103D3645A4BDD
:10178000DB6C03F001033B613B690F23FB66032322
:101790003B6700237B6707F16C0319464FF09040CD
:1017A00006F090FA514B524A1A60504B05225A608B
:1017B0004E4B00229A604D4B0022DA604B4B802248
:1017C0001A614A4B4FF480725A61484B4FF4806261
:1017D0009A61464B2022DA61444B4FF480521A62E0
:1017E000424806F009FC0346002B01D0FFF7FEFD3E
:1017F0007B683E4A5A653D4A7B6893626EE07B682F
:101800001B683C4A934269D14FF40043BB614FF0DF
:101810000053FB6507F11803184606F005F8034668
:10182000002B01D0FFF7E2FD2E4B1B6801332D4A40
:1018300013602C4B1B68012B0BD12B4BDB6C2A4A02
:1018400043F40053D364284BDB6C03F40053FB6078
:10185000FB68254BDB6C244A43F00103D364224B25
:10186000DB6C03F00103BB60BB683023FB66032322
:101870003B6700237B6707F16C0319464FF09040EC
:1018800006F020FA1C4B1D4A1A601B4B24225A609A
:10189000194B00229A60184B0022DA60164B802206
:1018A0001A61154B4FF480725A61134B4FF48062EA
:1018B0009A61114B2022DA610F4B4FF480521A6269
:1018C0000D4806F099FB0346002B01D0FFF78EFD73
:1018D0007B68094A5A65084A7B68936200BF803773
:1018E000BD4680BD44070020001002408406002051
:1018F0000800024000010050E40600201C000240E5
:1019000080B582B000AF164B9B6C154A43F00403C0
:101910009364134B9B6C03F004037B607B68104B58
:101920009B6C0F4A43F0010393640D4B9B6C03F0D7
:1019300001033B603B68002200210B2006F05DFFA5
:101940000B2006F074FF002200210C2006F055FF4A
:101950000C2006F06CFF00BF0837BD4680BD00BFFD
:101960000010024080B500AF1B4B1C4A1A601A4B96
:101970001B4A5A60184B00229A60174B0122DA600A
:10198000154B00221A61144B00225A61124B00229F
:101990009A61114B0022DA610F4B00221A620E4845
:1019A00008F0CEFB0346002B01D0FFF71FFD0021FE
:1019B000094808F060FC0346002B01D0FFF716FD34
:1019C0000021054808F0A2FC0346002B01D0FFF7D8
:1019D0000DFD00BF80BD00BF48070020005400403F
:1019E000FBA7A03080B59EB000AF786007F164031C
:1019F00000221A605A609A60DA601A6107F11003D7
:101A0000542200211846FEF793FF7B681B681F4A8B
:101A1000934236D140233B610023FB6207F1100360
:101A2000184605F001FF0346002B01D0FFF7DEFC4E
:101A3000174BDB6C164A43F00203D364144BDB6C88
:101A400003F00203FB60FB684FF440737B661223D4
:101A5000BB660023FB6600233B6704237B6707F11B
:101A6000640319460B4806F02DF9094B9B6D084A93
:101A700043F400139365064B9B6D03F40013BB60A6
:101A8000BB6800BF7837BD4680BD00BF0054004032
:101A9000001002400004004880B59CB000AF07F180
:101AA000600300221A605A609A60DA6007F15403FA
:101AB00000221A605A609A6007F1380300221A6007
:101AC0005A609A60DA601A615A619A613B1D342249
:101AD00000211846FEF72CFF514B524A1A60504B1A
:101AE00010225A604E4B00229A604D4B42F20F7208
:101AF000DA604B4B00221A61494B00225A61484B75
:101B000080229A61464808F04DFC0346002B01D024
:101B1000FFF76CFC4FF480533B6607F160031946F6
:101B20003F4808F08FFF0346002B01D0FFF75EFC13
:101B30003B4808F0FFFC0346002B01D0FFF756FCA2
:101B400000237B650023BB650023FB6507F154037D
:101B50001946334809F022FD0346002B01D0FFF758
:101B600045FC6023BB630023FB6300233B6400232D
:101B70007B640023BB640023FB6400233B6507F107
:101B8000380300221946264808F048FE0346002B79
:101B900001D0FFF72BFC07F1380304221946204837
:101BA00008F03CFE0346002B01D0FFF71FFC07F1B5
:101BB0003803082219461A4808F030FE0346002B65
:101BC00001D0FFF713FC00237B600023BB600023E0
:101BD000FB6000233B6100237B614FF40053BB613A
:101BE0000023FB6100233B6200237B624FF0007304
:101BF000BB620023FB6200233B6300237B633B1D2E
:101C00001946074809F060FD0346002B01D0FFF795
:101C1000EDFB034800F028F900BF7037BD4680BDDA
:101C20009C070020002C014080B58EB000AF07F16A
:101C3000280300221A605A609A60DA6007F11C03D8
:101C400000221A605A609A603B4600221A605A606D
:101C50009A60DA601A615A619A61384B4FF080429B
:101C60001A60364B10225A60344B00229A60334B74
:101C700042F20F72DA60314B00221A612F4B802240
:101C80009A612E4808F08EFB0346002B01D0FFF727
:101C9000ADFB4FF48053BB6207F128031946274878
:101CA00008F0D0FE0346002B01D0FFF79FFB23482E
:101CB00008F040FC0346002B01D0FFF797FB002300
:101CC000FB6100237B6207F11C0319461B4809F0E6
:101CD00065FC0346002B01D0FFF788FB60233B60C7
:101CE00000237B600023BB6000233B613B46002256
:101CF0001946124808F092FD0346002B01D0FFF769
:101D000075FB3B46042219460C4808F087FD034644
:101D1000002B01D0FFF76AFB3B4608221946074813
:101D200008F07CFD0346002B01D0FFF75FFB034862
:101D300000F09AF800BF3837BD4680BDE8070020A4
:101D400080B588B000AF07F1100300221A605A6016
:101D50009A60DA603B1D00221A605A609A601D4B3F
:101D60001D4A1A601B4BA9225A601A4B00229A6026
:101D7000184B40F2E732DA60164B00221A61154B1D
:101D800080229A61134808F00DFB0346002B01D016
:101D9000FFF72CFB4FF480533B6107F1100319460A
:101DA0000C4808F04FFE0346002B01D0FFF71EFB46
:101DB00020237B600023FB603B1D1946054809F08A
:101DC000EDFB0346002B01D0FFF710FB00BF2037CF
:101DD000BD4680BD340800200004004080B487B0B8
:101DE00000AF78607B681B681C4A93420CD11C4B87
:101DF0001B6E1B4A43F400631366194B1B6E03F4FE
:101E000000637B617B6922E07B681B68B3F1804FD4
:101E10000CD1134B9B6D124A43F001039365104B99
:101E20009B6D03F001033B613B6910E07B681B681D
:101E30000C4A93420BD10A4B9B6D094A43F00203B3
:101E40009365074B9B6D03F00203FB60FB6800BFCB
:101E50001C37BD465DF8047B704700BF002C014075
:101E6000001002400004004080B58AB000AF7860E6
:101E700007F1140300221A605A609A60DA601A614E
:101E80007B681B68324A93421ED1324BDB6C314A6D
:101E900043F00103D3642F4BDB6C03F001033B6180
:101EA0003B694FF4E0637B610223BB610023FB616C
:101EB00000233B6206237B6207F1140319464FF0AF
:101EC000904005F0FFFE3FE07B681B68B3F1804F58
:101ED0003AD1204BDB6C1F4A43F00203D3641D4B05
:101EE000DB6C03F00203FB60FB681A4BDB6C194AE6
:101EF00043F00103D364174BDB6C03F00103BB60B9
:101F0000BB684FF481637B610223BB610023FB61EB
:101F100000233B6201237B6207F1140319460E483C
:101F200005F0D0FE4FF400437B610223BB61002328
:101F3000FB6100233B6201237B6207F11403194616
:101F40004FF0904005F0BEFE00BF2837BD4680BD73
:101F5000002C0140001002400004004880B500AF92
:101F6000224B234A1A60214B4FF4E1325A601F4B37
:101F700000229A601D4B0022DA601C4B00221A617D
:101F80001A4B0C225A61194B00229A61174B0022FE
:101F9000DA61164B00221A62144B00225A62134B6C
:101FA00000229A62114809F023FC0346002B01D05D
:101FB000FFF71CFA00210D480AF0BEF90346002B7A
:101FC00001D0FFF713FA002108480AF0F3F903469D
:101FD000002B01D0FFF70AFA04480AF074F903460F
:101FE000002B01D0FFF702FA00BF80BD800800205F
:101FF0000038014080B59EB000AF786007F16403FF
:1020000000221A605A609A60DA601A6107F11003C0
:10201000542200211846FEF78BFC7B681B681E4A81
:10202000934235D101233B6100237B6107F110030B
:10203000184605F0F9FB0346002B01D0FFF7D6F94F
:10204000164B1B6E154A43F480431366134B1B6EED
:1020500003F48043FB60FB68104BDB6C0F4A43F0DA
:102060000203D3640D4BDB6C03F00203BB60BB685F
:10207000C0237B660223BB660023FB6600233B670D
:1020800007237B6707F164031946054805F01AFE2C
:1020900000BF7837BD4680BD0038014000100240C7
:1020A0000004004880B400AF00BFFDE780B400AF7B
:1020B00000BFFDE780B400AF00BFFDE780B400AF14
:1020C00000BFFDE780B400AF00BFFDE780B400AF04
:1020D00000BFBD465DF8047B704780B400AF00BF11
:1020E000BD465DF8047B704780B400AF00BFBD46BD
:1020F0005DF8047B704780B500AF04F04DFE00BF73
:1021000080BD000080B500AF024806F098F800BF1F
:1021100080BD00BF8406002080B500AF024806F0F5
:102120008EF800BF80BD00BFE406002080B500AF80
:10213000024800F022FE00BF80BD00BF140900204D
:1021400080B582B000AF0F4B1B6E0E4A43F0010307
:1021500013660C4B1B6E03F001037B607B68094B1D
:102160009B6D084A43F080539365064B9B6D03F0CB
:1021700080533B603B6806F055FA00BF0837BD4608
:1021800080BD00BF0010024080B598B000AF7860FD
:1021900007F10C03542200211846FEF7C9FB7B68A7
:1021A0001B68154A934222D14FF40053FB60002371
:1021B000BB6407F10C03184605F036FB0346002B01
:1021C00001D0FFF713F90D4B9B6D0C4A43F400034C
:1021D00093650A4B9B6D03F40003BB60BB68002250
:1021E0000021142006F009FB142006F020FB00BF9C
:1021F0006037BD4680BD00BF005C0040001002405B
:1022000080B582B000AF78607B68D3F8D8227B6855
:1022100003F52673194610460AF010FA00BF083776
:10222000BD4680BD80B582B000AF78600B46FB70C4
:102230007B68D3F8D802FA78796813469B00134478
:10224000DB000B4403F5B2731A68FB7819460AF0F9
:102250004AFA00BF0837BD4680BD80B582B000AFE6
:1022600078600B46FB707B68D3F8D802FA787968FF
:1022700013469B001344DB000B4424331A68FB789D
:1022800019460AF093FA00BF0837BD4680BD80B5F5
:1022900082B000AF78607B68D3F8D83218460AF075
:1022A000A7FB00BF0837BD4680BD80B584B000AF36
:1022B00078600123FB737B685B79022B01D0FFF709
:1022C00095F87B68D3F8D832FA7B114618460AF0A5
:1022D00051FB7B68D3F8D83218460AF0FDFA00BFEC
:1022E0001037BD4680BD000080B582B000AF786079
:1022F0007B68D3F8D83218460AF04CFB7B685B7ACF
:10230000002B05D0044B1B69034A43F006031361FD
:1023100000BF0837BD4680BD00ED00E080B582B04B
:1023200000AF78607B685B7A002B07D0084B1B6995
:10233000074A23F00603136100F0F8F97B68D3F82D
:10234000D83218460AF03CFB00BF0837BD4680BDB6
:1023500000ED00E080B582B000AF78602B4A7B686A
:10236000C2F8D8327B68294AC3F8C422274B284ACE
:102370001A60264B08221A71244B02225A71234BF1
:102380000222DA71214B00221A72204B00225A726B
:102390001E4B00229A721D4B0022DA721B4800F07D
:1023A000FCFB0346002B01D0FFF720F87B68D3F835
:1023B000C40218230022002102F0B5F87B68D3F88C
:1023C000C40258230022802102F0ADF87B68D3F8C4
:1023D000C402C0230022812102F0A5F87B68D3F853
:1023E000C4024FF488730022012102F09CF87B683C
:1023F000D3F8C4024FF480730022822102F093F8D4
:10240000002318460837BD4680BD00BF14090020D0
:10241000005C004080B584B000AF78600023FB739F
:102420000023BB737B68D3F8C432184600F083FCEA
:102430000346FB73FB7B184600F07EF90346BB7333
:10244000BB7B18461037BD4680BD80B584B000AF59
:102450007860084611461A460346FB700B46BB706F
:1024600013463B800023FB730023BB737B68D3F8C8
:10247000C402BB783A88F97800F0CAFD0346FB73C2
:10248000FB7B184600F058F90346BB73BB7B18462C
:102490001037BD4680BD80B584B000AF78600B4674
:1024A000FB700023FB730023BB737B68D3F8C4323B
:1024B000FA781146184600F008FE0346FB73FB7BD2
:1024C000184600F039F90346BB73BB7B184610373A
:1024D000BD4680BD80B584B000AF78600B46FB7010
:1024E0000023FB730023BB737B68D3F8C432FA78F4
:1024F0001146184600F0B1FE0346FB73FB7B1846FD
:1025000000F01AF90346BB73BB7B18461037BD4673
:1025100080BD80B584B000AF78600B46FB700023AF
:10252000FB730023BB737B68D3F8C432FA7811467F
:10253000184600F0E4FE0346FB73FB7B184600F0F0
:10254000FBF80346BB73BB7B18461037BD4680BD06
:1025500080B485B000AF78600B46FB707B68D3F821
:10256000C432FB6097F90330002B0BDAFB7803F0E1
:102570007F02F96813469B001344DB000B441233BF
:102580001B780BE0FB7803F07F02F96813469B0091
:102590001344DB000B4403F5A9731B78184614376A
:1025A000BD465DF8047B704780B584B000AF7860AD
:1025B0000B46FB700023FB730023BB737B68D3F8CF
:1025C000C432FA781146184600F0FEFC0346FB734D
:1025D000FB7B184600F0B0F80346BB73BB7B184684
:1025E0001037BD4680BD80B586B000AFF8607A6018
:1025F0003B600B46FB720023FB750023BB75FB6839
:10260000D3F8C402F97A3B687A6800F0EFFD03461C
:10261000FB75FB7D184600F08FF80346BB75BB7D4C
:1026200018461837BD4680BD80B586B000AFF8604B
:102630007A603B600B46FB720023FB750023BB7581
:10264000FB68D3F8C402F97A3B687A6800F085FD2C
:102650000346FB75FB7D184600F06EF80346BB751C
:10266000BB7D18461837BD4680BD80B582B000AF2F
:1026700078600B46FB707B68D3F8C432FA78114659
:10268000184600F09BFD034618460837BD4680BD3E
:1026900080B582B000AF78600B46FB70FB78002BF2
:1026A00002D0012B13D023E07B685B7A002B07D08C
:1026B00000F03CF8104B1B690F4A23F0060313612E
:1026C0007B68D3F8D83218460AF07AF910E07B68B4
:1026D000D3F8D83218460AF05DF97B685B7A002B94
:1026E00005D0054B1B69044A43F00603136100BF84
:1026F00000BF0837BD4680BD00ED00E080B483B068
:1027000000AF7860034B18460C37BD465DF8047B7C
:10271000704700BFF00B002080B483B000AF78603A
:1027200000BF0C37BD465DF8047B704780B500AF35
:10273000FEF762FC00BF80BD80B485B000AF0346E9
:10274000FB710023FB73FB79032B17D801A252F80E
:1027500023F000BF652701086B27010871270108D6
:10276000772701080023FB730BE00323FB7308E0CA
:102770000123FB7305E00323FB7302E00323FB73D8
:1027800000BFFB7B18461437BD465DF8047B7047DD
:1027900080B500AF00221249124809F0ADFE034691
:1027A000002B01D0FEF722FE0F490E4809F0D4FE9F
:1027B0000346002B01D0FEF719FE0C4909480BF027
:1027C00037FA0346002B01D0FEF710FE054809F04A
:1027D000EAFE0346002B01D0FEF708FE00BF80BDD5
:1027E00050000020100E0020D0000020A400002087
:1027F00080B483B000AF03463960FB713B6812229E
:102800001A80034B18460C37BD465DF8047B7047B1
:102810007000002080B483B000AF03463960FB71C4
:102820003B6804221A80034B18460C37BD465DF8FE
:10283000047B70478400002080B582B000AF03465F
:102840003960FB71FB79002B05D13A6807490848CC
:102850000AF091FE04E03A68044905480AF08BFE4C
:10286000024B18460837BD4680BD00BFE01000206F
:10287000ACE5010880B582B000AF03463960FB715A
:102880003A68044904480AF076FE024B18460837B5
:10289000BD4680BDE0100020C4E5010880B582B0CF
:1028A00000AF03463960FB713B681A221A8000F0C2
:1028B00043F8024B18460837BD4680BD880000200B
:1028C00080B582B000AF03463960FB71FB79002B05
:1028D00005D13A68074908480AF04DFE04E03A6815
:1028E000044905480AF047FE024B18460837BD4622
:1028F00080BD00BFE0100020D8E5010880B582B09F
:1029000000AF03463960FB71FB79002B05D13A68B3
:10291000074908480AF02FFE04E03A6804490548D0
:102920000AF029FE024B18460837BD4680BD00BF9D
:10293000E0100020E4E5010880B584B000AF0F4B43
:102940001B68FB600E4B1B68BB600E4B1B687B60FB
:10295000FA687B681344FB60FB68002B09D00822EF
:102960000949F86800F014F804220849B86800F032
:102970000FF800BF1037BD4680BD00BF9075FF1F28
:102980009475FF1F9875FF1F8A0000209A00002091
:1029900080B487B000AFF860B9601346FB710023C4
:1029A000FB750023FB7527E0FB681B0F092B0BD879
:1029B000FB681B0FDAB2FB7D5B001946BB680B445A
:1029C0003032D2B21A700AE0FB681B0FDAB2FB7D1C
:1029D0005B001946BB680B443732D2B21A70FB68F1
:1029E0001B01FB60FB7D5B000133BA6813440022CE
:1029F0001A70FB7D0133FB75FA7DFB799A42D3D3C4
:102A000000BF00BF1C37BD465DF8047B7047000067
:102A100080B500AF0022054905480BF01EF90549B5
:102A200003480BF038F90023184680BDE01A002057
:102A3000100E0020E012002080B400AF00231846E2
:102A4000BD465DF8047B704780B483B000AF034699
:102A50003960FB711346BB80FB79232B4AD801A256
:102A600052F823F0F52A0108F52A0108F52A010891
:102A7000F52A0108F52A0108F52A0108F52A0108B6
:102A8000F52A0108F52A0108F52A0108F52A0108A6
:102A9000F52A0108F52A0108F52A0108F52A010896
:102AA000F52A0108F52A0108F52A0108F52A010886
:102AB000F52A0108F52A0108F52A0108F52A010876
:102AC000F52A0108F52A0108F52A0108F52A010866
:102AD000F52A0108F52A0108F52A0108F52A010856
:102AE000F52A0108F52A0108F52A0108F52A010846
:102AF000F52A010800BF002318460C37BD465DF8D3
:102B0000047B704780B582B000AF78603960796827
:102B100005480BF0C0F804480BF006F900231846EE
:102B20000837BD4680BD00BF100E002080B584B0C0
:102B300000AF78600B467B800023FB730D4BD3F80E
:102B4000BC32BB60BB68D3F81432002B01D0012328
:102B50000BE07B881A46796806480BF07EF805483A
:102B60000BF0B2F80346FB73FB7B18461037BD46EB
:102B700080BD00BF100E002080B487B000AFF860A9
:102B8000B9601346FB710023FB7597F9173018469F
:102B90001C37BD465DF8047B704780B584B000AF3C
:102BA00078607B68002B01D10123C0E07B6893F83B
:102BB0009132DBB2002B06D17B68002283F8902291
:102BC0007868FFF7E1FA7B68032283F891227B683B
:102BD0001B68184601F02BFD0023FB733EE0FA7BD7
:102BE000796813469B001344DB000B441133012228
:102BF0001A70FA7B796813469B001344DB000B4480
:102C00001033FA7B1A70FA7B796813469B001344E1
:102C1000DB000B44133300221A70FA7B79681346E9
:102C20009B001344DB000B44203300221A60FA7B24
:102C3000796813469B001344DB000B4424330022C5
:102C40001A60FB7B79685A1C13469B001344DB0017
:102C50000B4400221A60FB7B0133FB737B681B79FA
:102C6000FA7B9A42BBD30023FB7344E0FA7B79687A
:102C700013469B001344DB000B4403F25113002264
:102C80001A70FA7B796813469B001344DB000B44EF
:102C900003F5A873FA7B1A70FA7B796813469B00D8
:102CA0001344DB000B4403F2531300221A70FA7B27
:102CB000796813469B001344DB000B4403F5B073A3
:102CC00000221A60FA7B796813469B001344DB00EC
:102CD0000B4403F5B27300221A60FA7B796813463D
:102CE0009B001344DB000B4403F5B47300221A600D
:102CF000FB7B0133FB737B681B79FA7B9A42B5D36C
:102D00007B6818687B68043393E8060001F0AAFC2E
:102D10007B6800221A737B68012283F891227B680A
:102D20009B7A012B02D1786801F040FC0023184601
:102D30001037BD4680BD80B582B000AF78607B683B
:102D400093F89032012B01D1022312E07B6801221B
:102D500083F890227B681B68184601F051FC7B6861
:102D60001B68184603F011FF7B68002283F890224D
:102D7000002318460837BD4680BD80B584B000AF3B
:102D800078607B681B68184603F016FFF860FB68E4
:102D900003F40043002B03D0786800F004FB10E13B
:102DA000FB6803F48063002B13D07B681B68B3F8C7
:102DB00044309AB27B681B6822F4806292B2A3F816
:102DC00044207868FFF771FA0021786800F0FCF879
:102DD000F7E0FB6803F48043002B0CD07B681B6892
:102DE000B3F844309AB27B681B6822F4804292B2F6
:102DF000A3F84420E5E0FB6803F40053002B0CD05B
:102E00007B681B68B3F844309AB27B681B6822F475
:102E1000005292B2A3F84420D3E0FB6803F480533D
:102E2000002B34D07B681B68B3F840309AB27B68C3
:102E30001B6822F0040292B2A3F840207B681B6852
:102E4000B3F840309AB27B681B6822F0080292B255
:102E5000A3F840207B6893F8C832012B07D17B6828
:102E6000002283F8C82200217868FFF711FC7868F7
:102E7000FFF754FA7B681B68B3F844309AB27B685A
:102E80001B6822F4805292B2A3F8442099E0FB68B8
:102E900003F40063002B27D07B681B68B3F8403035
:102EA0009AB27B681B6842F0080292B2A3F84020F5
:102EB0007B681B68B3F844309AB27B681B6822F4C5
:102EC000006292B2A3F844207B681B68B3F84030DC
:102ED0009AB27B681B6842F0040292B2A3F84020C9
:102EE0007868FFF701FA6CE0FB6803F08003002BC1
:102EF00040D07B681B68B3F844309AB27B681B688B
:102F000022F0800292B2A3F844207B6893F8C83282
:102F1000002B2BD17B681B68B3F840309AB27B68DA
:102F20001B6842F0040292B2A3F840207B681B6841
:102F3000B3F840309AB27B681B6842F0080292B244
:102F4000A3F840207B68012283F8C8227B681B68B5
:102F5000B3F854309BB29B0803F03C027B68C3F883
:102F6000CC2201217868FFF793FB2AE07868FFF70D
:102F7000BBF926E0FB6803F40073002B0FD07B68DD
:102F80001B68B3F844309AB27B681B6822F4007265
:102F900092B2A3F844207868FFF779F911E0FB6852
:102FA00003F48073002B0CD07B681B68B3F84430AB
:102FB0009AB27B681B6822F4807292B2A3F8442014
:102FC00000BF1037BD4680BD80B582B000AF7860CD
:102FD0000B46FB707B6893F89032012B01D10223E2
:102FE00012E07B68012283F890227B68FA781A73DA
:102FF0007B681B68FA781146184603F0B2FD7B68BF
:10300000002283F89022002318460837BD4680BD71
:1030100080B584B000AF7860084611461A46034672
:10302000FB700B463B801346BB700023FB7297F985
:103030000330002B0EDAFB7803F0070213469B00E7
:103040001344DB0010337A681344FB60FB680122F1
:103050005A700EE0FB7803F0070213469B001344FE
:10306000DB0003F5A8737A681344FB60FB68002259
:103070005A70FB7803F00703DAB2FB681A703A88DB
:10308000FB681A61FB68BA78DA70BB78022B02D150
:10309000FB6800221A717B6893F89032012B01D1F2
:1030A00002230EE07B68012283F890227B681B6874
:1030B000F968184601F0F4FA7B68002283F8902240
:1030C000FB7A18461037BD4680BD80B584B000AF8E
:1030D00078600B46FB7097F90330002B0EDAFB7813
:1030E00003F0070213469B001344DB0010337A6899
:1030F0001344FB60FB6801225A700EE0FB7803F07A
:10310000070213469B001344DB0003F5A8737A689B
:103110001344FB60FB6800225A70FB7803F007033E
:10312000DAB2FB681A707B6893F89032012B01D1F8
:1031300002230EE07B68012283F890227B681B68E3
:10314000F968184601F070FE7B68002283F890222F
:10315000002318461037BD4680BD80B586B000AF4D
:10316000F8607A603B600B46FB72FB7A03F0070263
:1031700013469B001344DB0003F5A873FA6813445D
:103180007B617B697A685A617B693A689A617B697D
:103190000022DA617B6900225A70FB7A03F0070390
:1031A000DAB27B691A70FB681B687969184602F00D
:1031B00028F8002318461837BD4680BD80B483B078
:1031C00000AF78600B46FB70FB7803F0070279686C
:1031D00013469B001344DB000B4403F5B6731B68D6
:1031E00018460C37BD465DF8047B704780B586B045
:1031F00000AFF8607A603B600B46FB72FB7A03F02D
:10320000070213469B001344DB001033FA68134493
:103210007B617B697A685A617B693A689A617B69EC
:10322000012283F824207B693A681A627B690022B4
:10323000DA617B6901225A70FB7A03F00703DAB284
:103240007B691A70FB681B687969184601F0D9FF21
:10325000002318461837BD4680BD80B584B000AF46
:1032600078600B46FB70FB7803F007037A681279ED
:10327000934201D901233EE097F90330002B0EDA87
:10328000FB7803F0070213469B001344DB00103366
:103290007A681344FB60FB6801225A700CE0FA78EC
:1032A00013469B001344DB0003F5A8737A681344AC
:1032B000FB60FB6800225A70FB6801229A70FB7861
:1032C00003F00703DAB2FB681A707B6893F8903258
:1032D000012B01D102230EE07B68012283F89022AA
:1032E0007B681B68F968184603F03CFB7B6800228A
:1032F00083F89022002318461037BD4680BD80B564
:1033000084B000AF78600B46FB70FB7803F00F03CE
:103310007A681279934201D9012340E097F903308A
:10332000002B0EDAFB7803F0070213469B001344D0
:10333000DB0010337A681344FB60FB6801225A708B
:103340000EE0FB7803F0070213469B001344DB00FA
:1033500003F5A8737A681344FB60FB6800225A7077
:10336000FB6800229A70FB7803F00703DAB2FB686F
:103370001A707B6893F89032012B01D102230EE082
:103380007B68012283F890227B681B68F9681846E5
:1033900003F039FB7B68002283F890220023184653
:1033A0001037BD4680BD80B596B000AF7860ADE304
:1033B0007B681B68B3F84430A7F84E30B7F84E303E
:1033C000DBB203F00F0387F84D3097F84D30002B38
:1033D00040F06F81B7F84E3003F01003002B4CD152
:1033E0007B681B681B889BB223F4E14323F07003C6
:1033F000FB817B681A68FB896FEA43436FEA53439A
:103400009BB213807B6810337B657B681B68B3F8C5
:1034100050309BB21A467B6D1B78DB0013447A68F0
:103420001268134403F202431B88C3F309027B6D45
:10343000DA617B6D5A697B6DDB691A447B6D5A6179
:1034400000217868FEF709FF7B681B7BDBB2002B4D
:1034500000F05C837B6D9B69002B40F057837B6899
:103460001B7BDBB263F07F03DAB27B681B68A3F8D7
:103470004C207B6800221A7348E37B6803F5A8732D
:103480007B657B681B681B88A7F84A30B7F84A3011
:1034900003F40063002B32D07B681B68B3F8503014
:1034A0009BB21A467B6D1B78DB0013447A68126866
:1034B000134403F206431B88C3F309027B6DDA61F0
:1034C0007B6818687B6803F526717B6DDA887B6DF5
:1034D000DB699BB203F0C2FB7B681B681B889AB256
:1034E00040F68F7313403B827B681B683A8A42F038
:1034F000800292B21A807868FEF782FE06E3B7F97E
:103500004A30002B80F202837B681B681B889AB2CA
:1035100040F68F731340FB837B681B68FA8B42F085
:10352000800292B21A807B681B68B3F850309BB25D
:103530001A467B6D1B78DB0013447A6812681344CB
:1035400003F206431B88C3F309027B6DDA617B6DCE
:10355000DB69002B19D07B6D5B69002B15D07B6874
:1035600018687B6D59697B6DDA887B6DDB699BB26E
:1035700003F074FB7B6D5A697B6DDB691A447B6DCC
:103580005A6100217868FEF74DFE7B681B681B8836
:10359000A7F84A30B7F84A3003F40063002B40F034
:1035A000B582B7F84A3003F44053B3F5405F00F0FA
:1035B000AD827B681B68BB617B681B68B3F85030C9
:1035C0009BB21A46BB691344BB61BB6903F2064355
:1035D0007B617B691B889BB2C3F309039AB27B6949
:1035E0001A807B6D1B693E2B1DD97B6D1B695B09A6
:1035F0007B647B6D1B6903F01F03002B02D17B6C86
:10360000013B7B647B691B889AB27B6C9BB29B02FB
:103610009BB213439BB26FEA43436FEA53439AB2A0
:103620007B691A8026E07B6D1B69002B0AD17B69C0
:103630001B889BB26FEA43436FEA53439AB27B699C
:103640001A8017E07B6D1B695B087B647B6D1B69CF
:1036500003F00103002B02D07B6C01337B647B6998
:103660001B889AB27B6C9BB29B029BB213439AB2AB
:103670007B691A807B681B681B889BB223F480439C
:1036800023F070037B827B8A83F480537B827B8A66
:1036900083F400537B827B681A687B8A43F07F4304
:1036A00043F47F0343F4004343F080039BB2138051
:1036B0002CE27B681B681A4697F84D309B00134438
:1036C0001B88A7F84A30B7F94A30002B80F2F68001
:1036D0007B681B681A4697F84D309B0013441B8883
:1036E0009AB240F68F731340A7F848307B681B6886
:1036F0001A4697F84D309B001344B7F8482042F023
:10370000800292B21A8097F84D2013469B00134412
:10371000DB0003F5A8737A6813447B657B6D1B7B24
:10372000002B23D17B681B68B3F850309BB21A463C
:103730007B6D1B78DB0013447A681268134403F234
:1037400006431B88C3F30903A7F85030B7F850307D
:10375000002B00F08E807B6818687B6D59697B6D4B
:10376000DA88B7F8503003F079FA82E07B6DDB78C5
:10377000022B0AD1B7F84A301A46796D786800F002
:10378000D3F90346A7F8503073E07B681B681A46EC
:103790007B6D1B789B0013441B889BB223F4E04392
:1037A00023F07003A7F852307B681B681A467B6DC4
:1037B0001B789B001A44B7F8523043F07F4343F420
:1037C0007F0343F4004343F0C0039BB213807B6844
:1037D0001B681A467B6D1B789B0013441B889BB2A9
:1037E00003F48043002B22D07B681B68B3F8503071
:1037F0009BB21A467B6D1B78DB0013447A68126813
:10380000134403F202431B88C3F30903A7F85030A3
:10381000B7F85030002B2CD07B6818687B6D596945
:103820007B6D1A89B7F8503003F018FA21E07B68F5
:103830001B68B3F850309BB21A467B6D1B78DB00D7
:1038400013447A681268134403F206431B88C3F3D7
:103850000903A7F85030B7F85030002B09D07B6827
:1038600018687B6D59697B6D5A89B7F8503003F041
:10387000F5F97B6DDA69B7F850301A447B6DDA617F
:103880007B6D5A69B7F850301A447B6D5A617B6D75
:103890009B69002B05D0B7F850207B6D1B699A42BD
:1038A00006D27B6D1B7819467868FEF7BBFC05E0F5
:1038B0007B681B68796D184601F0A3FCB7F84A30A5
:1038C00003F08003002B00F0218197F84D20134670
:1038D0009B001344DB0010337A6813447B657B68DC
:1038E0001B681A4697F84D309B0013441B889BB207
:1038F00023F4E14323F07003A7F842307B681B6890
:103900001A4697F84D309B001A44B7F842306FEAD8
:1039100043436FEA53439BB213807B6DDB78012BEB
:1039200040F0A2807B6D00229A617B6D1B7B002B97
:1039300000F09380B7F84A3003F04003002B46D0E4
:103940007B6D5B78002B26D17B681B687B627B6874
:103950001B68B3F850309BB21A467B6A13447B62F3
:103960007B6D1B78DA007B6A134403F202433B62EF
:103970003B6A1B889BB2C3F309039AB23B6A1A8065
:103980003B6A1B889BB26FEA43436FEA53439AB288
:103990003B6A1A8061E07B6D5B78012B5DD17B68AF
:1039A0001B68FB627B681B68B3F850309BB21A46F9
:1039B000FB6A1344FB627B6D1B78DA00FB6A1344DD
:1039C00003F20243BB62BB6A00221A8045E07B68B7
:1039D0001B68FB637B6D5B78002B26D17B681B68C3
:1039E0007B637B681B68B3F850309BB21A467B6BD5
:1039F00013447B637B6D1B78DA007B6B134403F20B
:103A000006433B633B6B1B889BB2C3F309039AB22B
:103A10003B6B1A803B6B1B889BB26FEA43436FEA98
:103A200053439AB23B6B1A8017E07B6D5B78012B96
:103A300013D17B681B68B3F850309BB21A46FB6BFE
:103A40001344FB637B6D1B78DA00FB6B134403F2BA
:103A50000643BB63BB6B00221A807B6D1B78194643
:103A60007868FEF7FAFB51E0B7F84A3003F4807348
:103A7000002B44D17B681B68B3F850309BB21A46C8
:103A80007B6D1B78DB0013447A681268134403F2E1
:103A900002431B88C3F30903A7F840307B6D9A6982
:103AA000B7F840309A4207D97B6D9A69B7F8403031
:103AB000D21A7B6D9A6102E07B6D00229A617B6D68
:103AC0009B69002B06D17B6D1B7819467868FEF741
:103AD000C4FB1BE07B6D5A69B7F840301A447B6D1C
:103AE0005A617B6DDA69B7F840301A447B6DDA6150
:103AF0007B681B68796D184601F083FB06E0B7F818
:103B00004A301A46796D786800F017F97B681B68AF
:103B1000B3F844309BB21BB2002BFFF649AC002334
:103B200018465837BD4680BD80B588B000AFF860F4
:103B3000B9601346FB80FB8803F48043002B7CD0E4
:103B4000FB681B68B3F850309BB21A46BB681B7801
:103B5000DB001344FA681268134403F202431B8823
:103B6000C3F309037B83BB689A697B8B9A4206D3B4
:103B7000BB689A697B8BD21ABB689A6102E0BB680A
:103B800000229A61BB689B69002B23D1FB681B68EC
:103B90001A46BB681B789B0013441B889BB223F416
:103BA000804323F070033B833B8B83F400533B83C0
:103BB000FB681B681A46BB681B789B001A443B8B4A
:103BC00043F07F4343F47F0343F4004343F0800317
:103BD0009BB21380FB8803F04003002B1FD0FB68CF
:103BE0001B681A46BB681B789B0013441B889BB25A
:103BF00023F4E04323F07003FB82FB681B681A4642
:103C0000BB681B789B001A44FB8A43F07F4343F454
:103C10007F0343F4004343F0C0039BB213807B8BCC
:103C2000002B00F08580FB681868BB685969BB6889
:103C30001A897B8B03F012F87AE0FB681B68B3F8F3
:103C400050309BB21A46BB681B78DB001344FA68FD
:103C50001268134403F206431B88C3F309037B83F2
:103C6000BB689A697B8B9A4206D3BB689A697B8B47
:103C7000D21ABB689A6102E0BB6800229A61BB68F5
:103C80009B69002B23D1FB681B681A46BB681B7815
:103C90009B0013441B889BB223F4804323F07003E2
:103CA000FB83FB8B83F40053FB83FB681B681A4682
:103CB000BB681B789B001A44FB8B43F07F4343F4A3
:103CC0007F0343F4004343F080039BB21380FB88DF
:103CD00003F04003002B1FD1FB681B681A46BB682A
:103CE0001B789B0013441B889BB223F4E04323F012
:103CF0007003BB83FB681B681A46BB681B789B007C
:103D00001A44BB8B43F07F4343F47F0343F40043E7
:103D100043F0C0039BB213807B8B002B08D0FB6861
:103D20001868BB685969BB685A897B8B02F096FF9B
:103D30007B8B18462037BD4680BD80B5A4B000AF50
:103D4000F860B9601346FB80FB8803F04003002B4A
:103D500000F0DB81FB681B68B3F850309BB21A4659
:103D6000BB681B78DB001344FA681268134403F243
:103D700002431B88C3F30903A7F88630BB689A691E
:103D8000B7F886309A4207D9BB689A69B7F8863087
:103D9000D21ABB689A6102E0BB6800229A61BB68D4
:103DA0009B69002B40F0B980BB685B78002B26D163
:103DB000FB681B68FB62FB681B68B3F850309BB262
:103DC0001A46FB6A1344FB62BB681B78DA00FB6A85
:103DD000134403F20243BB62BB6A1B889BB2C3F36A
:103DE00009039AB2BB6A1A80BB6A1B889BB26FEA4E
:103DF00043436FEA53439AB2BB6A1A801AE0BB6826
:103E00005B78012B16D1FB681B687B63FB681B6822
:103E1000B3F850309BB21A467B6B13447B63BB688C
:103E20001B78DA007B6B134403F202433B633B6B6A
:103E300000221A80FB681B687B62BB685B78002BE2
:103E400026D1FB681B68FB61FB681B68B3F8503028
:103E50009BB21A46FB691344FB61BB681B78DA000E
:103E6000FB69134403F20643BB61BB691B889BB229
:103E7000C3F309039AB2BB691A80BB691B889BB262
:103E80006FEA43436FEA53439AB2BB691A8017E063
:103E9000BB685B78012B13D1FB681B68B3F850300B
:103EA0009BB21A467B6A13447B62BB681B78DA00BC
:103EB0007B6A134403F206433B623B6A00221A808A
:103EC000BB681B781946F868FEF7C7F9FB8803F44E
:103ED0008043002B00F0FA82FB681B681A46BB681F
:103EE0001B789B0013441B889BB223F4E04323F010
:103EF0007003FB82FB681B681A46BB681B789B003B
:103F00001A44FB8A43F07F4343F47F0343F4404366
:103F100043F080039BB21380D8E2FB8803F4804314
:103F2000002B21D0FB681B681A46BB681B789B00DE
:103F300013441B889BB223F4E04323F07003A7F8DB
:103F40008A30FB681B681A46BB681B789B001A44C2
:103F5000B7F88A3043F07F4343F47F0343F4404390
:103F600043F080039BB21380BB6893F82430012B8D
:103F700040F0AC82BB685A69B7F886301A44BB6817
:103F80005A61BB68DA69B7F886301A44BB68DA61EF
:103F9000BB681A6ABB681B699A420BD3BB681B6972
:103FA000C7F88C30BB681A6AD7F88C30D21ABB6855
:103FB0001A6217E0BB681B6A002B08D1B7F886307D
:103FC000C7F88C30BB68002283F824200AE0BB6865
:103FD000002283F82420BB681B6AC7F88C30BB68BA
:103FE00000221A62BB685B78002B65D1FB681B68F6
:103FF000FB63FB681B68B3F850309BB21A46FB6B3F
:104000001344FB63BB681B78DA00FB6B134403F2B9
:104010000243BB63BB6B1B889BB2C3F309039AB219
:10402000BB6B1A80D7F88C303E2B1DD9D7F88C305B
:104030005B09BB64D7F88C3003F01F03002B02D15F
:10404000BB6C013BBB64BB6B1B889AB2BB6C9BB265
:104050009B029BB213439BB26FEA43436FEA534305
:104060009AB2BB6B1A8044E0D7F88C30002B0AD18F
:10407000BB6B1B889BB26FEA43436FEA53439AB210
:10408000BB6B1A8035E0D7F88C305B08BB64D7F87F
:104090008C3003F00103002B02D0BB6C0133BB64F6
:1040A000BB6B1B889AB2BB6C9BB29B029BB2134347
:1040B0009AB2BB6B1A801CE0BB685B78012B18D1ED
:1040C000FB681B687B64FB681B68B3F850309BB2CD
:1040D0001A467B6C13447B64BB681B78DA007B6CEC
:1040E000134403F202433B64D7F88C309AB23B6C22
:1040F0001A80FB681868BB685969BB681A89D7F8C9
:104100008C309BB202F068FDE0E1FB681B68B3F8FD
:1041100050309BB21A46BB681B78DB001344FA6828
:104120001268134403F206431B88C3F30903A7F87C
:104130008630BB689A69B7F886309A4207D3BB6865
:104140009A69B7F88630D21ABB689A6102E0BB68F8
:1041500000229A61BB689B69002B40F0C080BB685D
:104160005B78002B26D1FB681B68FB67FB681B682C
:10417000B3F850309BB21A46FB6F1344FB67BB6821
:104180001B78DA00FB6F134403F20243BB67BB6F7B
:104190001B889BB2C3F309039AB2BB6F1A80BB6F33
:1041A0001B889BB26FEA43436FEA53439AB2BB6FDB
:1041B0001A801AE0BB685B78012B16D1FB681B687C
:1041C0007B66FB681B68B3F850309BB21A467B6E67
:1041D00013447B66BB681B78DA007B6E134403F2E2
:1041E00002433B663B6E00221A80FB681B687B67BC
:1041F000BB685B78002B2BD1FB681B68FB66FB68F8
:104200001B68B3F850309BB21A46FB6E1344FB6632
:10421000BB681B78DA00FB6E134403F20643C7F851
:104220008030D7F880301B889BB2C3F309039AB261
:10423000D7F880301A80D7F880301B889BB26FEA9D
:1042400043436FEA53439AB2D7F880301A8017E09D
:10425000BB685B78012B13D1FB681B68B3F8503047
:104260009BB21A467B6F13447B67BB681B78DA00EE
:104270007B6F134403F206433B673B6F00221A80B7
:10428000BB681B781946F868FDF7E7FFFB8803F465
:104290008043002B40F01A81FB681B681A46BB68FC
:1042A0001B789B0013441B889BB223F4E04323F04C
:1042B0007003A7F88830FB681B681A46BB681B7838
:1042C0009B001A44B7F8883043F07F4343F47F03E0
:1042D00043F4404343F080039BB21380F6E0FB8835
:1042E00003F48043002B21D1FB681B681A46BB688E
:1042F0001B789B0013441B889BB223F4E04323F0FC
:104300007003A7F84E30FB681B681A46BB681B7821
:104310009B001A44B7F84E3043F07F4343F47F03C9
:1043200043F4404343F080039BB21380BB6893F88F
:104330002430012B40F0CA80BB685A69B7F8863038
:104340001A44BB685A61BB68DA69B7F886301A4408
:10435000BB68DA61BB681A6ABB681B699A420BD3F7
:10436000BB681B69C7F88C30BB681A6AD7F88C30F9
:10437000D21ABB681A6217E0BB681B6A002B08D10F
:10438000B7F88630C7F88C30BB68002283F8242049
:104390000AE0BB681B6AC7F88C30BB6800221A624F
:1043A000BB68002283F82420FB681B687B65BB6820
:1043B0005B78002B65D1FB681B68FB65FB681B689D
:1043C000B3F850309BB21A46FB6D1344FB65BB68D3
:1043D0001B78DA00FB6D134403F20643BB65BB6D2B
:1043E0001B889BB2C3F309039AB2BB6D1A80D7F83E
:1043F0008C303E2B1DD9D7F88C305B09BB66D7F8C3
:104400008C3003F01F03002B02D1BB6E013BBB6657
:10441000BB6D1B889AB2BB6E9BB29B029BB21343CF
:104420009BB26FEA43436FEA53439AB2BB6D1A8063
:1044300041E0D7F88C30002B0AD1BB6D1B889BB2B2
:104440006FEA43436FEA53439AB2BB6D1A8032E07E
:10445000D7F88C305B08BB66D7F88C3003F00103CB
:10446000002B02D0BB6E0133BB66BB6D1B889AB2BA
:10447000BB6E9BB29B029BB213439AB2BB6D1A8078
:1044800019E0BB685B78012B15D1FB681B68B3F89A
:1044900050309BB21A467B6D13447B65BB681B781A
:1044A000DA007B6D134403F206433B65D7F88C308A
:1044B0009AB23B6D1A80FB681868BB685969BB6883
:1044C0005A89D7F88C309BB202F086FBFB681B68D8
:1044D0001A46BB681B789B0013441B889BB223F4CD
:1044E000E04323F04003BB82BB8A83F01003BB820E
:1044F000BB8A83F02003BB82FB681B681A46BB683B
:104500001B789B001A44BB8A43F07F4343F47F032C
:1045100043F4004343F080039BB21380002318460A
:104520009037BD4680BD80B487B000AFF8607B6037
:104530000B467B8113463B817B8903F080039BB252
:10454000002B0BD07B8903F0070213469B0013441A
:10455000DB001033FA6813447B6109E07A89134663
:104560009B001344DB0003F5A873FA6813447B61D6
:104570003B89002B07D17B6900221A737B689AB2B2
:104580007B69DA800BE07B6901221A737B689AB23F
:104590007B691A817B681B0C9AB27B695A81002364
:1045A00018461C37BD465DF8047B704780B485B063
:1045B00000AF78607B681B68FB607B680122C3F8F2
:1045C000D0227B68002283F8C822FB68B3F85430FD
:1045D0009BB243F001039AB2FB68A3F85420FB6836
:1045E000B3F854309BB243F002039AB2FB68A3F8CD
:1045F0005420002318461437BD465DF8047B7047ED
:1046000080B485B000AF78607B680022A3F84420B6
:104610004BF68073FB60FB689AB27B68A3F840207E
:10462000002318461437BD465DF8047B704780B4FC
:1046300085B000AF78604BF68073FB607B68B3F8A1
:1046400040309AB2FB689BB2DB439BB213409AB2F4
:104650007B68A3F84020002318461437BD465DF858
:10466000047B704780B485B000AFF8603B1D83E8E1
:104670000600FB680122A3F84020FB680022A3F893
:104680004020FB680022A3F84420FB680022A3F826
:104690005020002318461437BD465DF8047B704750
:1046A00080B49DB000AF78603960002387F86F3028
:1046B0007A683B681B789B0013441B889BB223F4E9
:1046C000EC4323F07003A7F86C303B68DB78032BD6
:1046D0001FD801A252F823F0E94601080547010856
:1046E0001B470108F7460108B7F86C3043F4007324
:1046F000A7F86C3012E0B7F86C3043F4C063A7F849
:104700006C300BE0B7F86C3043F48063A7F86C3082
:1047100004E0012387F86F3000E000BF7A683B684F
:104720001B789B001A44B7F86C3043F07F4343F486
:104730007F0343F4004343F080039BB213807A6805
:104740003B681B789B0013441B889BB21BB223F46D
:10475000E04323F070031AB23B681B781BB213438B
:104760001BB2A7F866307A683B681B789B001A4436
:10477000B7F8663043F07F4343F47F0343F40043CC
:1047800043F080039BB213803B681B7B002B40F0FF
:1047900078813B685B78002B00F084807B68BB618C
:1047A0007B68B3F850309BB21A46BB691344BB61B7
:1047B0003B681B78DA00BB69134403F580637B61B7
:1047C0003B68DB885B089BB25B009AB27B691A800E
:1047D0007A683B681B789B0013441B887B827B8A2A
:1047E00003F04003002B1BD07A683B681B789B00CA
:1047F00013441B889BB223F4E04323F070033B82F5
:104800007A683B681B789B001A443B8A43F07F43DD
:1048100043F47F0343F4004343F0C0039BB213808F
:104820003B68DB78012B20D07A683B681B789B00C3
:1048300013441B889BB223F4E04323F04003BB8165
:10484000BB8983F02003BB817A683B681B789B009F
:104850001A44BB8943F07F4343F47F0343F400438E
:1048600043F080039BB21380D5E27A683B681B78E3
:104870009B0013441B889BB223F4E04323F04003C6
:10488000FB817A683B681B789B001A44FB8943F0E4
:104890007F4343F47F0343F4004343F080039BB220
:1048A0001380B8E27B683B637B68B3F850309BB2FF
:1048B0001A463B6B13443B633B681B78DA003B6B47
:1048C000134403F20443FB623B68DB885B089BB242
:1048D0005B009AB2FB6A1A807B68BB627B68B3F8A4
:1048E00050309BB21A46BB6A1344BB623B681B78CC
:1048F000DA00BB6A134403F206437B627B6A1B88BF
:104900009BB2C3F309039AB27B6A1A803B681B69A6
:104910003E2B1DD93B681B695B09BB663B681B6965
:1049200003F01F03002B02D1BB6E013BBB667B6A09
:104930001B889AB2BB6E9BB29B029BB213439BB285
:104940006FEA43436FEA53439AB27B6A1A8026E0C8
:104950003B681B69002B0AD17B6A1B889BB26FEAFC
:1049600043436FEA53439AB27B6A1A8017E03B686D
:104970001B695B08BB663B681B6903F00103002BE6
:1049800002D0BB6E0133BB667B6A1B889AB2BB6EDA
:104990009BB29B029BB213439AB27B6A1A807A68DD
:1049A0003B681B789B0013441B887B847B8C03F43F
:1049B0008043002B1BD07A683B681B789B00134414
:1049C0001B889BB223F4E04323F070033B847A6896
:1049D0003B681B789B001A443B8C43F07F4343F4B5
:1049E0007F0343F4404343F080039BB213803B6852
:1049F0001B78002B24D17A683B681B789B001344FA
:104A00001B889BB223F4804323F07003BB83BB8BD2
:104A100083F48053BB83BB8B83F40053BB837A68DE
:104A20003B681B789B001A44BB8B43F07F4343F4E5
:104A30007F0343F4004343F080039BB21380EAE119
:104A40007A683B681B789B0013441B889BB223F455
:104A5000804323F07003FB83FB8B83F40053FB83C1
:104A60007A683B681B789B001A44FB8B43F07F43BA
:104A700043F47F0343F4004343F080039BB213806D
:104A8000C9E13B68DB78022B1ED17A683B681B7852
:104A90009B0013441B889BB223F4E04323F0700374
:104AA000A7F862307A683B681B789B001A44B7F815
:104AB000623043F07F4343F47F0343F4014343F008
:104AC00080039BB213801DE07A683B681B789B00D3
:104AD00013441B889BB223F4E24323F07003A7F82E
:104AE00064307A683B681B789B001A44B7F86430DE
:104AF00043F07F4343F47F0343F4004343F08003D8
:104B00009BB213807B68FB657B68B3F850309BB227
:104B10001A46FB6D1344FB653B681B78DA00FB6D9E
:104B2000134403F58063BB653B681B895B089BB23C
:104B30005B009AB2BB6D1A807B687B657B68B3F8BB
:104B400050309BB21A467B6D13447B653B681B78E3
:104B5000DA007B6D134403F204433B653B685B89D9
:104B60005B089BB25B009AB23B6D1A803B685B7836
:104B7000002B40F093807A683B681B789B001344BD
:104B80001B88A7F84030B7F8403003F48043002B6F
:104B90001BD07A683B681B789B0013441B889BB230
:104BA00023F4E04323F07003FB877A683B681B78AB
:104BB0009B001A44FB8F43F07F4343F47F0343F48D
:104BC000404343F080039BB213807A683B681B78B4
:104BD0009B0013441B88BB87BB8F03F04003002B53
:104BE0001BD07A683B681B789B0013441B889BB2E0
:104BF00023F4E04323F070037B877A683B681B78DB
:104C00009B001A447B8F43F07F4343F47F0343F4BC
:104C1000004343F0C0039BB213807A683B681B7863
:104C20009B0013441B889BB223F4804323F0700342
:104C30003B873B8F83F480533B873B8F83F4005348
:104C40003B877A683B681B789B001A443B8F43F094
:104C50007F4343F47F0343F4004343F080039BB25C
:104C600013807A683B681B789B0013441B889BB2B7
:104C700023F4E04323F04003FB867A683B681B780B
:104C80009B001A44FB8E43F07F4343F47F0343F4BD
:104C9000004343F080039BB21380BCE07A683B681A
:104CA0001B789B0013441B88A7F84E30B7F84E3092
:104CB00003F48043002B1DD07A683B681B789B006F
:104CC00013441B889BB223F4E04323F07003A7F83E
:104CD0004C307A683B681B789B001A44B7F84C301C
:104CE00043F07F4343F47F0343F4404343F08003A6
:104CF0009BB213807A683B681B789B0013441B8827
:104D0000A7F84A30B7F84A3003F04003002B1DD013
:104D10007A683B681B789B0013441B889BB223F482
:104D2000E04323F07003A7F848307A683B681B78AB
:104D30009B001A44B7F8483043F07F4343F47F03A5
:104D400043F4004343F0C0039BB213803B68DB781D
:104D5000012B24D07A683B681B789B0013441B8886
:104D60009BB223F4E04323F04003A7F84430B7F8A4
:104D7000443083F02003A7F844307A683B681B78FE
:104D80009B001A44B7F8443043F07F4343F47F0359
:104D900043F4004343F080039BB213801DE07A6824
:104DA0003B681B789B0013441B889BB223F4E043B1
:104DB00023F04003A7F846307A683B681B789B00D5
:104DC0001A44B7F8463043F07F4343F47F0343F47B
:104DD000004343F080039BB213807A683B681B78E2
:104DE0009B0013441B889BB223F4804323F0700381
:104DF000A7F842307A683B681B789B001A44B7F8E2
:104E0000423043F07F4343F47F0343F4004343F0D5
:104E100080039BB2138097F86F3018467437BD46F5
:104E20005DF8047B704700BF80B48DB000AF786040
:104E300039603B681B7B002B40F08E803B685B78C1
:104E4000002B44D07A683B681B789B0013441B8876
:104E5000BB81BB8903F04003002B1BD07A683B6801
:104E60001B789B0013441B889BB223F4E04323F080
:104E700070037B817A683B681B789B001A447B89AE
:104E800043F07F4343F47F0343F4004343F0C00304
:104E90009BB213807A683B681B789B0013441B8885
:104EA0009BB223F4E04323F040033B817A683B68E4
:104EB0001B789B001A443B8943F07F4343F47F03F4
:104EC00043F4004343F080039BB2138092E17A687D
:104ED0003B681B789B0013441B887B827B8A03F40E
:104EE0008043002B1BD07A683B681B789B001344DF
:104EF0001B889BB223F4E04323F070033B827A6863
:104F00003B681B789B001A443B8A43F07F4343F481
:104F10007F0343F4404343F080039BB213807A68DD
:104F20003B681B789B0013441B889BB223F480438F
:104F300023F07003FB817A683B681B789B001A445E
:104F4000FB8943F07F4343F47F0343F4004343F082
:104F500080039BB213804DE13B685B78002B40F0EF
:104F6000A5807A683B681B789B0013441B883B84B0
:104F70003B8C03F48043002B1BD07A683B681B7882
:104F80009B0013441B889BB223F4E04323F070037F
:104F9000FB837A683B681B789B001A44FB8B43F0C9
:104FA0007F4343F47F0343F4404343F080039BB2C9
:104FB00013807A683B681B789B0013441B88BB8373
:104FC000BB8B03F04003002B1BD07A683B681B7837
:104FD0009B0013441B889BB223F4E04323F070032F
:104FE0007B837A683B681B789B001A447B8B43F079
:104FF0007F4343F47F0343F4004343F0C0039BB279
:1050000013807A683B681B789B0013441B889BB213
:1050100023F4E04323F070033B837A683B681B78FA
:105020009B001A443B8B43F07F4343F47F0343F4DC
:10503000004343F0C0039BB213807A683B681B783F
:105040009B0013441B889BB223F4804323F070031E
:10505000FB827A683B681B789B001A44FB8A43F00A
:105060007F4343F47F0343F4004343F080039BB248
:1050700013807A683B681B789B0013441B889BB2A3
:1050800023F4E04323F04003BB827A683B681B783B
:105090009B001A44BB8A43F07F4343F47F0343F4ED
:1050A000004343F080039BB21380A3E07A683B681F
:1050B0001B789B0013441B88FB85FB8D03F4804306
:1050C000002B1BD07A683B681B789B0013441B881D
:1050D0009BB223F4E04323F07003BB857A683B68FE
:1050E0001B789B001A44BB8D43F07F4343F47F033E
:1050F00043F4404343F080039BB213807A683B68DB
:105100001B789B0013441B887B857B8D03F0400339
:10511000002B1BD07A683B681B789B0013441B88CC
:105120009BB223F4E04323F070033B857A683B682D
:105130001B789B001A443B8D43F07F4343F47F036D
:1051400043F4004343F0C0039BB213807A683B688A
:105150001B789B0013441B889BB223F4E04323F08D
:105160007003FB847A683B681B789B001A44FB8CB5
:1051700043F07F4343F47F0343F4404343F0800311
:105180009BB213807A683B681B789B0013441B8892
:105190009BB223F4E04323F04003BB847A683B686E
:1051A0001B789B001A44BB8C43F07F4343F47F037E
:1051B00043F4004343F080039BB213807A683B685A
:1051C0001B789B0013441B889BB223F4804323F07D
:1051D00070037B847A683B681B789B001A447B8C45
:1051E00043F07F4343F47F0343F4004343F08003E1
:1051F0009BB21380002318463437BD465DF8047B0C
:10520000704780B5C2B000AF07F58473A3F5827311
:10521000186007F58473A3F58473196007F5847328
:10522000A3F584731B685B78012B40F0B78607F504
:105230008473A3F584731B689A6907F58473A3F5D7
:1052400084731B681B699A4208D907F58473A3F518
:1052500084731B681B69C7F8043107E007F5847382
:10526000A3F584731B689B69C7F8043107F5847341
:10527000A3F584731B681B7B002B3AD107F584735D
:10528000A3F584731B68596907F58473A3F58473C8
:105290001B68DA88D7F804319BB207F58470A0F553
:1052A0008270006801F098FC07F58473A3F582739F
:1052B0001B683B6107F58473A3F582731B68B3F821
:1052C00050309BB21A463B6913443B6107F5847327
:1052D000A3F584731B681B78DA003B69134403F25F
:1052E0000243FB60D7F804319AB2FB681A8000F0E1
:1052F0001FBE07F58473A3F584731B68DB78022B4C
:1053000040F0628407F58473A3F584731B681A6AFE
:1053100007F58473A3F584731B681B699A4240F2F6
:10532000DF8307F58473A3F582731A6807F5847326
:10533000A3F584731B681B789B0013441B889BB2E6
:1053400023F4E04323F07003A7F8563007F5847385
:10535000A3F582731A6807F58473A3F584731B6839
:105360001B789B001A44B7F8563043F07F4343F450
:105370007F0343F4014343F080039BB2138007F59E
:105380008473A3F584731B681A6AD7F80431D21AA0
:1053900007F58473A3F584731B681A6207F5847399
:1053A000A3F582731A6807F58473A3F584731B68E9
:1053B0001B789B0013441B889BB203F04003002B17
:1053C00000F0C78107F58473A3F582731B683B6304
:1053D00007F58473A3F584731B685B78002B77D182
:1053E00007F58473A3F582731B68BB6207F58473AA
:1053F000A3F582731B68B3F850309BB21A46BB6AA0
:105400001344BB6207F58473A3F584731B681B7890
:10541000DA00BB6A134403F206437B627B6A1B8893
:105420009BB2C3F309039AB27B6A1A80D7F804319E
:105430003E2B21D9D7F804315B09C7F80031D7F8E2
:10544000043103F01F03002B04D1D7F80031013BD6
:10545000C7F800317B6A1B889AB2D7F800319BB23B
:105460009B029BB213439BB26FEA43436FEA5343E1
:105470009AB27B6A1A8050E0D7F80431002B0AD127
:105480007B6A1B889BB26FEA43436FEA53439AB22D
:105490007B6A1A8041E0D7F804315B08C7F8003115
:1054A000D7F8043103F00103002B04D0D7F8003102
:1054B0000133C7F800317B6A1B889AB2D7F80031F4
:1054C0009BB29B029BB213439AB27B6A1A8024E080
:1054D00007F58473A3F584731B685B78012B1CD1DB
:1054E00007F58473A3F582731B68B3F850309BB241
:1054F0001A463B6B13443B6307F58473A3F584732F
:105500001B681B78DA003B6B134403F20643FB6213
:10551000D7F804319AB2FB6A1A8007F58473A3F5B1
:1055200084731B685B89A7F8763007F58473A3F54D
:1055300084731B685969D7F804319BB2B7F8762099
:1055400007F58470A0F58270006801F045FB07F54F
:105550008473A3F584731B685A69D7F804311A441D
:1055600007F58473A3F584731B685A6107F5847388
:10557000A3F584731B681A6A07F58473A3F5847313
:105580001B681B699A420FD907F58473A3F58473CE
:105590001B681A6AD7F80431D21A07F58473A3F589
:1055A00084731B681A620EE007F58473A3F5847395
:1055B0001B681B6AC7F8043107F58473A3F584736D
:1055C0001B6800221A6207F58473A3F584731B68B5
:1055D0005B78002B77D107F58473A3F582731B6882
:1055E000BB6107F58473A3F582731B68B3F8503071
:1055F0009BB21A46BB691344BB6107F58473A3F5DC
:1056000084731B681B78DA00BB69134403F20243FE
:105610007B617B691B889BB2C3F309039AB27B69E8
:105620001A80D7F804313E2B21D9D7F804315B0911
:10563000C7F8FC30D7F8043103F01F03002B04D166
:10564000D7F8FC30013BC7F8FC307B691B889AB265
:10565000D7F8FC309BB29B029BB213439BB26FEA1C
:1056600043436FEA53439AB27B691A8056E0D7F8F6
:105670000431002B0AD17B691B889BB26FEA43433C
:105680006FEA53439AB27B691A8047E0D7F8043136
:105690005B08C7F8FC30D7F8043103F00103002B96
:1056A00004D0D7F8FC300133C7F8FC307B691B8885
:1056B0009AB2D7F8FC309BB29B029BB213439AB2CA
:1056C0007B691A802AE007F58473A3F584731B684D
:1056D0005B78012B22D107F58473A3F582731B68D5
:1056E0003B6207F58473A3F582731B68B3F85030EF
:1056F0009BB21A463B6A13443B6207F58473A3F5D9
:1057000084731B681B78DA003B6A134403F202437C
:10571000FB61D7F804319AB2FB691A8007F58473EC
:10572000A3F584731B681B89A7F8763007F584738B
:10573000A3F584731B685969D7F804319BB2B7F895
:10574000762007F58470A0F58270006801F044FAB5
:10575000EEE307F58473A3F584731B685B78002B75
:1057600077D107F58473A3F582731B68BB6407F5D3
:105770008473A3F582731B68B3F850309BB21A464A
:10578000BB6C1344BB6407F58473A3F584731B6877
:105790001B78DA00BB6C134403F202437B647B6C1E
:1057A0001B889BB2C3F309039AB27B6C1A80D7F8AB
:1057B00004313E2B21D9D7F804315B09C7F8F83002
:1057C000D7F8043103F01F03002B04D1D7F8F830C9
:1057D000013BC7F8F8307B6C1B889AB2D7F8F830D9
:1057E0009BB29B029BB213439BB26FEA43436FEAA7
:1057F00053439AB27B6C1A8056E0D7F80431002BE1
:105800000AD17B6C1B889BB26FEA43436FEA534318
:105810009AB27B6C1A8047E0D7F804315B08C7F86E
:10582000F830D7F8043103F00103002B04D0D7F887
:10583000F8300133C7F8F8307B6C1B889AB2D7F880
:10584000F8309BB29B029BB213439AB27B6C1A80D6
:105850002AE007F58473A3F584731B685B78012B3A
:1058600022D107F58473A3F582731B683B6507F5A6
:105870008473A3F582731B68B3F850309BB21A4649
:105880003B6D13443B6507F58473A3F584731B6874
:105890001B78DA003B6D134403F20243FB64D7F834
:1058A00004319AB2FB6C1A8007F58473A3F58473F4
:1058B0001B681B89A7F8763007F58473A3F58473FA
:1058C0001B685969D7F804319BB2B7F8762007F501
:1058D0008470A0F58270006801F07EF907F584738A
:1058E000A3F584731B685A69D7F804311A4407F585
:1058F0008473A3F584731B685A6107F58473A3F559
:1059000084731B681A6A07F58473A3F584731B6894
:105910001B699A420FD907F58473A3F584731B683A
:105920001A6AD7F80431D21A07F58473A3F5847381
:105930001B681A620EE007F58473A3F584731B6875
:105940001B6AC7F8043107F58473A3F584731B68D9
:1059500000221A6207F58473A3F582731B683B6407
:1059600007F58473A3F584731B685B78002B77D1EC
:1059700007F58473A3F582731B68BB6307F5847313
:10598000A3F582731B68B3F850309BB21A46BB6B09
:105990001344BB6307F58473A3F584731B681B78FA
:1059A000DA00BB6B134403F206437B637B6B1B88FB
:1059B0009BB2C3F309039AB27B6B1A80D7F8043108
:1059C0003E2B21D9D7F804315B09C7F8F430D7F85A
:1059D000043103F01F03002B04D1D7F8F430013B4E
:1059E000C7F8F4307B6B1B889AB2D7F8F4309BB2BF
:1059F0009B029BB213439BB26FEA43436FEA53434C
:105A00009AB27B6B1A8050E0D7F80431002B0AD190
:105A10007B6B1B889BB26FEA43436FEA53439AB296
:105A20007B6B1A8041E0D7F804315B08C7F8F4308B
:105A3000D7F8043103F00103002B04D0D7F8F43079
:105A40000133C7F8F4307B6B1B889AB2D7F8F43077
:105A50009BB29B029BB213439AB27B6B1A8024E0E9
:105A600007F58473A3F584731B685B78012B1CD145
:105A700007F58473A3F582731B68B3F850309BB2AB
:105A80001A463B6C13443B6407F58473A3F5847397
:105A90001B681B78DA003B6C134403F20643FB637C
:105AA000D7F804319AB2FB6B1A8007F58473A3F51B
:105AB00084731B685B89A7F8763007F58473A3F5B8
:105AC00084731B685969D7F804319BB2B7F8762004
:105AD00007F58470A0F58270006801F07DF827E278
:105AE00007F58473A3F584731B681B6AC7F8043138
:105AF00007F58473A3F582731A6807F58473A3F519
:105B000084731B681B789B0013441B889BB223F48F
:105B1000E24323F07003A7F8623007F58473A3F51E
:105B200082731A6807F58473A3F584731B681B7866
:105B30009B001A44B7F8623043F07F4343F47F037D
:105B400043F4004343F080039BB2138007F5847352
:105B5000A3F582731B68FB6507F58473A3F5827355
:105B60001B68B3F850309BB21A46FB6D1344FB65BB
:105B700007F58473A3F584731B681B78DA00FB6D4B
:105B8000134403F20243BB65D7F804319AB2BB6DEC
:105B90001A8007F58473A3F584731B681B89A7F823
:105BA000763007F58473A3F584731B685969D7F8B9
:105BB00004319BB2B7F8762007F58470A0F58270A7
:105BC000006801F009F8B3E107F58473A3F5847365
:105BD0001B681A6AD7F80431D21A07F58473A3F543
:105BE00084731B681A6207F58473A3F582731A68BD
:105BF00007F58473A3F584731B681B789B0013441B
:105C00001B889BB203F04003002B00F0C68007F511
:105C10008473A3F582731B683B6707F58473A3F550
:105C200084731B685B78002B77D107F58473A3F529
:105C300082731B68BB6607F58473A3F582731B68C8
:105C4000B3F850309BB21A46BB6E1344BB6607F5DF
:105C50008473A3F584731B681B78DA00BB6E13444E
:105C600003F206437B667B6E1B889BB2C3F309037A
:105C70009AB27B6E1A80D7F804313E2B21D9D7F81F
:105C800004315B09C7F8F030D7F8043103F01F0383
:105C9000002B04D1D7F8F030013BC7F8F0307B6E11
:105CA0001B889AB2D7F8F0309BB29B029BB2134389
:105CB0009BB26FEA43436FEA53439AB27B6E1A80FA
:105CC00050E0D7F80431002B0AD17B6E1B889BB2C1
:105CD0006FEA43436FEA53439AB27B6E1A8041E006
:105CE000D7F804315B08C7F8F030D7F8043103F077
:105CF0000103002B04D0D7F8F0300133C7F8F0309F
:105D00007B6E1B889AB2D7F8F0309BB29B029BB295
:105D100013439AB27B6E1A8024E007F58473A3F5CF
:105D200084731B685B78012B1CD107F58473A3F582
:105D300082731B68B3F850309BB21A463B6F134412
:105D40003B6707F58473A3F584731B681B78DA003F
:105D50003B6F134403F20643FB66D7F804319AB253
:105D6000FB6E1A8007F58473A3F584731B685B8947
:105D7000A7F8763007F58473A3F584731B68596917
:105D8000D7F804319BB2B7F8762007F58470A0F5F8
:105D90008270006800F020FFCAE007F58473A3F565
:105DA00084731B685B78002B77D107F58473A3F5A8
:105DB00082731B68FB6707F58473A3F582731B6806
:105DC000B3F850309BB21A46FB6F1344FB6707F5DC
:105DD0008473A3F584731B681B78DA00FB6F13448C
:105DE00003F20243BB67BB6F1B889BB2C3F309037B
:105DF0009AB2BB6F1A80D7F804313E2B21D9D7F85D
:105E000004315B09C7F8EC30D7F8043103F01F0305
:105E1000002B04D1D7F8EC30013BC7F8EC30BB6F56
:105E20001B889AB2D7F8EC309BB29B029BB213430B
:105E30009BB26FEA43436FEA53439AB2BB6F1A8037
:105E40005CE0D7F80431002B0AD1BB6F1B889BB2F2
:105E50006FEA43436FEA53439AB2BB6F1A804DE037
:105E6000D7F804315B08C7F8EC30D7F8043103F0F9
:105E70000103002B04D0D7F8EC300133C7F8EC3025
:105E8000BB6F1B889AB2D7F8EC309BB29B029BB2D7
:105E900013439AB2BB6F1A8030E007F58473A3F501
:105EA00084731B685B78012B28D107F58473A3F5F5
:105EB00082731B68C7F8843007F58473A3F5827377
:105EC0001B68B3F850309BB21A46D7F8843013449D
:105ED000C7F8843007F58473A3F584731B681B78B7
:105EE000DA00D7F88430134403F20243C7F8803055
:105EF000D7F804319AB2D7F880301A8007F5847346
:105F0000A3F584731B681B89A7F8763007F58473A3
:105F1000A3F584731B685969D7F804319BB2B7F8AD
:105F2000762007F58470A0F58270006800F054FEBA
:105F300007F58473A3F582731A6807F58473A3F5D4
:105F400084731B681B789B0013441B889BB223F44B
:105F5000E04323F040037B817B8983F010037B8146
:105F60007B8983F020037B8107F58473A3F582731B
:105F70001A6807F58473A3F584731B681B789B006C
:105F80001A447B8943F07F4343F47F0343F4004387
:105F900043F080039BB2138000F0DEBC07F58473EE
:105FA000A3F584731B681B7B002B40F0BB8007F5B7
:105FB0008473A3F584731B689A6907F58473A3F54A
:105FC00084731B681B699A4217D907F58473A3F57C
:105FD00084731B681B69C7F8043107F58473A3F544
:105FE00084731B689A69D7F80431D21A07F5847351
:105FF000A3F584731B689A610EE007F58473A3F51B
:1060000084731B689B69C7F8043107F58473A3F593
:1060100084731B6800229A6107F58473A3F5827369
:106020001B68C7F8903007F58473A3F582731B686B
:10603000B3F850309BB21A46D7F890301344C7F8E3
:10604000903007F58473A3F584731B681B78DA001E
:10605000D7F89030134403F20643C7F88C30D7F8D2
:106060008C301B889BB2C3F309039AB2D7F88C30EB
:106070001A80D7F804313E2B24D9D7F804315B09B4
:10608000C7F8E830D7F8043103F01F03002B04D120
:10609000D7F8E830013BC7F8E830D7F88C301B88D8
:1060A0009AB2D7F8E8309BB29B029BB213439BB2E3
:1060B0006FEA43436FEA53439AB2D7F88C301A80A1
:1060C00000F010BCD7F80431002B0CD1D7F88C307D
:1060D0001B889BB26FEA43436FEA53439AB2D7F8E7
:1060E0008C301A80FEE3D7F804315B08C7F8E8303B
:1060F000D7F8043103F00103002B04D0D7F8E830BF
:106100000133C7F8E830D7F88C301B889AB2D7F83B
:10611000E8309BB29B029BB213439AB2D7F88C3003
:106120001A80DFE307F58473A3F584731B68DB78BB
:10613000022B40F0188207F58473A3F584731B6863
:106140005B78002B40F09D8007F58473A3F5827384
:106150001B68C7F8AC3007F58473A3F582731B681E
:10616000B3F850309BB21A46D7F8AC301344C7F896
:10617000AC3007F58473A3F584731B681B78DA00D1
:10618000D7F8AC30134403F20243C7F8A830D7F86D
:10619000A8301B889BB2C3F309039AB2D7F8A83082
:1061A0001A8007F58473A3F584731B681B693E2B63
:1061B0002BD907F58473A3F584731B681B695B09EE
:1061C000C7F8E43007F58473A3F584731B681B6973
:1061D00003F01F03002B04D1D7F8E430013BC7F8CC
:1061E000E430D7F8A8301B889AB2D7F8E4309BB2D5
:1061F0009B029BB213439BB26FEA43436FEA534344
:106200009AB2D7F8A8301A8070E007F58473A3F526
:1062100084731B681B69002B0CD1D7F8A8301B882E
:106220009BB26FEA43436FEA53439AB2D7F8A83060
:106230001A805BE007F58473A3F584731B681B6900
:106240005B08C7F8E43007F58473A3F584731B6813
:106250001B6903F00103002B04D0D7F8E4300133AD
:10626000C7F8E430D7F8A8301B889AB2D7F8E430E2
:106270009BB29B029BB213439AB2D7F8A8301A8004
:1062800034E007F58473A3F584731B685B78012BF6
:106290002CD107F58473A3F582731B68C7F8B4305B
:1062A00007F58473A3F582731B68B3F850309BB273
:1062B0001A46D7F8B4301344C7F8B43007F58473DE
:1062C000A3F584731B681B78DA00D7F8B430134445
:1062D00003F20243C7F8B03007F58473A3F5847363
:1062E0001B681B699AB2D7F8B0301A8007F584731F
:1062F000A3F582731B68C7F8A43007F58473A3F570
:1063000084731B685B78002B40F09D8007F58473D5
:10631000A3F582731B68C7F89C3007F58473A3F557
:1063200082731B68B3F850309BB21A46D7F89C3082
:106330001344C7F89C3007F58473A3F584731B6876
:106340001B78DA00D7F89C30134403F20643C7F8F1
:106350009830D7F898301B889BB2C3F309039AB2E0
:10636000D7F898301A8007F58473A3F584731B68F7
:106370001B693E2B2BD907F58473A3F584731B6827
:106380001B695B09C7F8E03007F58473A3F58473D4
:106390001B681B6903F01F03002B04D1D7F8E03002
:1063A000013BC7F8E030D7F898301B889AB2D7F88D
:1063B000E0309BB29B029BB213439BB26FEA434314
:1063C0006FEA53439AB2D7F898301A8069E007F51C
:1063D0008473A3F584731B681B69002B0CD1D7F859
:1063E00098301B889BB26FEA43436FEA53439AB2DB
:1063F000D7F898301A8054E007F58473A3F58473B6
:106400001B681B695B08C7F8E03007F58473A3F5C8
:1064100084731B681B6903F00103002B04D0D7F8B9
:10642000E0300133C7F8E030D7F898301B889AB2D3
:10643000D7F8E0309BB29B029BB213439AB2D7F8D5
:1064400098301A802DE007F58473A3F584731B68D8
:106450005B78012B25D107F58473A3F582731B6844
:10646000B3F850309BB21A46D7F8A4301344C7F89B
:10647000A43007F58473A3F584731B681B78DA00D6
:10648000D7F8A430134403F20643C7F8A03007F549
:106490008473A3F584731B681B699AB2D7F8A03084
:1064A0001A8007F58473A3F584731B68DB69002BDE
:1064B00000F0188207F58473A3F582731A6807F554
:1064C0008473A3F584731B681B789B0013441B889B
:1064D000A7F89630B7F8963003F48043002B05D028
:1064E000B7F8963003F04003002B0DD1B7F8963083
:1064F00003F48043002B40F0F581B7F8963003F0A9
:106500004003002B40F0EE8107F58473A3F58273FE
:106510001A6807F58473A3F584731B681B789B00C6
:1065200013441B889BB223F4E04323F07003A7F8C5
:10653000943007F58473A3F582731A6807F58473A2
:10654000A3F584731B681B789B001A44B7F894303A
:1065500043F07F4343F47F0343F4004343F0C0031D
:106560009BB21380BEE107F58473A3F584731B68A7
:10657000DB78012B40F0B48107F58473A3F58473B5
:106580001B689A6907F58473A3F584731B681B69FC
:106590009A4217D907F58473A3F584731B681B69A6
:1065A000C7F8043107F58473A3F584731B689A69EF
:1065B000D7F80431D21A07F58473A3F584731B68E6
:1065C0009A610EE007F58473A3F584731B689B69D9
:1065D000C7F8043107F58473A3F584731B680022A0
:1065E0009A6107F58473A3F584731B685B78002BAD
:1065F00040F0858007F58473A3F582731B68C7F8A4
:10660000CC3007F58473A3F582731B68B3F8503060
:106610009BB21A46D7F8CC301344C7F8CC3007F5F4
:106620008473A3F584731B681B78DA00D7F8CC3029
:10663000134403F20243C7F8C830D7F8C8301B88A8
:106640009BB2C3F309039AB2D7F8C8301A80D7F8BF
:1066500004313E2B23D9D7F804315B09C7F8DC306D
:10666000D7F8043103F01F03002B04D1D7F8DC3036
:10667000013BC7F8DC30D7F8C8301B889AB2D7F88E
:10668000DC309BB29B029BB213439BB26FEA434345
:106690006FEA53439AB2D7F8C8301A8060E0D7F84F
:1066A0000431002B0CD1D7F8C8301B889BB26FEA9D
:1066B00043436FEA53439AB2D7F8C8301A804FE089
:1066C000D7F804315B08C7F8DC30D7F8043103F0A1
:1066D0000103002B04D0D7F8DC300133C7F8DC30DD
:1066E000D7F8C8301B889AB2D7F8DC309BB29B022F
:1066F0009BB213439AB2D7F8C8301A8030E007F53E
:106700008473A3F584731B685B78012B28D107F58C
:106710008473A3F582731B68C7F8D43007F58473BC
:10672000A3F582731B68B3F850309BB21A46D7F8B2
:10673000D4301344C7F8D43007F58473A3F58473B9
:106740001B681B78DA00D7F8D430134403F20243F5
:10675000C7F8D030D7F804319AB2D7F8D0301A80C1
:1067600007F58473A3F582731B68C7F8C43007F577
:106770008473A3F584731B685B78002B40F08580DD
:1067800007F58473A3F582731B68C7F8BC3007F55F
:106790008473A3F582731B68B3F850309BB21A461A
:1067A000D7F8BC301344C7F8BC3007F58473A3F5A1
:1067B00084731B681B78DA00D7F8BC30134403F2EB
:1067C0000643C7F8B830D7F8B8301B889BB2C3F37C
:1067D00009039AB2D7F8B8301A80D7F804313E2BA3
:1067E00023D9D7F804315B09C7F8D830D7F804317A
:1067F00003F01F03002B04D1D7F8D830013BC7F8B2
:10680000D830D7F8B8301B889AB2D7F8D8309BB2B6
:106810009B029BB213439BB26FEA43436FEA53431D
:106820009AB2D7F8B8301A805CE0D7F80431002B60
:106830000CD1D7F8B8301B889BB26FEA43436FEA9C
:1068400053439AB2D7F8B8301A804BE0D7F80431E6
:106850005B08C7F8D830D7F8043103F00103002BE8
:1068600004D0D7F8D8300133C7F8D830D7F8B830CB
:106870001B889AB2D7F8D8309BB29B029BB21343C5
:106880009AB2D7F8B8301A802CE007F58473A3F5D4
:1068900084731B685B78012B24D107F58473A3F5FF
:1068A00082731B68B3F850309BB21A46D7F8C430D5
:1068B0001344C7F8C43007F58473A3F584731B68C9
:1068C0001B78DA00D7F8C430134403F20643C7F844
:1068D000C030D7F804319AB2D7F8C0301A8001E03E
:1068E00001233AE007F58473A3F582731A6807F56C
:1068F0008473A3F584731B681B789B0013441B8867
:106900009BB223F4804323F07003A7F88A30B7F8D2
:106910008A3083F48053A7F88A30B7F88A3083F43A
:106920000053A7F88A3007F58473A3F582731A68B9
:1069300007F58473A3F584731B681B789B001A44C6
:10694000B7F88A3043F07F4343F47F0343F40043B6
:1069500043F080039BB213800023184607F5847729
:10696000BD4680BD80B485B000AF786039603B68BB
:106970005B78002B20D07A683B681B789B0013441F
:106980001B889BB223F4E04323F04003BB81BB8907
:1069900083F01003BB817A683B681B789B001A4424
:1069A000BB8943F07F4343F47F0343F4004343F048
:1069B00080039BB213801FE07A683B681B789B00C2
:1069C00013441B889BB223F4804323F07003FB81A4
:1069D000FB8983F48053FB817A683B681B789B00BA
:1069E0001A44FB8943F07F4343F47F0343F400439D
:1069F00043F080039BB21380002318461437BD4632
:106A00005DF8047B704780B487B000AF7860396070
:106A10003B681B7B002B40F09D803B685B78002B24
:106A20004CD07A683B681B789B0013441B883B82E0
:106A30003B8A03F04003002B1BD07A683B681B782D
:106A40009B0013441B889BB223F4E04323F07003A4
:106A5000FB817A683B681B789B001A44FB8943F0F2
:106A60007F4343F47F0343F4004343F0C0039BB2EE
:106A700013803B68DB78012B6CD07A683B681B780D
:106A80009B0013441B889BB223F4E04323F0400394
:106A9000BB81BB8983F02003BB817A683B681B788C
:106AA0009B001A44BB8943F07F4343F47F0343F4C4
:106AB000004343F080039BB213804BE07A683B684D
:106AC0001B789B0013441B88FB82FB8A03F48043E2
:106AD000002B1BD07A683B681B789B0013441B88F3
:106AE0009BB223F4E04323F07003BB827A683B68D7
:106AF0001B789B001A44BB8A43F07F4343F47F0317
:106B000043F4404343F080039BB213807A683B68B0
:106B10001B789B0013441B889BB223F4804323F013
:106B200070037B827B8A83F480537B827B8A83F42D
:106B300000537B827A683B681B789B001A447B8AEF
:106B400043F07F4343F47F0343F4004343F0800367
:106B50009BB21380002318461C37BD465DF8047BAA
:106B6000704780B483B000AF78600B46FB70FB7851
:106B7000002B03D17B688022A3F84C200023184609
:106B80000C37BD465DF8047B704780B483B000AF1E
:106B900078607B68B3F858309BB26FEA43436FEA82
:106BA00053439AB27B68A3F85820002318460C3749
:106BB000BD465DF8047B704780B485B000AF786057
:106BC0007B68B3F844309BB2FB60FB68184614370F
:106BD000BD465DF8047B704780B48BB000AFF860B1
:106BE000B96011461A460B46FB801346BB80BB8832
:106BF00001335B08BB61FB687B61BB68FB61FA88A2
:106C00007B69134403F580633B62BB697B621BE0D5
:106C1000FB691B787B82FB6901331B781B021AB26C
:106C2000B7F9123013431BB27B823B6A7A8A1A800F
:106C30003B6A02333B62FB690133FB61FB69013351
:106C4000FB617B6A013B7B627B6A002BE0D100BF6A
:106C500000BF2C37BD465DF8047B704780B48BB015
:106C600000AFF860B96011461A460B46FB80134628
:106C7000BB80BB885B089BB2BB61FB687B61BB6868
:106C8000FB61FA887B69134403F580633B62BB694F
:106C90007B6218E03B6A1B889BB23B613B6A023314
:106CA0003B623B69DAB2FB691A70FB690133FB6135
:106CB0003B691B0ADAB2FB691A70FB690133FB619D
:106CC0007B6A013B7B627B6A002BE3D1BB8803F0CC
:106CD00001039BB2002B07D03B6A1B889BB23B6130
:106CE0003B69DAB2FB691A7000BF2C37BD465DF80C
:106CF000047B704780B582B000AF0023FB71032096
:106D000001F070FD0F2000F00DF80346002B02D0BB
:106D10000123FB7101E0FBF713FAFB7918460837F2
:106D2000BD4680BD80B584B000AF78600023FB73A2
:106D3000164B1B68002B22D0154B1A68134B1B688F
:106D40004FF47A71B1FBF3F3B2FBF3F3184601F0A1
:106D50007CFD0346002B0FD17B680F2B09D8002246
:106D600079684FF0FF3001F048FD0A4A7B681360F4
:106D700007E00123FB7304E00123FB7301E001231F
:106D8000FB73FB7B18461037BD4680BDBC0000205E
:106D9000C0000020B800002080B400AF054B1A6886
:106DA000054B1B681344034A136000BFBD465DF8E2
:106DB000047B7047E0220020BC00002080B400AFBC
:106DC000034B1B681846BD465DF8047B704700BF47
:106DD000E022002080B588B000AF78607B68002B8F
:106DE00001D10123FEE27B681B6803F00103002B45
:106DF00075D0974B9B6803F00C03BB61944BDB6829
:106E000003F003037B61BB690C2B02D17B69032B6D
:106E100002D0BB69082B0BD18D4B1B6803F40033E8
:106E2000002B5BD07B685B68002B57D10123D9E234
:106E30007B685B68B3F5803F06D1854B1B68844A4D
:106E400043F4803313601DE07B685B68B3F5A02FCB
:106E50000CD17F4B1B687E4A43F4802313607C4B2C
:106E60001B687B4A43F4803313600BE0784B1B684C
:106E7000774A23F480331360754B1B68744A23F4FC
:106E8000802313607B685B68002B13D0FFF796FFAD
:106E9000386108E0FFF792FF02463B69D31A642B82
:106EA00001D903239EE26A4B1B6803F40033002BD5
:106EB000F0D014E0FFF782FF386108E0FFF77EFFB3
:106EC00002463B69D31A642B01D903238AE2604B43
:106ED0001B6803F40033002BF0D100E000BF7B6897
:106EE0001B6803F00203002B75D0594B9B6803F01D
:106EF0000C03BB61564BDB6803F003037B61BB698A
:106F00000C2B02D17B69022B02D0BB69042B1FD151
:106F10004F4B1B6803F48063002B05D07B68DB6854
:106F2000002B01D101235DE2494B5B6823F0FE4257
:106F30007B681B691B06464913434B60454B1B6826
:106F40001846FFF7EFFE0346002B43D0012349E22A
:106F50007B68DB68002B23D03D4B1B683C4A43F425
:106F600080731360FFF72AFF386108E0FFF726FF00
:106F700002463B69D31A022B01D9032332E2344B78
:106F80001B6803F48063002BF0D0314B5B6823F067
:106F9000FE427B681B691B062D4913434B601AE0B8
:106FA0002B4B1B682A4A23F480731360FFF706FFFC
:106FB000386108E0FFF702FF02463B69D31A022B53
:106FC00001D903230EE2224B1B6803F48063002BDC
:106FD000F0D100E000BF7B681B6803F00803002BC2
:106FE00041D07B685B69002B1CD0194BD3F89430DF
:106FF000174A43F00103C2F89430FFF7DFFE38610F
:1070000008E0FFF7DBFE02463B69D31A022B01D9E9
:107010000323E7E10E4BD3F8943003F00203002B77
:10702000EFD020E00A4BD3F89430094A23F0010353
:10703000C2F89430FFF7C2FE38610DE0FFF7BEFEE4
:1070400002463B69D31A022B06D90323CAE100BFCB
:1070500000100240B80000208C4BD3F8943003F0AD
:107060000203002BEAD17B681B6803F00403002BAA
:1070700000F0A6800023FB77844B9B6D03F08053C8
:10708000002B01D1012300E00023002B0DD07F4B0A
:107090009B6D7E4A43F0805393657C4B9B6D03F060
:1070A0008053FB60FB680123FB77794B1B6803F47B
:1070B0008073002B18D1764B1B68754A43F480739C
:1070C0001360FFF77BFE386108E0FFF777FE0246AA
:1070D0003B69D31A022B01D9032383E16C4B1B6854
:1070E00003F48073002BF0D07B689B68012B08D1E0
:1070F000664BD3F89030654A43F00103C2F89030F4
:1071000024E07B689B68052B10D1604BD3F890304E
:107110005E4A43F00403C2F890305C4BD3F89030E1
:107120005A4A43F00103C2F890300FE0574BD3F8AE
:107130009030564A23F00103C2F89030534BD3F8F5
:107140009030524A23F00403C2F890307B689B6869
:10715000002B16D0FFF732FE38610AE0FFF72EFE53
:1071600002463B69D31A41F28832934201D9032384
:1071700038E1464BD3F8903003F00203002BEDD0FA
:1071800015E0FFF71BFE38610AE0FFF717FE024625
:107190003B69D31A41F28832934201D9032321E19A
:1071A0003A4BD3F8903003F00203002BEDD1FB7F74
:1071B000012B05D1354B9B6D344A23F080539365E9
:1071C0007B681B6803F02003002B3CD07B689B6925
:1071D000002B1CD02D4BD3F898302C4A43F00103E0
:1071E000C2F89830FFF7EAFD386108E0FFF7E6FDE6
:1071F00002463B69D31A022B01D90323F2E0234B49
:10720000D3F8983003F00203002BEFD01BE01F4BA4
:10721000D3F898301D4A23F00103C2F89830FFF7E5
:10722000CDFD386108E0FFF7C9FD02463B69D31A7E
:10723000022B01D90323D5E0144BD3F8983003F087
:107240000203002BEFD17B68DB69002B00F0C980C3
:107250000E4B9B6803F00C030C2B00F083807B68C3
:10726000DB69022B5ED1094B1B68084A23F080734F
:107270001360FFF7A3FD38610CE0FFF79FFD0246A6
:107280003B69D31A022B05D90323ABE0001002405F
:1072900000700040554B1B6803F00073002BECD1CD
:1072A000524BDA68524B13407A68116A7A68526A14
:1072B000013A120111437A68926A120211437A6804
:1072C000126B5208013A520511437A68526B520808
:1072D000013A520611437A68D26AD2060A434349F8
:1072E0001343CB60414B1B68404A43F080731360EB
:1072F0003E4BDB683D4A43F08073D360FFF75EFD91
:10730000386108E0FFF75AFD02463B69D31A022BA9
:1073100001D9032366E0354B1B6803F00073002B93
:10732000F0D05EE0314B1B68304A23F0807313606D
:10733000FFF744FD386108E0FFF740FD02463B6976
:10734000D31A022B01D903234CE0284B1B6803F00E
:107350000073002BF0D1254BDA682449254B1340EC
:10736000CB603EE07B68DB69012B01D1012339E072
:107370001E4BDB687B617B6903F003027B681B6A41
:107380009A422CD17B6903F0F0027B685B6A013B77
:107390001B019A4223D17B6903F4FE427B689B6AFE
:1073A0001B029A421BD17B6903F078427B68DB6A3F
:1073B000DB069A4213D17B6903F4C0027B681B6B26
:1073C0005B08013B5B059A4209D17B6903F0C0620F
:1073D0007B685B6B5B08013B5B069A4201D0012333
:1073E00000E0002318462037BD4680BD0010024053
:1073F0000C809F01FCFFEEFE80B586B000AF786088
:10740000396000237B617B68002B01D101231EE1E1
:10741000914B1B6803F00F033A689A4210D98E4BC8
:107420001B6823F00F028C493B6813430B608A4BA7
:107430001B6803F00F033A689A4201D0012306E16A
:107440007B681B6803F00103002B73D07B685B68CB
:10745000032B29D1814B1B6803F00073002B01D152
:107460000123F4E000F09CF938613B697C4A9342C7
:107470003FD97A4B9B6803F0F003002B09D07B685F
:107480001B6803F00203002B33D07B689B68002B42
:107490002FD1724B9B6823F0F003704A43F08003B6
:1074A000936080237B6124E07B685B68022B07D1BB
:1074B0006A4B1B6803F40033002B09D10123C6E09B
:1074C000664B1B6803F48063002B01D10123BEE0EF
:1074D00000F0CEF838613B69614A934209D95F4BAD
:1074E0009B6823F0F0035D4A43F0800393608023A0
:1074F0007B615A4B9B6823F003027B685B685749AA
:1075000013438B60FFF75AFCF8600AE0FFF756FC64
:107510000246FB68D31A41F28832934201D9032311
:1075200095E04E4B9B6803F00C027B685B689B0008
:107530009A42EBD17B681B6803F00203002B23D037
:107540007B681B6803F00403002B05D0434B9B684A
:10755000424A43F4E06393607B681B6803F00803CE
:10756000002B07D03D4B9B6823F47C533B4A43F4EC
:10757000E0639360394B9B6823F0F0027B689B6863
:10758000364913438B6008E07B69802B05D1334B70
:107590009B68324A23F0F00393602F4B1B6803F083
:1075A0000F033A689A421DD22B4B1B6823F00F023F
:1075B00029493B6813430B60FFF700FCF8600AE0C1
:1075C000FFF7FCFB0246FB68D31A41F28832934274
:1075D00001D903233BE0204B1B6803F00F033A68FB
:1075E0009A42EDD17B681B6803F00403002B08D09E
:1075F0001A4B9B6823F4E0627B68DB6817491343EE
:107600008B607B681B6803F00803002B09D0134BC9
:107610009B6823F460527B681B69DB000F491343AE
:107620008B6000F025F802460C4B9B681B0903F0A9
:107630000F030C49CB5C03F01F0322FA03F30A4A41
:1076400013600A4B1B681846FFF76CFB034618468D
:107650001837BD4680BD00BF002002400010024028
:1076600000B4C4041CE60108C0000020B8000020DB
:1076700080B487B000AF2C4B9B6803F00C03042B45
:1076800002D12A4B3B6147E0274B9B6803F00C0378
:10769000082B02D1254B3B613EE0234B9B6803F056
:1076A0000C030C2B36D1204BDB6803F00303FB608B
:1076B0001D4BDB681B0903F00F030133BB60FB6844
:1076C000032B0CD1194ABB68B2FBF3F3164AD268FC
:1076D000120A02F07F0202FB03F37B610CE0134A03
:1076E000BB68B2FBF3F3104AD268120A02F07F02C1
:1076F00002FB03F37B6100BF0B4BDB685B0E03F007
:10770000030301335B007B607A697B68B2FBF3F3B0
:107710003B6101E000233B613B6918461C37BD46D5
:107720005DF8047B704700BF001002400024F400A5
:1077300080B400AF034B1B681846BD465DF8047B60
:10774000704700BFC000002080B500AFFFF7F0FF1A
:107750000246064B9B681B0A03F007030449CB5CF7
:1077600003F01F0322FA03F3184680BD0010024005
:107770002CE6010880B500AFFFF7DAFF0246064BA2
:107780009B68DB0A03F007030449CB5C03F01F038B
:1077900022FA03F3184680BD001002402CE60108CF
:1077A00080B487B000AF1E4BDB6803F003033B617E
:1077B0001B4BDB681B0903F00F030133FB603B69C4
:1077C000032B0CD1174AFB68B2FBF3F3144AD268BF
:1077D000120A02F07F0202FB03F37B610CE0114A04
:1077E000FB68B2FBF3F30E4AD268120A02F07F0282
:1077F00002FB03F37B6100BF094BDB685B0E03F008
:10780000030301335B00BB607A69BB68B2FBF3F32F
:107810007B607B6818461C37BD465DF8047B70476B
:10782000001002400024F40080B586B000AF7860FC
:107830000023FB740023BB747B681B6803F40023E4
:10784000002B00F0988000237B74434B9B6D03F06A
:107850008053002B0DD1404B9B6D3F4A43F080532A
:1078600093653D4B9B6D03F08053BB60BB68012368
:107870007B743A4B1B68394A43F480731360FFF7FB
:107880009DFAF86009E0FFF799FA0246FB68D31AFF
:10789000022B02D90323FB7405E0304B1B6803F471
:1078A0008073002BEFD0FB7C002B59D12A4BD3F8EF
:1078B000903003F440737B617B69002B1ED07B68A2
:1078C0001B6D7A699A4219D0234BD3F8903023F478
:1078D00040737B61204BD3F890301F4A43F48033D0
:1078E000C2F890301C4BD3F890301B4A23F48033FD
:1078F000C2F89030184A7B69C2F890307B6903F077
:107900000103002B16D0FFF759FAF8600BE0FFF7E0
:1079100055FA0246FB68D31A41F28832934202D9E3
:107920000323FB7406E00C4BD3F8903003F0020302
:10793000002BECD0FB7C002B0BD1074BD3F8903005
:1079400023F440727B681B6D03491343C1F89030E8
:1079500008E0FB7CBB7405E00010024000700040B2
:10796000FB7CBB747B7C012B05D1A74B9B6DA64A8E
:1079700023F0805393657B681B6803F00103002BA1
:107980000AD0A14BD3F8883023F003027B685B68F0
:107990009D491343C1F888307B681B6803F00203DC
:1079A000002B0AD0984BD3F8883023F00C027B6868
:1079B0009B6895491343C1F888307B681B6803F0C6
:1079C0000403002B0AD0904BD3F8883023F0300208
:1079D0007B68DB688C491343C1F888307B681B687F
:1079E00003F00803002B0AD0874BD3F8883023F02C
:1079F000C0027B681B6984491343C1F888307B68E7
:107A00001B6803F01003002B0AD07F4BD3F888309B
:107A100023F440727B685B697B491343C1F888306B
:107A20007B681B6803F02003002B0AD0764BD3F849
:107A3000883023F440627B689B6973491343C1F823
:107A400088307B681B6803F04003002B0AD06E4B24
:107A5000D3F8883023F440527B68DB696A491343CA
:107A6000C1F888307B681B6803F08003002B0AD0C4
:107A7000654BD3F8883023F440427B681B6A624927
:107A80001343C1F888307B681B6803F48073002BB4
:107A90000AD05D4BD3F8883023F440327B685B6AB0
:107AA00059491343C1F888307B681B6803F40033DD
:107AB000002B0AD0544BD3F89C3023F003027B6890
:107AC0009B6A51491343C1F89C307B681B6803F4DF
:107AD0000073002B0AD04C4BD3F8883023F440229B
:107AE0007B68DB6A48491343C1F888307B681B68B0
:107AF00003F48063002B15D0434BD3F8883023F474
:107B000040127B681B6B40491343C1F888307B6887
:107B10001B6BB3F5801F05D13B4BDB683A4A43F43E
:107B20008013D3607B681B6803F40063002B15D0BF
:107B3000354BD3F8883023F440027B685B6B3249C5
:107B40001343C1F888307B685B6BB3F5800F05D1B8
:107B50002D4BDB682C4A43F48013D3607B681B6891
:107B600003F48053002B15D0274BD3F8883023F033
:107B700040727B689B6B24491343C1F888307B6853
:107B80009B6BB3F1807F05D11F4BDB681E4A43F42A
:107B90008013D3607B681B6803F40053002B15D05F
:107BA000194BD3F8883023F040627B68DB6B1649B1
:107BB0001343C1F888307B68DB6BB3F1006F05D1EC
:107BC000114BDB68104A43F48013D3607B681B6859
:107BD00003F48043002B19D00B4BD3F8883023F0EB
:107BE00040627B681B6C08491343C1F888307B688E
:107BF0001B6CB3F1006F09D1034BDB68024A43F4FD
:107C00008013D36002E000BF001002407B681B6855
:107C100003F40043002B15D0294BD3F8883023F010
:107C200040527B685B6C26491343C1F888307B68FF
:107C30005B6CB3F1805F05D1214BDB68204A43F4D4
:107C40008033D3607B681B6803F48033002B15D02E
:107C50001B4BD3F8883023F040427B689B6C18495B
:107C60001343C1F888307B689B6CB3F1804F05D11A
:107C7000134BDB68124A43F48033D3607B681B6884
:107C800003F48023002B15D00D4BD3F89C3023F444
:107C900040127B68DB6C0A491343C1F89C307B6857
:107CA000DB6CB3F5001F05D1054BDB68044A43F4D8
:107CB0008013D360BB7C18461837BD4680BD00BF1B
:107CC0000010024080B487B000AF786039600023B4
:107CD0007B615AE13B681A6801217B6901FA03F371
:107CE0001340FB60FB68002B00F04C813B685B6835
:107CF00003F00303012B05D03B685B6803F003032B
:107D0000022B30D17B689B683B617B695B0003225F
:107D100002FA03F3DB433A6913403B613B68DA68DC
:107D20007B695B0002FA03F33A6913433B617B68AA
:107D30003A699A607B685B683B6101227B6902FA61
:107D400003F3DB433A6913403B613B685B681B0903
:107D500003F001027B6902FA03F33A6913433B61C2
:107D60007B683A695A603B685B6803F00303032B46
:107D700017D07B68DB683B617B695B00032202FAFA
:107D800003F3DB433A6913403B613B689A687B69C4
:107D90005B0002FA03F33A6913433B617B683A697B
:107DA000DA603B685B6803F00303022B23D17B6935
:107DB000DA087B68083253F822303B617B6903F0B4
:107DC00007039B000F2202FA03F3DB433A691340D7
:107DD0003B613B681A697B6903F007039B0002FA69
:107DE00003F33A6913433B617B69DA087B68083225
:107DF000396943F822107B681B683B617B695B0033
:107E0000032202FA03F3DB433A6913403B613B6808
:107E10005B6803F003027B695B0002FA03F33A69D3
:107E200013433B617B683A691A603B685B6803F403
:107E30004033002B00F0A6805B4B1B6E5A4A43F088
:107E400001031366584B1B6E03F00103BB60BB6854
:107E5000564A7B699B08023352F823303B617B69A9
:107E600003F003039B000F2202FA03F3DB433A699A
:107E700013403B617B68B3F1904F1FD07B684C4A45
:107E8000934219D07B684B4A934213D07B684A4A8D
:107E900093420DD07B68494A934207D07B68484A99
:107EA000934201D105230AE0062308E0042306E0FB
:107EB000032304E0022302E0012300E000237A69A7
:107EC00002F00302920093403A6913433B61374941
:107ED0007B699B0802333A6941F82320394B9B6840
:107EE0003B61FB68DB433A6913403B613B685B687D
:107EF00003F48013002B03D03A69FB6813433B6102
:107F0000304A3B6993602F4BDB683B61FB68DB4386
:107F10003A6913403B613B685B6803F40013002B34
:107F200003D03A69FB6813433B61264A3B69D3603F
:107F3000244B5B683B61FB68DB433A6913403B6160
:107F40003B685B6803F40033002B03D03A69FB689D
:107F500013433B611B4A3B6953601A4B1B683B61EF
:107F6000FB68DB433A6913403B613B685B6803F4A1
:107F70008033002B03D03A69FB6813433B61114AFD
:107F80003B6913607B6901337B613B681A687B69DD
:107F900022FA03F3002B7FF49DAE00BF00BF1C3715
:107FA000BD465DF8047B70470010024000000140B0
:107FB0000004004800080048000C00480010004879
:107FC000001400480004014080B485B000AF786020
:107FD0000B467B807B681A697B881340002B02D09C
:107FE0000123FB7301E00023FB73FB7B184614376E
:107FF000BD465DF8047B704780B584B000AF786003
:108000007B68002B01D101238DE07B681B681A4639
:10801000474B9A420FD87B681B681A46454B13445E
:10802000454AA2FB03231B099A007B685A647B68BC
:10803000424A1A640EE07B681B681A46404B1344A0
:108040003D4AA2FB03231B099A007B685A647B68A4
:108050003C4A1A647B68022283F825207B681B68EF
:108060001B68FB60FB6823F4FF4323F07003FB6095
:108070007B689A687B68DB681A437B681B691A43D4
:108080007B685B691A437B689B691A437B68DB6981
:108090001A437B681B6A1343FA681343FB607B68CF
:1080A0001B68FA681A60786800F0B6F97B689B680C
:1080B000B3F5804F02D17B6800225A607B685A6812
:1080C0007B689B6CD2B21A607B68DB6C7A68126D3D
:1080D0005A607B685B68002B10D07B685B68042B60
:1080E0000CD8786800F0D6F97B685B6D00221A60C6
:1080F0007B689B6D7A68D26D5A6008E07B680022CD
:108100005A657B6800229A657B680022DA657B6885
:108110000022DA637B68012283F825207B68002235
:1081200083F82420002318461037BD4680BD00BFC9
:1081300007040240F8FFFDBFCDCCCCCC00000240CC
:10814000F8FBFDBF0004024080B586B000AFF860C8
:10815000B9607A603B600023FB75FB6893F82430BC
:10816000012B01D1022366E0FB68012283F8242061
:10817000FB6893F82530DBB2012B55D1FB68022256
:1081800083F82520FB680022DA63FB681B681A6805
:10819000FB681B6822F001021A603B687A68B968C4
:1081A000F86800F0FBF8FB681B6B002B08D0FB683D
:1081B0001B681A68FB681B6842F00E021A600FE029
:1081C000FB681B681A68FB681B6822F004021A60CF
:1081D000FB681B681A68FB681B6842F00A021A6099
:1081E000FB689B6C1B6803F48033002B07D0FB6893
:1081F0009B6C1A68FB689B6C42F480721A60FB6887
:108200005B6D002B07D0FB685B6D1A68FB685B6DCC
:1082100042F480721A60FB681B681A68FB681B686E
:1082200042F001021A6005E0FB68002283F8242076
:108230000223FB75FB7D18461837BD4680BD80B50F
:1082400084B000AF78607B681B6C1B68FB607B6848
:108250001B681B68BB607B685B6C03F01F03042218
:108260009A40FB681340002B26D0BB6803F0040340
:10827000002B21D07B681B681B6803F02003002BB8
:1082800007D17B681B681A687B681B6822F00402B0
:108290001A607B685B6C03F01F027B681B6C042117
:1082A00001FA02F25A607B681B6B002B71D07B686D
:1082B0001B6B786898476CE07B685B6C03F01F036E
:1082C00002229A40FB681340002B2ED0BB6803F0BB
:1082D0000203002B29D07B681B681B6803F0200376
:1082E000002B0BD17B681B681A687B681B6822F027
:1082F0000A021A607B68012283F825207B685B6C88
:1083000003F01F027B681B6C022101FA02F25A6023
:108310007B68002283F824207B68DB6A002B38D03E
:108320007B68DB6A7868984733E07B685B6C03F0B6
:108330001F0308229A40FB681340002B2AD0BB6819
:1083400003F00803002B25D07B681B681A687B6844
:108350001B6822F00E021A607B685B6C03F01F0240
:108360007B681B6C012101FA02F25A607B680122D2
:10837000DA637B68012283F825207B68002283F87A
:1083800024207B685B6B002B04D07B685B6B786878
:10839000984700BF00BF1037BD4680BD80B485B090
:1083A00000AFF860B9607A603B60FB68DB6CFA682C
:1083B000126D5A60FB685B6D002B04D0FB689B6DEF
:1083C000FA68D26D5A60FB685B6C03F01F02FB68B1
:1083D0001B6C012101FA02F25A60FB681B683A68C3
:1083E0005A60FB689B68102B08D1FB681B687A6891
:1083F0009A60FB681B68BA68DA6007E0FB681B6874
:10840000BA689A60FB681B687A68DA6000BF143744
:10841000BD465DF8047B704780B487B000AF7860DC
:108420007B681B681A46164B9A4202D8154B7B6133
:1084300001E0154B7B617B693B617B681B68DBB2AC
:10844000083B124AA2FB03231B09FB607B685B6CA1
:108450009B089A003B6913441A467B689A647B68C0
:108460000B4ADA64FB6803F01F0301229A407B6821
:108470001A6500BF1C37BD465DF8047B704700BF1E
:10848000070402400008024020080240CDCCCCCCBA
:108490008008024080B485B000AF78607B685B687C
:1084A000DBB2FB60FA680B4B13449B001A467B68F7
:1084B0005A657B68084A9A65FB68013B03F01F0315
:1084C00001229A407B68DA6500BF1437BD465DF82B
:1084D000047B70473F8200104009024080B485B0A1
:1084E00000AF78607B68002B41D14B4B1B6803F4D5
:1084F000C063B3F5806F31D1474BD3F88030464A23
:1085000023F48073C2F88030434B1B6823F4C063AC
:10851000414A43F400731360404B1B68322202FB54
:1085200003F33F4AA2FB03239B0C0133FB6002E0F1
:10853000FB68013BFB60384B5B6903F48063B3F578
:10854000806F02D1FB68002BF2D1334B5B6903F4DF
:108550008063B3F5806F58D1032357E02E4BD3F8D7
:1085600080302D4A23F48073C2F880304DE07B6860
:10857000B3F5007F41D1284B1B6803F4C063B3F50A
:10858000806F31D1244BD3F88030234A43F4807379
:10859000C2F88030204B1B6823F4C0631E4A43F4AA
:1085A000007313601D4B1B68322202FB03F31C4A4D
:1085B000A2FB03239B0C0133FB6002E0FB68013B41
:1085C000FB60154B5B6903F48063B3F5806F02D1E8
:1085D000FB68002BF2D1104B5B6903F48063B3F5A9
:1085E000806F12D1032311E00B4BD3F880300A4A7D
:1085F00043F48073C2F8803007E0074B1B6823F414
:10860000C063054A43F4806313600023184614379F
:10861000BD465DF8047B704700700040C00000203C
:1086200083DE1B4380B400AF054B9B68044A43F4D0
:108630008043936000BFBD465DF8047B704700BF78
:108640000070004080B485B000AF78607B6803F0B4
:108650000703FB600C4BDB68BB60BA684FF6FF0397
:108660001340BB60FB681A02BB68134343F0BF634F
:1086700043F40033BB60044ABB68D36000BF1437C7
:10868000BD465DF8047B704700ED00E080B400AFAC
:10869000044BDB681B0A03F007031846BD465DF870
:1086A000047B704700ED00E080B483B000AF034668
:1086B000FB7197F90730002B0BDBFB7903F01F02EE
:1086C000074997F907305B09012000FA02F241F8E7
:1086D000232000BF0C37BD465DF8047B704700BF08
:1086E00000E100E080B483B000AF03463960FB7165
:1086F00097F90730002B0ADB3B68DAB20C4997F98F
:1087000007301201D2B20B4483F800230AE03B6821
:10871000DAB20849FB7903F00F03043B1201D2B22D
:108720000B441A7600BF0C37BD465DF8047B7047DA
:1087300000E100E000ED00E080B489B000AFF86037
:10874000B9607A60FB6803F00703FB61FB69C3F162
:108750000703042B28BF0423BB61FB690433062BEA
:1087600002D9FB69033B00E000237B614FF0FF323D
:10877000BB6902FA03F3DA43BB681A407B699A408B
:108780004FF0FF317B6901FA03F3D9437B680B405B
:10879000134318462437BD465DF8047B704700003C
:1087A00080B582B000AF78607B68013BB3F1807F19
:1087B00001D301230FE00A4A7B68013B53600F217C
:1087C0004FF0FF30FFF78EFF054B00229A60044BFD
:1087D00007221A60002318460837BD4680BD00BF37
:1087E00010E000E080B582B000AF78607868FFF7F5
:1087F00029FF00BF0837BD4680BD80B586B000AFF9
:108800000346B9607A60FB73FFF740FF78617A68CE
:10881000B9687869FFF790FF024697F90F30114663
:108820001846FFF75FFF00BF1837BD4680BD80B513
:1088300082B000AF0346FB7197F907301846FFF787
:1088400033FF00BF0837BD4680BD80B582B000AFA2
:1088500078607868FFF7A4FF034618460837BD46DE
:1088600080BD80B483B000AF786039607B689B685E
:1088700023F47C123B681A437B689A6000BF0C3774
:10888000BD465DF8047B704780B483B000AF78606C
:1088900039607B689B6823F0E0723B681A437B6811
:1088A0009A6000BF0C37BD465DF8047B704780B40A
:1088B00083B000AF78607B689B6803F0E073184674
:1088C0000C37BD465DF8047B7047000080B487B06C
:1088D00000AFF860B9607A603B60FB6860331A46AD
:1088E000BB689B0013447B617B691A68084B13408B
:1088F0007A6802F0F8413A680A43134343F00042B1
:108900007B691A6000BF1C37BD465DF8047B704769
:1089100000F0FF0380B485B000AF786039607B68F9
:1089200060331A463B689B001344FB60FB681B687E
:1089300003F0F84318461437BD465DF8047B7047D2
:1089400080B487B000AFF860B9607A60FB686033CC
:108950001A46BB689B0013447B617B691B6823F04C
:1089600000427B681A437B691A6000BF1C37BD4612
:108970005DF8047B704780B487B000AFF860B960E1
:108980007A60FB6860331A46BB689B0013447B61C6
:108990007B691B6823F080727B681A437B691A60CD
:1089A00000BF1C37BD465DF8047B704780B487B0BC
:1089B00000AFF860B9607A60FB6860331A46BB6844
:1089C0009B0013447B617B691B6823F000727B680A
:1089D0001A437B691A6000BF1C37BD465DF8047BF3
:1089E000704780B483B000AF786039607B685B69A2
:1089F00023F000423B681A437B685A6100BF0C3782
:108A0000BD465DF8047B704780B483B000AF7860EA
:108A10007B68DB6803F44063002B01D1012300E095
:108A2000002318460C37BD465DF8047B704780B4C0
:108A300087B000AFF860B9607A60FB6830331A46DF
:108A4000BB681B0A9B0003F00C0313447B617B692A
:108A50001A68BB6803F01F031F2101FA03F3DB430D
:108A60001A407B689B0E03F01F01BB6803F01F03D5
:108A700001FA03F31A437B691A6000BF1C37BD4635
:108A80005DF8047B704780B487B000AFF860B960D0
:108A90007A60FB6814331A46BB685B0E9B0003F0D8
:108AA000040313447B617B691A68BB681B0D03F0E8
:108AB0001F03072101FA03F3DB431A40BB681B0DB8
:108AC00003F01F03796801FA03F31A437B691A6004
:108AD00000BF1C37BD465DF8047B704780B485B08D
:108AE00000AFF860B9607A60FB68D3F8B020BB686B
:108AF000C3F31203DB431A407B6803F018030849F1
:108B0000D940BB680B40C3F312031A43FB68C3F898
:108B1000B02000BF1437BD465DF8047B704700BF2E
:108B2000FFFF070080B483B000AF78607B689B686C
:108B300003F01F0318460C37BD465DF8047B7047F1
:108B400080B483B000AF78607B689B6823F02043DB
:108B500023F03F037A68936000BF0C37BD465DF891
:108B6000047B704780B483B000AF78607B689B68FB
:108B700003F00053B3F1005F01D1012300E00023B3
:108B800018460C37BD465DF8047B704780B483B04F
:108B900000AF78607B689B6823F0104323F03F03AD
:108BA00043F080527B689A6000BF0C37BD465DF889
:108BB000047B704780B483B000AF78607B689B68AB
:108BC00003F08053B3F1805F01D1012300E0002363
:108BD00018460C37BD465DF8047B704780B483B0FF
:108BE00000AF78607B689B6823F0004323F03F036D
:108BF00043F001027B689A6000BF0C37BD465DF808
:108C0000047B704780B483B000AF78607B689B685A
:108C100023F0004323F03F0343F002027B689A6095
:108C200000BF0C37BD465DF8047B704780B483B04D
:108C300000AF78607B689B6803F00103012B01D1D2
:108C4000012300E0002318460C37BD465DF8047B85
:108C5000704780B483B000AF78607B689B6803F096
:108C60000203022B01D1012300E0002318460C3738
:108C7000BD465DF8047B704780B483B000AF786078
:108C80007B689B6823F0004323F03F0343F004021A
:108C90007B689A6000BF0C37BD465DF8047B704767
:108CA00080B483B000AF78607B689B6803F00403F6
:108CB000042B01D1012300E0002318460C37BD46E8
:108CC0005DF8047B704780B483B000AF78607B6848
:108CD0009B6803F00803082B01D1012300E0002367
:108CE00018460C37BD465DF8047B704790B589B0D7
:108CF00000AF78600023FB770023FB607B68002BCC
:108D000001D10123A9E17B685B69002B7B68DB6DE6
:108D1000002B09D17868F8F7EFFC7B6800221A660F
:108D20007B68002283F858207B681B681846FFF791
:108D300019FF0346002B04D07B681B681846FFF719
:108D4000FFFE7B681B681846FFF734FF0346002BC5
:108D500015D17B681B681846FFF718FF9C4B1B68F2
:108D60009B099C4AA2FB03239B0901335B00FB6028
:108D700002E0FB68013BFB60FB68002BF9D17B68DC
:108D80001B681846FFF716FF0346002B0DD17B68C2
:108D9000DB6D43F010027B68DA657B681B6E43F085
:108DA00001027B681A660123FB777B681B68184603
:108DB000FFF776FF78617B68DB6D03F01003002B13
:108DC00040F042817B69002B40F03E817B68DB6D87
:108DD00023F4817343F002027B68DA657B681B68C9
:108DE0001846FFF723FF0346002B41D17B681B6821
:108DF000B3F1A04F04D07B681B68774A93420FD130
:108E00004FF0A040FFF712FF04467348FFF70EFF34
:108E100003462343002B0CBF01230023DBB212E0E7
:108E20006E48FFF703FF04466D48FFF7FFFE034659
:108E30001C436C48FFF7FAFE03462343002B0CBF8C
:108E400001230023DBB2002B12D07B681B68B3F137
:108E5000A04F04D07B681B685F4A934201D1624AED
:108E600000E0624A7B685B6819461046FFF7F9FC30
:108E70007B685B7F5A037B68DB6B1A437B68DB682C
:108E80001A437B689B681A437B6893F824301B0461
:108E90001343BB617B6893F82430012B06D17B68B8
:108EA0009B6A013B5B04BA691343BB617B68DB6A65
:108EB000002B09D07B68DB6A03F478727B681B6B3C
:108EC0001343BA691343BB617B681B68DA68484B7C
:108ED00013407A681268B9690B43D3607B681B68DA
:108EE0001B6923F040617B685A6B7B681B680A43EF
:108EF0001A617B681B681846FFF7E5FE38617B69DD
:108F0000002B7FD13B69002B7CD17B681B7F9A03B0
:108F10007B6893F838305B001343BB617B681B6848
:108F2000DB6823F4804323F002037A681268B9698E
:108F30000B43D3607B681B69002B17D07B681B68D1
:108F40001A697B681B6842F480321A617B681B686F
:108F5000D3F8C03023F47F5323F03F037A681169BC
:108F60007A6812680B43C2F8C03013E07B681B6854
:108F70001A697B681B6822F480321A617B681B685F
:108F8000D3F8C0307A68126823F47F5323F03F038C
:108F9000C2F8C0307B6893F84030012B2AD17B683F
:108FA0001B681B6923F4FF6323F004037A68516C88
:108FB0007A68926C11437A68D26C11437A68126DA8
:108FC0000A431A437B681B6842F001021A6119E0E8
:108FD000C0000020632D3E05000100500004005039
:108FE000000500500006005000030050000700502C
:108FF0000740F0FF7B681B681A697B681B6822F0DA
:1090000001021A617B685B69012B0CD17B681B68CC
:109010001B6B23F00F017B681B6A5A1E7B681B6861
:109020000A431A6307E07B681B681A6B7B681B683E
:1090300022F00F021A637B68DB6D23F0030343F019
:1090400001027B68DA6507E07B68DB6D43F01002A4
:109050007B68DA650123FB77FB7F18462437BD4622
:1090600090BD00BF80B586B000AFF860B9607A608F
:10907000FB681B68B3F1A04F04D0FB681B685A4A19
:10908000934201D1594B00E0594B1846FFF74AFD76
:109090003861FB681B681846FFF702FE0346002B89
:1090A00040F09B80FB6893F85830012B01D10223DC
:1090B00096E0FB68012283F85820FB681B684D4A44
:1090C000934208D03B69002B05D03B69052B02D0A9
:1090D0003B69092B7AD1F86800F0ECFC0346FB757C
:1090E000FB7D002B6DD1FB68DB6D23F4706323F0F7
:1090F000010343F48072FB68DA65FB681B683A4A37
:10910000934209D0FB681B683B4A934202D0FB683C
:109110001B6803E0394B01E04FF0A043FA68126886
:10912000934202D03B69002B05D1FB68DB6D23F431
:109130008012FB68DA65FB68DB6D03F48053002B5B
:1091400006D0FB681B6E23F00602FB681A6602E07D
:10915000FB6800221A66FB685B6D294ADA62FB68CD
:109160005B6D284A1A63FB685B6D274A5A63FB688C
:109170001B681C221A60FB68002283F85820FB68D9
:109180001B685A68FB681B6842F010025A60FB6853
:109190001B68DA68FB681B6842F00102DA60FB6852
:1091A000586DFB681B6840331946BA687B68FEF748
:1091B000CBFF0346FB75FB681B681846FFF75CFD99
:1091C0000DE0FB68002283F8582008E00123FB75BE
:1091D000FB68002283F8582001E00223FB75FB7D29
:1091E00018461837BD4680BD0001005000030050EE
:1091F0000007005000060050000500500004005019
:109200009F9C0108779D0108939D010880B483B05D
:1092100000AF786000BF0C37BD465DF8047B704737
:1092200080B483B000AF786000BF0C37BD465DF8F6
:10923000047B704780B5B6B000AF7860396000231A
:1092400087F8D7300023FB607B6893F85830012BF8
:1092500002D1022300F013BC7B68012283F858205E
:109260007B681B681846FFF71BFD0346002B40F088
:10927000F3837B6818683B6859683B681B681A462B
:10928000FFF7D5FB7B681B681846FFF709FDC7F899
:10929000D0007B681B681846FFF715FDC7F8CC00A7
:1092A000D7F8D030002B40F0D981D7F8CC30002B44
:1092B00040F0D4813B689B68B3F1004F0FD17B68CD
:1092C00018683B681B6800221946FFF7DCFB7B68C7
:1092D0001B684FF000411846FFF783FB0EE07B68E8
:1092E00018683B6819683B689B681A46FFF7CBFB18
:1092F0007B681B6800211846FFF773FB3B685A69BF
:109300007B681B68DB68DB0803F003035B0002FA81
:1093100003F3C7F8C8303B681B69042B22D07B6875
:1093200018683B6819693B681A68D7F8C830FFF7B6
:10933000CDFA7B6818683B6819693B689B691A46D7
:10934000FFF719FB7B6818683B6819693B681B7F4E
:10935000012B02D14FF0007300E000231A46FFF703
:1093600025FB7BE17B681B6800211846FFF7D2FADA
:109370000346C3F31203002B0AD17B681B6800214C
:109380001846FFF7C7FA03469B0E03F01F021EE0C4
:109390007B681B6800211846FFF7BCFA0346C7F834
:1093A000BC30D7F8BC3093FAA3F3C7F8B830D7F87D
:1093B000B830C7F8C030D7F8C030002B01D1202317
:1093C00004E0D7F8C030B3FA83F3DBB21A463B6847
:1093D0001B68C3F31203002B05D13B681B689B0E6F
:1093E00003F01F0318E03B681B68C7F8B030D7F8DC
:1093F000B03093FAA3F3C7F8AC30D7F8AC30C7F865
:10940000B430D7F8B430002B01D1202304E0D7F8D2
:10941000B430B3FA83F3DBB29A4206D17B681B689F
:10942000002200211846FFF78BFA7B681B68012198
:109430001846FFF76FFA0346C3F31203002B0AD155
:109440007B681B6801211846FFF764FA03469B0EF0
:1094500003F01F021EE07B681B6801211846FFF71E
:1094600059FA0346C7F8A430D7F8A43093FAA3F307
:10947000C7F8A030D7F8A030C7F8A830D7F8A83080
:10948000002B01D1202304E0D7F8A830B3FA83F3EE
:10949000DBB21A463B681B68C3F31203002B05D1ED
:1094A0003B681B689B0E03F01F0318E03B681B68BA
:1094B000C7F89830D7F8983093FAA3F3C7F89430E8
:1094C000D7F89430C7F89C30D7F89C30002B01D1E6
:1094D000202304E0D7F89C30B3FA83F3DBB29A423E
:1094E00006D17B681B68002201211846FFF728FA85
:1094F0007B681B6802211846FFF70CFA0346C3F38A
:109500001203002B0AD17B681B6802211846FFF763
:1095100001FA03469B0E03F01F021EE07B681B68E6
:1095200002211846FFF7F6F90346C7F88C30D7F842
:109530008C3093FAA3F3C7F88830D7F88830C7F88F
:109540009030D7F89030002B01D1202304E0D7F8D9
:109550009030B3FA83F3DBB21A463B681B68C3F35F
:109560001203002B05D13B681B689B0E03F01F0301
:1095700016E03B681B68C7F88030D7F8803093FA54
:10958000A3F3FB67FB6FC7F88430D7F88430002B58
:1095900001D1202304E0D7F88430B3FA83F3DBB29F
:1095A0009A4206D17B681B68002202211846FFF709
:1095B000C7F97B681B6803211846FFF7ABF9034620
:1095C000C3F31203002B0AD17B681B6803211846E2
:1095D000FFF7A0F903469B0E03F01F0217E07B681C
:1095E0001B6803211846FFF795F903467B677B6FDD
:1095F00093FAA3F33B673B6FBB67BB6F002B01D1B3
:10960000202303E0BB6FB3FA83F3DBB21A463B6857
:109610001B68C3F31203002B05D13B681B689B0E2C
:1096200003F01F0311E03B681B68BB66BB6E93FA37
:10963000A3F37B667B6EFB66FB6E002B01D12023C0
:1096400003E0FB6EB3FA83F3DBB29A4206D17B6888
:109650001B68002203211846FFF772F97B681B681C
:109660001846FFF7E3FA0346002B40F03D817B6884
:1096700018683B6819683B68DB681A46FFF72EFAE2
:109680003B68DB68A24A934240F02E817B681868F1
:109690003B681B68C3F31203002B0BD13B681B68AC
:1096A0009B0E013303F01F03092B94BF01230023FA
:1096B000DBB219E03B681B68FB65FB6D93FAA3F313
:1096C000BB65BB6D3B663B6E002B01D1202303E0E5
:1096D0003B6EB3FA83F3DBB2013303F01F03092BB4
:1096E00094BF01230023DBB2002B79D03B681B68B9
:1096F000C3F31203002B07D13B681B689B0E013399
:109700009B0603F0F84215E03B681B683B653B6D28
:1097100093FAA3F3FB64FB6C7B657B6D002B01D19B
:10972000202303E07B6DB3FA83F3DBB201339B06A6
:1097300003F0F8423B681B68C3F31203002B09D106
:109740003B681B689B0E013303F01F03012101FAE4
:1097500003F317E03B681B687B647B6C93FAA3F30D
:109760003B643B6CBB64BB6C002B01D1202303E04A
:10977000BB6CB3FA83F3DBB2013303F01F030121A7
:1097800001FA03F342EA03013B681B68C3F31203C7
:10979000002B0AD13B681B689B0E013303F01F02AC
:1097A00013465B0013441B0518E03B681B68BB6352
:1097B000BB6B93FAA3F37B637B6BFB63FB6B002BAD
:1097C00001D1202303E0FB6BB3FA83F3DBB2013357
:1097D00003F01F0213465B0013441B050B437EE09E
:1097E0003B681B68C3F31203002B07D13B681B685F
:1097F0009B0E01339B0603F0F84215E03B681B68A3
:10980000FB62FB6A93FAA3F3BB62BB6A3B633B6BED
:10981000002B01D1202303E03B6BB3FA83F3DBB2CF
:1098200001339B0603F0F8423B681B68C3F3120345
:10983000002B09D13B681B689B0E013303F01F030B
:10984000012101FA03F317E03B681B683B623B6AA6
:1098500093FAA3F3FB61FB697B627B6A002B01D166
:10986000202303E07B6AB3FA83F3DBB2013303F016
:109870001F03012101FA03F342EA03013B681B685D
:10988000C3F31203002B0DD13B681B689B0E013301
:1098900003F01F0213465B0013441E3B1B0543F0FD
:1098A00000731BE03B681B687B617B6993FAA3F341
:1098B0003B613B69BB61BB69002B01D1202303E005
:1098C000BB69B3FA83F3DBB2013303F01F02134623
:1098D0005B0013441E3B1B0543F000730B433A68C7
:1098E00092681946FFF7CFF83B681A68094B134096
:1098F000002B00F0BE807B681B68B3F1A04F04D042
:109900007B681B68044A93420AD1044B09E000BFFC
:1099100000007F400000088000010050000300505C
:10992000594B1846FEF7C3FFC7F8C4003B681B68D5
:10993000564A934204D03B681B68554A93423AD139
:10994000D7F8C43003F40003002B34D17B681B68C4
:10995000B3F1A04F05D07B681B684E4A934240F09C
:1099600085807B681B68B3F1A04F04D07B681B68BF
:10997000494A934201D1494A00E0434AD7F8C430EA
:1099800043F4000319461046FEF77EFF444B1B6864
:109990009B09444AA2FB03239B095A1C13465B0004
:1099A00013449B00FB6002E0FB68013BFB60FB682B
:1099B000002BF9D15AE03B681B683B4A934225D102
:1099C000D7F8C43003F08073002B1FD17B681B686D
:1099D000314A934204D17B681B68344A934247D092
:1099E0007B681B68B3F1A04F04D07B681B682A4AD0
:1099F000934201D1294A00E0234AD7F8C43043F00A
:109A0000807319461046FEF73FFF31E03B681B6844
:109A1000274A93422DD1D7F8C43003F48003002B9A
:109A200027D17B681B681C4A934222D07B681B6845
:109A3000B3F1A04F04D07B681B68174A934201D151
:109A4000164A00E0104AD7F8C43043F480031946A0
:109A50001046FEF719FF0CE07B68DB6D43F0200237
:109A60007B68DA65012387F8D73002E000BF00E0A9
:109A700000BF7B68002283F8582097F8D73018463B
:109A8000D837BD4680BD00BF00070050000021C38D
:109A90001000C0900006005000010050000300506C
:109AA000C0000020632D3E05000052C70005005095
:109AB000000084CB80B584B000AF78600023BB6029
:109AC0007B681B681846FFF7B1F80346002B76D178
:109AD0007B681B689A683C4B1340002B0DD07B6859
:109AE000DB6D43F010027B68DA657B681B6E43F028
:109AF00001027B681A66012362E07B681B681846D6
:109B0000FFF76CF87B681B68B3F1A04F04D07B684B
:109B10001B682E4A934201D12D4B00E02D4B184675
:109B2000FEF7C5FE034603F40003002B13D02A4BB7
:109B30001B689B09294AA2FB03239B095A1C134655
:109B40005B0013449B00BB6002E0BB68013BBB6051
:109B5000BB68002BF9D1FDF731F9F86028E07B688C
:109B60001B681846FFF762F80346002B04D17B6898
:109B70001B681846FFF732F8FDF720F90246FB682C
:109B8000D31A022B14D97B681B681B6803F00103EE
:109B9000012B0DD07B68DB6D43F010027B68DA652A
:109BA0007B681B6E43F001027B681A66012307E0A5
:109BB0007B681B681B6803F00103012BCFD10023D6
:109BC00018461037BD4680BD3F00008000010050A0
:109BD0000003005000070050C0000020632D3E0528
:109BE00080B584B000AF78607B681B681846FFF7CB
:109BF00030F8F8607B681B681846FFF717F80346D3
:109C0000002B47D0FB68002B44D17B681B689B6806
:109C100003F00D03012B0CD17B681B681846FEF77F
:109C2000F1FF7B681B6803221A60FDF7C7F8B86074
:109C300029E07B68DB6D43F010027B68DA657B68A6
:109C40001B6E43F001027B681A66012323E0FDF7D7
:109C5000B5F80246BB68D31A022B14D97B681B687F
:109C60009B6803F00103002B0DD07B68DB6D43F094
:109C700010027B68DA657B681B6E43F001027B682B
:109C80001A66012307E07B681B689B6803F00103E9
:109C9000002BDCD1002318461037BD4680BD80B5AF
:109CA00084B000AF78607B689B6AFB60FB68DB6D0B
:109CB00003F05003002B4BD1FB68DB6D43F40072C3
:109CC000FB68DA65FB681B681B6803F00803002B60
:109CD00021D0FB681B681846FEF796FE0346002B52
:109CE00032D0FB681B68DB6803F40053002B2BD1D8
:109CF000FB68DB6D23F48072FB68DA65FB68DB6D63
:109D000003F48053002B1FD1FB68DB6D43F001028D
:109D1000FB68DA6518E0FB681B68DB6803F0020388
:109D2000002B11D1FB68DB6D23F48072FB68DA65D0
:109D3000FB68DB6D03F48053002B05D1FB68DB6D02
:109D400043F00102FB68DA65F868F7F7A1F90EE065
:109D5000FB68DB6D03F01003002B03D0F868FFF7FE
:109D60005FFA04E0FB685B6D5B6B7868984700BF47
:109D70001037BD4680BD80B584B000AF78607B6889
:109D80009B6AFB60F868FFF741FA00BF1037BD46D9
:109D900080BD80B584B000AF78607B689B6AFB6053
:109DA000FB68DB6D43F04002FB68DA65FB681B6E05
:109DB00043F00402FB681A66F868FFF731FA00BF47
:109DC0001037BD4680BD80B483B000AF78607B683B
:109DD0009B6803F00103012B01D1012300E0002364
:109DE00018460C37BD465DF8047B704780B483B0DD
:109DF00000AF786039607B689B6823F0404323F0B4
:109E00003F033A6802F08042134343F000427B680C
:109E10009A6000BF0C37BD465DF8047B704780B484
:109E200083B000AF78607B689B6803F00043B3F1B8
:109E3000004F01D1012300E0002318460C37BD4636
:109E40005DF8047B704780B483B000AF78607B68B6
:109E50009B6803F00403042B01D1012300E00023DD
:109E600018460C37BD465DF8047B704780B584B05A
:109E700000AF786039600023BB607B6893F858308E
:109E8000012B01D102234DE07B68012283F8582089
:109E90007868FFF7A5FE0346FB73FB7B002B36D1EA
:109EA0007B68DB6D23F4885323F0020343F0020246
:109EB0007B68DA657B681B6839681846FFF796FF90
:109EC00014E0BB680133BB60BB68184A93420DD9EC
:109ED0007B68DB6D23F0120343F010027B68DA65C8
:109EE0007B68002283F8582001231BE07B681B68F5
:109EF0001846FFF794FF0346002BE2D17B68DB6D29
:109F000023F0030343F001027B68DA6505E07B6818
:109F1000DB6D43F010027B68DA657B68002283F812
:109F20005820FB7B18461037BD4680BD01DE04007B
:109F300090B5A1B000AF78603960002387F87F301A
:109F40007B6893F85830012B01D10223E7E07B684E
:109F5000012283F8582000237B660023BB667B68C0
:109F60001B68B3F1A04F02D16F4BBB6009E07B6867
:109F70001B686E4A934202D16D4BBB6001E0002327
:109F8000BB60BB68002B0BD17B68DB6D43F020020C
:109F90007B68DA657B68002283F858200123BEE0E5
:109FA000BB681846FFF74FFFB8677B681B68184609
:109FB000FFF749FF0346002B40F0A080BB6F002B4A
:109FC00040F09C807B681B68B3F1A04F04D07B6895
:109FD0001B68554A934201D1564B00E0564B7B67B4
:109FE0003B681B68002B4BD07B6F9B6823F460425F
:109FF0003B6859687B6893F838305B030B431A431E
:10A000007B6F9A607B681B68B3F1A04F04D07B68BC
:10A010001B68454A93420FD14FF0A040FFF7D3FE93
:10A0200004464148FFF7CFFE03462343002B0CBFF5
:10A0300001230023DBB212E03C48FFF7C4FE0446D4
:10A040003B48FFF7C0FE03461C433C48FFF7BBFEFE
:10A0500003462343002B0CBF01230023DBB2002B5C
:10A0600056D07B6F9B6823F4716323F00F033A682B
:10A0700011683A6892680A431A437B6F9A6047E016
:10A080007B6F9B6823F460427B6F9A607B681B68E0
:10A09000B3F1A04F04D07B681B68234A93420FD1D1
:10A0A0004FF0A040FFF78FFE04461F48FFF78BFEDE
:10A0B00003462343002B0CBF01230023DBB212E035
:10A0C0001A48FFF780FE04461948FFF77CFE034656
:10A0D0001C431A48FFF777FE03462343002B0CBFAF
:10A0E00001230023DBB2002B12D07B6F9B6823F48B
:10A0F000716323F00F037A6F936009E07B68DB6D77
:10A1000043F020027B68DA65012387F87F3000E0A6
:10A1100000BF7B68002283F8582097F87F301846EC
:10A120008437BD4690BD00BF0001005000040050C0
:10A1300000050050000300500007005000060050CA
:10A1400080B582B000AF78607B68002B01D101231D
:10A150008DE07B6893F84130DBB2002B06D17B6841
:10A16000002283F840207868F7F73CFC7B682422C3
:10A1700083F841207B681B681A687B681B6822F0A3
:10A1800001021A607B685A687B681B6822F0706263
:10A190001A617B681B689A687B681B6822F400421E
:10A1A0009A607B68DB68012B07D17B689A687B68C3
:10A1B0001B6842F400429A6006E07B689A687B68FC
:10A1C0001B6842F404429A607B68DB68022B08D16A
:10A1D0007B681B685A687B681B6842F400625A609F
:10A1E00007E07B681B685A687B681B6822F4006282
:10A1F0005A607B681B685B687A68126843F000737A
:10A2000043F4004353607B681B68DA687B681B6813
:10A2100022F40042DA607B681A697B685B6942EA73
:10A2200003017B689B691A027B681B680A43DA603A
:10A230007B68D9697B681A6A7B681B680A431A6065
:10A240007B681B681A687B681B6842F001021A6011
:10A250007B6800225A647B68202283F841207B6857
:10A2600000221A637B68002283F8422000231846EC
:10A270000837BD4680BD80B483B000AF78603960D8
:10A280007B6893F84130DBB2202B38D17B6893F8A0
:10A290004030012B01D1022332E07B68012283F898
:10A2A00040207B68242283F841207B681B681A6861
:10A2B0007B681B6822F001021A607B681B681A68C1
:10A2C0007B681B6822F480521A607B681B681968DF
:10A2D0007B681B683A680A431A607B681B681A68C7
:10A2E0007B681B6842F001021A607B68202283F8B9
:10A2F00041207B68002283F84020002300E00223F5
:10A3000018460C37BD465DF8047B704780B485B0B5
:10A3100000AF786039607B6893F84130DBB2202B66
:10A3200039D17B6893F84030012B01D1022333E00F
:10A330007B68012283F840207B68242283F8412037
:10A340007B681B681A687B681B6822F001021A6030
:10A350007B681B681B68FB60FB6823F47063FB6011
:10A360003B681B02FA681343FB607B681B68FA6852
:10A370001A607B681B681A687B681B6842F00102E0
:10A380001A607B68202283F841207B68002283F8D2
:10A390004020002300E0022318461437BD465DF834
:10A3A000047B704780B582B000AF78607B68002B7B
:10A3B00001D1012349E07B6893F83D30DBB2002BEB
:10A3C00006D17B68002283F83C207868F7F706FD09
:10A3D0007B68022283F83D207B681A687B6804331F
:10A3E0001946104600F03AFC7B68012283F84820A9
:10A3F0007B68012283F83E207B68012283F83F209E
:10A400007B68012283F840207B68012283F8412089
:10A410007B68012283F842207B68012283F8432075
:10A420007B68012283F844207B68012283F8452061
:10A430007B68012283F846207B68012283F847204D
:10A440007B68012283F83D20002318460837BD466B
:10A4500080BD000080B485B000AF78607B6893F861
:10A460003D30DBB2012B01D001234CE07B6802229E
:10A4700083F83D207B681B68264A934222D07B6884
:10A480001B68B3F1804F1DD07B681B68224A934242
:10A4900018D07B681B68214A934213D07B681B68E5
:10A4A0001F4A93420ED07B681B681E4A934209D014
:10A4B0007B681B681C4A934204D07B681B681B4A5C
:10A4C000934215D17B681B689A68194B1340FB6057
:10A4D000FB68062B15D0FB68B3F5803F11D07B6875
:10A4E0001B681A687B681B6842F001021A6008E06A
:10A4F0007B681B681A687B681B6842F001021A605F
:10A5000000E000BF002318461437BD465DF8047B09
:10A51000704700BF002C01400004004000080040CC
:10A52000000C004000340140004001400050014058
:10A530000700010080B582B000AF78607B68002B17
:10A5400001D1012349E07B6893F83D30DBB2002B59
:10A5500006D17B68002283F83C20786800F041F83F
:10A560007B68022283F83D207B681A687B6804338D
:10A570001946104600F072FB7B68012283F84820E0
:10A580007B68012283F83E207B68012283F83F200C
:10A590007B68012283F840207B68012283F84120F8
:10A5A0007B68012283F842207B68012283F84320E4
:10A5B0007B68012283F844207B68012283F84520D0
:10A5C0007B68012283F846207B68012283F84720BC
:10A5D0007B68012283F83D20002318460837BD46DA
:10A5E00080BD80B483B000AF786000BF0C37BD463B
:10A5F0005DF8047B7047000080B584B000AF7860E0
:10A6000039603B68002B09D17B6893F83E30DBB2A0
:10A61000012B14BF01230023DBB23CE03B68042B79
:10A6200009D17B6893F83F30DBB2012B14BF0123C3
:10A630000023DBB22FE03B68082B09D17B6893F83D
:10A640004030DBB2012B14BF01230023DBB222E038
:10A650003B680C2B09D17B6893F84130DBB2012BAE
:10A6600014BF01230023DBB215E03B68102B09D196
:10A670007B6893F84230DBB2012B14BF0123002327
:10A68000DBB208E07B6893F84330DBB2012B14BFE8
:10A6900001230023DBB2002B01D00123A6E03B689D
:10A6A000002B04D17B68022283F83E2023E03B6824
:10A6B000042B04D17B68022283F83F201BE03B6817
:10A6C000082B04D17B68022283F8402013E03B680A
:10A6D0000C2B04D17B68022283F841200BE03B68FD
:10A6E000102B04D17B68022283F8422003E07B68B0
:10A6F000022283F843207B681B68012239681846D0
:10A7000000F026FF7B681B683A4A934218D07B68AA
:10A710001B68394A934213D07B681B68374A9342BF
:10A720000ED07B681B68364A934209D07B681B6851
:10A73000344A934204D07B681B68334A934201D168
:10A74000012300E00023002B07D07B681B685A6CB4
:10A750007B681B6842F400425A647B681B68254A88
:10A76000934222D07B681B68B3F1804F1DD07B6879
:10A770001B68264A934218D07B681B68244A934280
:10A7800013D07B681B68234A93420ED07B681B68FA
:10A79000194A934209D07B681B68184A934204D037
:10A7A0007B681B68184A934215D17B681B689A68BE
:10A7B000194B1340FB60FB68062B15D0FB68B3F503
:10A7C000803F11D07B681B681A687B681B6842F069
:10A7D00001021A6008E07B681B681A687B681B68C6
:10A7E00042F001021A6000E000BF00231846103753
:10A7F000BD4680BD002C01400034014000400140B6
:10A800000044014000480140005001400004004065
:10A8100000080040000C00400700010080B586B031
:10A8200000AFF860B9607A600023FB75FB6893F8AD
:10A830003C30012B01D10223FFE0FB68012283F8A9
:10A840003C207B68142B00F2F08001A252F823F028
:10A85000A5A801082BAA01082BAA01082BAA010808
:10A86000E5A801082BAA01082BAA01082BAA0108B8
:10A8700027A901082BAA01082BAA01082BAA010865
:10A8800067A901082BAA01082BAA01082BAA010815
:10A89000A9A901082BAA01082BAA01082BAA0108C3
:10A8A000E9A90108FB681B68B968184600F08AFA34
:10A8B000FB681B689A69FB681B6842F008029A6192
:10A8C000FB681B689A69FB681B6822F004029A61A6
:10A8D000FB681B689969BB681A69FB681B680A43B7
:10A8E0009A61A5E0FB681B68B968184600F004FB94
:10A8F000FB681B689A69FB681B6842F400629A61F6
:10A90000FB681B689A69FB681B6822F480629A6185
:10A91000FB681B689969BB681B691A02FB681B68A6
:10A920000A439A6184E0FB681B68B968184600F026
:10A9300077FBFB681B68DA69FB681B6842F008025A
:10A94000DA61FB681B68DA69FB681B6822F00402A5
:10A95000DA61FB681B68D969BB681A69FB681B6808
:10A960000A43DA6164E0FB681B68B968184600F0C6
:10A97000E9FBFB681B68DA69FB681B6842F400624C
:10A98000DA61FB681B68DA69FB681B6822F4806285
:10A99000DA61FB681B68D969BB681B691A02FB682E
:10A9A0001B680A43DA6143E0FB681B68B968184614
:10A9B00000F05CFCFB681B681A6DFB681B6842F0CA
:10A9C00008021A65FB681B681A6DFB681B6822F099
:10A9D00004021A65FB681B68196DBB681A69FB687D
:10A9E0001B680A431A6523E0FB681B68B9681846B0
:10A9F00000F0A6FCFB681B681A6DFB681B6842F43C
:10AA000000621A65FB681B681A6DFB681B6822F4FC
:10AA100080621A65FB681B68196DBB681B691A02A6
:10AA2000FB681B680A431A6502E00123FB7500BF3F
:10AA3000FB68002283F83C20FB7D18461837BD4692
:10AA400080BD00BF80B584B000AF7860396000235E
:10AA5000FB737B6893F83C30012B01D10223EEE0BD
:10AA60007B68012283F83C207B68022283F83D202A
:10AA70007B681B689B68BB60BB6823F4441323F0AE
:10AA80007703BB60BB6823F47F43BB607B681B68B4
:10AA9000BA689A603B681B686B4A934200F0B980C1
:10AAA000694A934200F2BE80684A934200F0B18046
:10AAB000664A934200F2B680654A934200F0A9804C
:10AAC000634A934200F2AE80624A934200F0A18052
:10AAD000604A934200F2A6805F4A934200F0998058
:10AAE0005D4A934200F29E80B3F1101F00F0918006
:10AAF000B3F1101F00F29680B3F5801F00F089803B
:10AB0000B3F5801F00F28E80B3F5005F3ED0B3F541
:10AB1000005F00F28780B3F5805F00F08680B3F5B8
:10AB2000805F7FD8702B1AD0702B7BD8602B50D0D1
:10AB3000602B77D8502B3CD0502B73D8402B58D05B
:10AB4000402B6FD8302B64D0302B6BD8202B60D0AB
:10AB5000202B67D8002B5CD0102B5AD062E07B688A
:10AB600018683B6899683B685A683B68DB6800F086
:10AB7000CFFC7B681B689B68BB60BB6843F07703B6
:10AB8000BB607B681B68BA689A604FE07B68186896
:10AB90003B6899683B685A683B68DB6800F0B8FC22
:10ABA0007B681B689A687B681B6842F480429A60E5
:10ABB0003CE07B6818683B6859683B68DB681A466C
:10ABC00000F02AFC7B681B685021184600F083FCCB
:10ABD0002CE07B6818683B6859683B68DB681A465C
:10ABE00000F049FC7B681B686021184600F073FC8C
:10ABF0001CE07B6818683B6859683B68DB681A464C
:10AC000000F00AFC7B681B684021184600F063FCDA
:10AC10000CE07B681A683B681B681946104600F018
:10AC20005AFC03E00123FB7300E000BF7B680122B4
:10AC300083F83D207B68002283F83C20FB7B18468C
:10AC40001037BD4680BD00BF7000100050001000DE
:10AC500040001000300010002000100080B485B0CB
:10AC600000AF786039607B681B68FB607B684C4A8A
:10AC7000934217D07B68B3F1804F13D07B68494A69
:10AC800093420FD07B68484A93420BD07B68474A77
:10AC9000934207D07B68464A934203D07B68454A7B
:10ACA000934208D1FB6823F07003FB603B685B684C
:10ACB000FA681343FB607B68394A934223D07B6870
:10ACC000B3F1804F1FD07B68364A93421BD07B681C
:10ACD000354A934217D07B68344A934213D07B683D
:10ACE000334A93420FD07B68334A93420BD07B6840
:10ACF000324A934207D07B68314A934203D07B6843
:10AD00002C4A934208D1FB6823F44073FB603B68F4
:10AD1000DB68FA681343FB60FB6823F080023B6842
:10AD20005B691343FB607B68FA681A603B689A684A
:10AD30007B68DA623B681A687B689A627B68184AAB
:10AD4000934213D07B681A4A93420FD07B681A4A09
:10AD500093420BD07B68194A934207D07B68184A0C
:10AD6000934203D07B68134A934203D13B681A692C
:10AD70007B681A637B6801225A617B681B6903F058
:10AD80000103012B05D17B681B6923F001027B685D
:10AD90001A6100BF1437BD465DF8047B704700BFE1
:10ADA000002C01400004004000080040000C00405E
:10ADB0000034014000500140004001400044014087
:10ADC0000048014080B487B000AF786039607B688C
:10ADD0001B6A7B617B681B6A23F001027B681A6235
:10ADE0007B685B683B617B689B69FB60FB6823F465
:10ADF000803323F07003FB60FB6823F00303FB60E8
:10AE00003B681B68FA681343FB607B6923F002030D
:10AE10007B613B689B687A6913437B617B68304A3E
:10AE2000934213D07B682F4A93420FD07B682E4AFF
:10AE300093420BD07B682D4A934207D07B682C4A03
:10AE4000934203D07B682B4A93420CD17B6923F059
:10AE500008037B613B68DB687A6913437B617B692C
:10AE600023F004037B617B681D4A934213D07B6807
:10AE70001C4A93420FD07B681B4A93420BD07B68DD
:10AE80001A4A934207D07B68194A934203D07B68E1
:10AE9000184A934211D13B6923F480733B613B69AB
:10AEA00023F400733B613B685B693A6913433B6180
:10AEB0003B689B693A6913433B617B683A695A6016
:10AEC0007B68FA689A613B685A687B685A637B685A
:10AED0007A691A6200BF1C37BD465DF8047B704773
:10AEE000002C01400034014000400140004401407A
:10AEF000004801400050014080B487B000AF786046
:10AF000039607B681B6A7B617B681B6A23F01002D7
:10AF10007B681A627B685B683B617B689B69FB604E
:10AF2000FB6823F0807323F4E043FB60FB6823F4A9
:10AF30004073FB603B681B681B02FA681343FB60AD
:10AF40007B6923F020037B613B689B681B017A6966
:10AF500013437B617B682C4A934207D07B682B4A62
:10AF6000934203D07B682A4A93420DD17B6923F038
:10AF700080037B613B68DB681B017A6913437B615B
:10AF80007B6923F040037B617B681F4A934213D0A7
:10AF90007B681E4A93420FD07B681E4A93420BD0B7
:10AFA0007B681D4A934207D07B681C4A934203D0BA
:10AFB0007B68174A934213D13B6923F480633B615A
:10AFC0003B6923F400633B613B685B699B003A6922
:10AFD00013433B613B689B699B003A6913433B61A8
:10AFE0007B683A695A607B68FA689A613B685A687C
:10AFF0007B689A637B687A691A6200BF1C37BD461A
:10B000005DF8047B704700BF002C01400034014014
:10B010000050014000400140004401400048014010
:10B0200080B487B000AF786039607B681B6A7B6151
:10B030007B681B6A23F480727B681A627B685B689A
:10B040003B617B68DB69FB60FB6823F4803323F0A2
:10B050007003FB60FB6823F00303FB603B681B6825
:10B06000FA681343FB607B6923F400737B613B68E0
:10B070009B681B027A6913437B617B682B4A93426E
:10B0800007D07B682A4A934203D07B68294A9342BF
:10B090000DD17B6923F400637B613B68DB681B0295
:10B0A0007A6913437B617B6923F480637B617B68EE
:10B0B0001E4A934213D07B681D4A93420FD07B688F
:10B0C0001D4A93420BD07B681C4A934207D07B6891
:10B0D0001B4A934203D07B68164A934213D13B69C3
:10B0E00023F480533B613B6923F400533B613B688D
:10B0F0005B691B013A6913433B613B689B691B0118
:10B100003A6913433B617B683A695A607B68FA6825
:10B11000DA613B685A687B68DA637B687A691A622D
:10B1200000BF1C37BD465DF8047B7047002C014012
:10B130000034014000500140004001400044014003
:10B140000048014080B487B000AF786039607B6808
:10B150001B6A7B617B681B6A23F480527B681A62DE
:10B160007B685B683B617B68DB69FB60FB6823F0A5
:10B17000807323F4E043FB60FB6823F44073FB60BF
:10B180003B681B681B02FA681343FB607B6923F46E
:10B1900000537B613B689B681B037A6913437B61A7
:10B1A0007B682C4A934207D07B682B4A934203D09A
:10B1B0007B682A4A93420DD17B6923F400437B616B
:10B1C0003B68DB681B037A6913437B617B6923F46B
:10B1D00080437B617B681F4A934213D07B681E4A81
:10B1E00093420FD07B681E4A93420BD07B681D4A66
:10B1F000934207D07B681C4A934203D07B68174A6E
:10B20000934213D13B6923F480433B613B6923F4B0
:10B2100000433B613B685B699B013A6913433B61B7
:10B220003B689B699B013A6913433B617B683A69C0
:10B230005A607B68FA68DA613B685A687B681A640E
:10B240007B687A691A6200BF1C37BD465DF8047BD3
:10B25000704700BF002C0140003401400050014005
:10B2600000400140004401400048014080B487B0E4
:10B2700000AF786039607B681B6A3B617B681B6A42
:10B2800023F480327B681A627B685B687B617B6831
:10B290001B6DFB60FB6823F4803323F07003FB60BD
:10B2A0003B681B68FA681343FB603B6923F4003377
:10B2B0003B613B689B681B043A6913433B617B68B5
:10B2C000194A934213D07B68184A93420FD07B6887
:10B2D000174A93420BD07B68164A934207D07B688B
:10B2E000154A934203D07B68144A934209D17B6983
:10B2F00023F480337B613B685B691B027A691343EB
:10B300007B617B687A695A607B68FA681A653B687A
:10B310005A687B689A647B683A691A6200BF1C3776
:10B32000BD465DF8047B7047002C014000340140AD
:10B3300000400140004401400048014000500140ED
:10B3400080B487B000AF786039607B681B6A3B616E
:10B350007B681B6A23F480127B681A627B685B68D7
:10B360007B617B681B6DFB60FB6823F0807323F4BB
:10B37000E043FB603B681B681B02FA681343FB60F9
:10B380003B6923F400133B613B689B681B053A69EA
:10B3900013433B617B681A4A934213D07B68194A76
:10B3A00093420FD07B68184A93420BD07B68174AB0
:10B3B000934207D07B68164A934203D07B68154AB4
:10B3C000934209D17B6923F480237B613B685B69ED
:10B3D0009B027A6913437B617B687A695A607B6858
:10B3E000FA681A653B685A687B68DA647B683A6970
:10B3F0001A6200BF1C37BD465DF8047B704700BF72
:10B40000002C014000340140004001400044014054
:10B41000004801400050014080B487B000AFF860A0
:10B42000B9607A60FB681B6A7B61FB681B6A23F06A
:10B430000102FB681A62FB689B693B613B6923F070
:10B44000F0033B617B681B013A6913433B617B69F5
:10B4500023F00A037B617A69BB6813437B61FB6855
:10B460003A699A61FB687A691A6200BF1C37BD4667
:10B470005DF8047B704780B487B000AFF860B960B6
:10B480007A60FB681B6A7B61FB681B6A23F0100211
:10B49000FB681A62FB689B693B613B6923F470435C
:10B4A0003B617B681B033A6913433B617B6923F073
:10B4B000A0037B61BB681B017A6913437B61FB6856
:10B4C0003A699A61FB687A691A6200BF1C37BD4607
:10B4D0005DF8047B704780B485B000AF7860396058
:10B4E0007B689B68FB60FB6823F4401323F07003C8
:10B4F000FB603A68FB68134343F00703FB607B681B
:10B50000FA689A6000BF1437BD465DF8047B704747
:10B5100080B487B000AFF860B9607A603B60FB68C8
:10B520009B687B617B6923F47F437B613B681A02E4
:10B530007B681A43BB6813437A6913437B61FB68DA
:10B540007A699A6000BF1C37BD465DF8047B70477E
:10B5500080B487B000AFF860B9607A60BB6803F070
:10B560001F03012202FA03F37B61FB681A6A7B69FD
:10B57000DB431A40FB681A62FB681A6ABB6803F077
:10B580001F03796801FA03F31A43FB681A6200BFCC
:10B590001C37BD465DF8047B7047000080B485B061
:10B5A00000AF786039607B6893F83C30012B01D1A3
:10B5B000022374E07B68012283F83C207B6802222E
:10B5C00083F83D207B681B685B68FB607B681B68B9
:10B5D0009B68BB607B681B68344A934209D07B68D8
:10B5E0001B68334A934204D07B681B68314A9342FC
:10B5F00008D1FB6823F47003FB603B685B68FA6862
:10B600001343FB60FB6823F0007323F07003FB60BF
:10B610003B681B68FA681343FB607B681B68FA6829
:10B620005A607B681B68214A934222D07B681B6862
:10B63000B3F1804F1DD07B681B681F4A934218D01E
:10B640007B681B681D4A934213D07B681B681C4AA9
:10B6500093420ED07B681B68154A934209D07B68E1
:10B660001B68184A934204D07B681B68114A9342B6
:10B670000CD1BB6823F08003BB603B689B68BA6851
:10B680001343BB607B681B68BA689A607B680122C1
:10B6900083F83D207B68002283F83C200023184675
:10B6A0001437BD465DF8047B704700BF002C014095
:10B6B00000340140005001400004004000080040F8
:10B6C000000C00400040014080B485B000AF7860BD
:10B6D00039600023FB607B6893F83C30012B01D17B
:10B6E000022378E07B68012283F83C20FB6823F08A
:10B6F000FF023B68DB681343FB60FB6823F4407286
:10B700003B689B681343FB60FB6823F480623B68E3
:10B710005B681343FB60FB6823F400623B681B68B3
:10B720001343FB60FB6823F480523B681B6913439F
:10B73000FB60FB6823F400523B685B691343FB60CA
:10B74000FB6823F480423B681B6B1343FB60FB6880
:10B7500023F470223B689B691B041343FB60FB6866
:10B7600023F080523B68DB691343FB607B681B68F6
:10B770001C4A934209D07B681B681B4A934204D041
:10B780007B681B68194A93421CD1FB6823F4700242
:10B790003B689B6A1B051343FB60FB6823F08072C8
:10B7A0003B681B6A1343FB60FB6823F000723B6835
:10B7B0005B6A1343FB60FB6823F000523B68DB6A63
:10B7C0001343FB607B681B68FA685A647B6800223D
:10B7D00083F83C20002318461437BD465DF8047BEF
:10B7E000704700BF002C0140003401400050014070
:10B7F00080B582B000AF78607B68002B01D1012357
:10B8000042E07B68D3F88830002B06D17B680022A9
:10B8100083F884207868F6F7EDFB7B682422C3F870
:10B8200088207B681B681A687B681B6822F001020D
:10B830001A607B689B6A002B02D0786800F024FBBA
:10B84000786800F025F80346012B01D101231BE0A5
:10B850007B681B685A687B681B6822F490425A60B8
:10B860007B681B689A687B681B6822F02A029A60D2
:10B870007B681B681A687B681B6842F001021A60CB
:10B88000786800F0A3FB034618460837BD4680BD24
:10B890002DE9B04F8CB000AF7861002387F82A30D3
:10B8A0007B699A687B691B691A437B695B691A43E8
:10B8B0007B69DB691343FB627B691B681A68AA4BCF
:10B8C00013407A691268F96A0B4313607B691B683D
:10B8D0005B6823F440517B69DA687B691B680A4323
:10B8E0005A607B699B69FB627B691B689F4A934234
:10B8F00004D07B691B6AFA6A1343FB627B691B688D
:10B900009B6823F06E4323F430637A691268F96A06
:10B910000B4393607B691B68DB6A23F00F017B6933
:10B920005A6A7B691B680A43DA627B691B68904A22
:10B93000934225D18F4BD3F8883003F00303032BB8
:10B940001AD801A252F823F059B9010869B90108BF
:10B9500061B9010871B90108012387F82B3016E19C
:10B96000022387F82B3012E1042387F82B300EE1F5
:10B97000082387F82B300AE1102387F82B3006E1E3
:10B980007B691B687C4A934238D17A4BD3F8883064
:10B9900003F00C030C2B2DD801A252F823F000BFAA
:10B9A000D5B90108F5B90108F5B90108F5B90108DB
:10B9B000E5B90108F5B90108F5B90108F5B90108BB
:10B9C000DDB90108F5B90108F5B90108F5B90108B3
:10B9D000EDB90108002387F82B30D8E0022387F85F
:10B9E0002B30D4E0042387F82B30D0E0082387F8ED
:10B9F0002B30CCE0102387F82B30C8E07B691B6824
:10BA00005E4A934225D15B4BD3F8883003F0300374
:10BA1000302B16D0302B18D8202B0AD0202B14D83E
:10BA2000002B02D0102B08D00FE0002387F82B301A
:10BA3000ADE0022387F82B30A9E0042387F82B30F0
:10BA4000A5E0082387F82B30A1E0102387F82B30DE
:10BA50009DE07B691B684A4A934225D1454BD3F848
:10BA6000883003F0C003C02B16D0C02B18D8802B11
:10BA70000AD0802B14D8002B02D0402B08D00FE026
:10BA8000002387F82B3082E0022387F82B307EE0FA
:10BA9000042387F82B307AE0082387F82B3076E0F0
:10BAA000102387F82B3072E07B691B68354A93427C
:10BAB0002AD1304BD3F8883003F44073B3F5407F7C
:10BAC0001AD0B3F5407F1BD8B3F5007F0CD0B3F587
:10BAD000007F15D8002B03D0B3F5807F08D00FE08E
:10BAE000002387F82B3052E0022387F82B304EE0FA
:10BAF000042387F82B304AE0082387F82B3046E0F0
:10BB0000102387F82B3042E07B691B68174A934269
:10BB10003AD1184BD3F8883003F44063B3F5406F43
:10BB20001AD0B3F5406F1BD8B3F5006F0CD0B3F546
:10BB3000006F15D8002B03D0B3F5806F08D00FE04D
:10BB4000002387F82B3022E0022387F82B301EE0F9
:10BB5000042387F82B301AE0082387F82B3016E0EF
:10BB6000102387F82B3012E0F369FFCF00800040EC
:10BB700000380140001002400044004000480040EE
:10BB8000004C004000500040102387F82B307B69A8
:10BB90001B68AE4A934240F0978097F82B30082BF1
:10BBA00023D801A252F823F0CDBB0108EBBB01085A
:10BBB000D5BB0108EBBB0108DBBB0108EBBB0108EF
:10BBC000EBBB0108EBBB0108E3BB0108FBF7BCFDC5
:10BBD000786210E09E4B7B620DE0FBF749FD7862D6
:10BBE00009E04FF400437B6205E000237B62012300
:10BBF00087F82A3000BF7B6A002B00F030817B6918
:10BC00005B6A944A32F813301A467B6AB3FBF2F34C
:10BC1000BB617B695A6813465B001344BA699A4258
:10BC200005D37B695B681B03BA699A4203D9012378
:10BC300087F82A3013E17B6A0022BB60FA607B69D7
:10BC40005B6A844A32F813309BB200223B607A6010
:10BC5000D7E90023D7E90201F4F79EFC02460B4620
:10BC6000104619464FF000024FF000030B0243EA62
:10BC70001063020279694968490800200C460546AC
:10BC800012EB040843EB05097B695B6800229A46C6
:10BC9000934652465B4640464946F4F77DFC0246D1
:10BCA0000B4613463B623B6AB3F5407F08D33B6AC1
:10BCB000B3F5801F04D27B691B683A6ADA60CEE074
:10BCC000012387F82A30CAE07B69DB69B3F5004FAE
:10BCD00066D197F82B30082B27D801A252F823F011
:10BCE00005BD01080DBD010815BD01082BBD0108EA
:10BCF0001BBD01082BBD01082BBD01082BBD010890
:10BD000023BD0108FBF720FD786214E0FBF732FD4C
:10BD1000786210E04E4B7B620DE0FBF7A9FC786285
:10BD200009E04FF400437B6205E000237B620123BE
:10BD300087F82A3000BF7B6A002B00F090807B6977
:10BD40005B6A444A32F813301A467B6AB3FBF2F35B
:10BD50005A007B695B685B081A447B695B68B2FBCD
:10BD6000F3F33B623B6A0F2B16D93B6AB3F5803F76
:10BD700012D23B6A9BB223F00F03FB833B6A5B0842
:10BD80009BB203F007039AB2FB8B1343FB837B69DF
:10BD90001B68FA8BDA6062E0012387F82A305EE0E4
:10BDA00097F82B30082B28D801A252F823F000BFB7
:10BDB000D5BD0108DDBD0108E5BD0108FBBD0108D9
:10BDC000EBBD0108FBBD0108FBBD0108FBBD01087F
:10BDD000F3BD0108FBF7B8FC786214E0FBF7CAFC7E
:10BDE000786210E01A4B7B620DE0FBF741FC786251
:10BDF00009E04FF400437B6205E000237B620123EE
:10BE000087F82A3000BF7B6A002B28D07B695B6AE9
:10BE1000104A32F813301A467B6AB3FBF2F27B69A0
:10BE20005B685B081A447B695B68B2FBF3F33B62B7
:10BE30003B6A0F2B10D93B6AB3F5803F0CD23B6AAB
:10BE40009AB27B691B68DA6009E000BF008000409D
:10BE50000024F400F4E50108012387F82A307B6907
:10BE60000122A3F86A207B690122A3F868207B697C
:10BE700000225A677B6900229A6797F82A30184691
:10BE80003037BD46BDE8B08F80B483B000AF786076
:10BE90007B689B6A03F00803002B0AD07B681B6851
:10BEA0005B6823F400417B689A6B7B681B680A43DC
:10BEB0005A607B689B6A03F00103002B0AD07B6801
:10BEC0001B685B6823F400317B68DA6A7B681B6857
:10BED0000A435A607B689B6A03F00203002B0AD076
:10BEE0007B681B685B6823F480317B681A6B7B6816
:10BEF0001B680A435A607B689B6A03F00403002BAB
:10BF00000AD07B681B685B6823F480217B685A6BCE
:10BF10007B681B680A435A607B689B6A03F01003C6
:10BF2000002B0AD07B681B689B6823F480517B68D8
:10BF3000DA6B7B681B680A439A607B689B6A03F034
:10BF40002003002B0AD07B681B689B6823F40051F8
:10BF50007B681A6C7B681B680A439A607B689B6AE3
:10BF600003F04003002B1AD07B681B685B6823F446
:10BF700080117B685A6C7B681B680A435A607B6837
:10BF80005B6CB3F5801F0AD17B681B685B6823F488
:10BF9000C0017B689A6C7B681B680A435A607B68A7
:10BFA0009B6A03F08003002B0AD07B681B685B68E8
:10BFB00023F400217B68DA6C7B681B680A435A60B3
:10BFC00000BF0C37BD465DF8047B704780B598B064
:10BFD00002AF78607B680022C3F89020FAF7EEFE8B
:10BFE00078657B681B681B6803F00803082B2FD15A
:10BFF0006FF07E4300937B6D00224FF40011786850
:10C0000000F08EF80346002B22D07B681B68BB63D0
:10C01000BB6B53E8003F7B637B6B23F080033B6586
:10C020007B681B681A463B6D7B643A64396C7A6C9A
:10C0300041E80023FB63FB6B002BE6D17B682022E9
:10C04000C3F888207B68002283F88420032363E000
:10C050007B681B681B6803F00403042B49D16FF055
:10C060007E4300937B6D00224FF48001786800F0DE
:10C0700057F80346002B3CD07B681B687B627B6AC9
:10C0800053E8003F3B623B6A23F49073FB647B6898
:10C090001B681A46FB6C3B63FA62F96A3A6B41E82B
:10C0A0000023BB62BB6A002BE6D17B681B680833A8
:10C0B0003B613B6953E8003FFB60FB6823F00103F1
:10C0C000BB647B681B680833BA6CFA61BB61B969F1
:10C0D000FA6941E800237B617B69002BE5D17B682D
:10C0E0002022C3F88C207B68002283F8842003235D
:10C0F00012E07B682022C3F888207B682022C3F8E6
:10C100008C207B680022DA667B6800221A677B68D5
:10C11000002283F88420002318465837BD4680BD8E
:10C1200080B584B000AFF860B9603B601346FB7126
:10C130004FE0BB69B3F1FF3F4BD0FAF73FFE024639
:10C140003B68D31ABA699A4202D3BB69002B01D16A
:10C1500003234EE0FB681B681B6803F00403002BFD
:10C1600037D0BB68802B34D0BB68402B31D0FB6804
:10C170001B68DB6903F00803082B10D1FB681B6800
:10C1800008221A62F86800F038F8FB680822C3F841
:10C190009020FB68002283F88420012329E0FB68BB
:10C1A0001B68DB6903F40063B3F5006F11D1FB6812
:10C1B0001B684FF400621A62F86800F01EF8FB6812
:10C1C0002022C3F89020FB68002283F884200323F8
:10C1D0000FE0FB681B68DA69BB681340BA689A42D3
:10C1E0000CBF01230023DBB21A46FB799A42A0D090
:10C1F000002318461037BD4680BD80B495B000AF0F
:10C2000078607B681B687B637B6B53E8003F3B6314
:10C210003B6B23F49073FB647B681B681A46FB6CD2
:10C220003B64FA63F96B3A6C41E80023BB63BB6B78
:10C23000002BE6D17B681B6808333B623B6A53E8FE
:10C24000003FFB61FB6923F0805323F00103BB64D3
:10C250007B681B680833BA6CFA62BB62B96AFA6A17
:10C2600041E800237B627B6A002BE3D17B68DB6EB5
:10C27000012B18D17B681B68FB60FB6853E8003F0B
:10C28000BB60BB6823F010037B647B681B681A46A5
:10C290007B6CBB617A617969BA6941E800233B61D3
:10C2A0003B69002BE6D17B682022C3F88C207B6899
:10C2B0000022DA667B6800225A6700BF5437BD4609
:10C2C0005DF8047B704780B485B000AF78607B6810
:10C2D00093F88430012B01D1022327E07B680122EF
:10C2E00083F884207B682422C3F888207B681B683D
:10C2F0001B68FB607B681B681A687B681B6822F000
:10C3000001021A60FB6823F00053FB607B68002287
:10C310005A667B681B68FA681A607B682022C3F83B
:10C3200088207B68002283F8842000231846143775
:10C33000BD465DF8047B704780B584B000AF78607F
:10C3400039607B6893F88430012B01D102232DE002
:10C350007B68012283F884207B682422C3F888202C
:10C360007B681B681B68FB607B681B681A687B68BE
:10C370001B6822F001021A607B681B689B6823F02F
:10C3800060417B681B683A680A439A60786800F0ED
:10C390004FF87B681B68FA681A607B682022C3F834
:10C3A00088207B68002283F88420002318461037F9
:10C3B000BD4680BD80B584B000AF786039607B68D1
:10C3C00093F88430012B01D102232DE07B680122F8
:10C3D00083F884207B682422C3F888207B681B684C
:10C3E0001B68FB607B681B681A687B681B6822F00F
:10C3F00001021A607B681B689B6823F060617B68A0
:10C400001B683A680A439A60786800F011F87B6804
:10C410001B68FA681A607B682022C3F888207B6852
:10C42000002283F88420002318461037BD4680BDC3
:10C4300080B485B000AF78607B685B6E002B08D15C
:10C440007B680122A3F86A207B680122A3F8682098
:10C4500031E00823FB730823BB737B681B689B6870
:10C460005B0EDBB203F007037B737B681B689B6882
:10C470005B0FDBB203F007033B73BB7B3A7B1149D5
:10C480008A5C02FB03F33A7B0F498A5C93FBF2F36D
:10C490009AB27B68A3F86A20FB7B7A7B09498A5CA5
:10C4A00002FB03F37A7B08498A5C93FBF2F39AB2AE
:10C4B0007B68A3F8682000BF1437BD465DF8047B95
:10C4C000704700BF0CE6010814E6010880B400AF15
:10C4D000074BD3F88830064A43F47003C2F888301B
:10C4E000034B044A9A6000BFBD465DF8047B704769
:10C4F00000ED00E00000010880B586B000AFF860F4
:10C50000B9601346FB71FB68002B01D103231FE0C8
:10C51000FB680022C3F8B822FB680022C3F8C022DF
:10C52000FB680022C3F8CC22BB68002B03D0FB6859
:10C53000BA68C3F8B422FB68012283F89C22FB6826
:10C54000FA791A70F868F5F705FF0346FB75FB7D6D
:10C5500018461837BD4680BD80B584B000AF7860FE
:10C5600039600023FB813B68002B01D1032316E0D7
:10C570007B683A68C3F8B8227B68D3F8B832DB6AC4
:10C58000002B0BD07B68D3F8B832DB6A07F10E02C0
:10C590001046984702467B68C3F8CC220023184611
:10C5A0001037BD4680BD80B582B000AF7860786836
:10C5B000F5F730FF034618460837BD4680BD80B406
:10C5C00083B000AF7860002318460C37BD465DF895
:10C5D000047B704780B584B000AF78600B46FB7079
:10C5E0000323FB737B68D3F8B832002B09D07B6838
:10C5F000D3F8B8321B68FA78114678689847034632
:10C60000FB73FB7B18461037BD4680BD80B582B0FA
:10C6100000AF78600B46FB707B68D3F8B832002B14
:10C6200007D07B68D3F8B8325B68FA78114678682F
:10C630009847002318460837BD4680BD80B584B0B2
:10C6400000AF786039607B6803F2AA233968184626
:10C6500000F046FF7B680122C3F894227B68B3F8A0
:10C66000B0321A467B68C3F898227B6893F8AA32E6
:10C6700003F01F03022B1AD0022B22D8002B02D06A
:10C68000012B0AD01DE07B6803F2AA2319467868C3
:10C6900000F0EEF90346FB7320E07B6803F2AA2367
:10C6A0001946786800F052FA0346FB7316E07B687F
:10C6B00003F2AA231946786800F091FA0346FB7347
:10C6C0000CE07B6893F8AA3223F07F03DBB21946B3
:10C6D0007868F5F7FFFE0346FB7300BFFB7B184647
:10C6E0001037BD4680BD80B586B000AFF8600B4600
:10C6F0007A60FB72FB7A002B38D1FB6803F5AA73D2
:10C700003B61FB68D3F89432032B4AD13B699A68AA
:10C710003B69DB689A4213D93B699A683B69DB68DD
:10C72000D21A3B699A603B69DA683B699B6893421D
:10C7300028BF13461A467968F86800F0C5FF30E054
:10C74000FB6893F89C32DBB2032B0BD1FB68D3F868
:10C75000B8321B69002B05D0FB68D3F8B8321B69CF
:10C76000F8689847F86800F0C0FF1AE0FB6893F893
:10C770009C32DBB2032B14D1FB68D3F8B8329B692F
:10C78000002B0ED0FB68D3F8B8329B69FA7A1146B9
:10C79000F86898470346FB75FB7D002B01D0FB7DB5
:10C7A00000E0002318461837BD4680BD80B586B02E
:10C7B00000AFF8600B467A60FB72FB7A002B6BD1FE
:10C7C000FB6814333B61FB68D3F89432022B56D1DB
:10C7D0003B699A683B69DB689A4214D93B699A685D
:10C7E0003B69DB68D21A3B699A603B699B681A46D1
:10C7F0007968F86800F03AFF002300220021F86809
:10C80000F5F712FF3BE03B69DA683B699B689A42A7
:10C810001CD13B695A683B69DB689A4216D33B6975
:10C820005A68FB68D3F898329A420FD2002200214E
:10C83000F86800F01BFFFB680022C3F89822002371
:10C8400000220021F868F5F7EFFE18E0FB6893F886
:10C850009C32DBB2032B0BD1FB68D3F8B832DB6818
:10C86000002B05D0FB68D3F8B832DB68F86898472E
:10C870008021F868F5F72EFEF86800F049FFFB68A4
:10C8800093F8A032012B22D1F868FFF798FEFB68DD
:10C89000002283F8A0221AE0FB6893F89C32DBB2F6
:10C8A000032B14D1FB68D3F8B8325B69002B0ED090
:10C8B000FB68D3F8B8325B69FA7A1146F868984792
:10C8C0000346FB75FB7D002B01D0FB7D00E00023C0
:10C8D00018461837BD4680BD80B582B000AF78607D
:10C8E0007B68012283F89C227B680022C3F8942293
:10C8F0007B6800225A607B680022C3F8A4227B6810
:10C90000D3F8B832002B01D103232FE07B68D3F892
:10C91000BC32002B0FD07B68D3F8B8325B68002B99
:10C9200009D07B68D3F8B8325B687A685268D2B2B3
:10C930001146786898474023002200217868F5F76F
:10C9400084FD7B680122A3F864217B684022C3F840
:10C9500060214023002280217868F5F776FD7B680E
:10C9600001229A847B6840221A6200231846083705
:10C97000BD4680BD80B483B000AF78600B46FB70CD
:10C980007B68FA781A74002318460C37BD465DF8A8
:10C99000047B704780B483B000AF78607B6893F805
:10C9A0009C32DAB27B6883F89D227B68042283F88C
:10C9B0009C22002318460C37BD465DF8047B704767
:10C9C00080B483B000AF78607B6893F89C32DBB2B0
:10C9D000042B06D17B6893F89D32DAB27B6883F82A
:10C9E0009C22002318460C37BD465DF8047B704737
:10C9F00080B582B000AF78607B68D3F8B832002B86
:10CA000001D1032312E07B6893F89C32DBB2032B45
:10CA10000BD17B68D3F8B832DB69002B05D07B687B
:10CA2000D3F8B832DB69786898470023184608378E
:10CA3000BD4680BD80B487B000AF78607B687B6105
:10CA40007B691B787B827B6901337B617B691B7807
:10CA50003B823B8A1B021AB2B7F9123013431BB256
:10CA6000FB81FB8918461C37BD465DF8047B704787
:10CA700080B584B000AF786039600023FB733B68F9
:10CA80001B7803F06003402B05D0402B53D8002BBC
:10CA90000BD0202B4FD17B68D3F8B8329B68396814
:10CAA000786898470346FB734AE03B685B78092B3C
:10CAB0003BD801A252F823F00DCB010821CB01088D
:10CAC0002BCB010817CB01082BCB0108EBCA0108BF
:10CAD000E1CA01082BCB010803CB0108F5CA010804
:10CAE0003968786800F0DEF924E03968786800F089
:10CAF0006DFB1FE03968786800F0ACFB0346FB7300
:10CB000018E03968786800F04BFC13E03968786801
:10CB100000F07CFC0EE03968786800F0ABFC09E0BE
:10CB20003968786800F0BAFC04E03968786800F089
:10CB300011FD00BF04E03968786800F00BFD00BF0C
:10CB4000FB7B18461037BD4680BD00BF80B584B062
:10CB500000AF786039600023FB733B681B7803F0FB
:10CB60006003402B05D0402B2FD8002B01D0202B69
:10CB70002BD17B6893F89C32DBB2013B022B1DD892
:10CB80003B689B88DBB2012B13D87B68D3F8B832A3
:10CB90009B683968786898470346FB733B68DB8875
:10CBA000002B10D1FB7B002B0DD1786800F09DFD90
:10CBB00009E03968786800F0CDFC04E039687868ED
:10CBC00000F0C8FC00E000BF04E03968786800F0BD
:10CBD000C1FC00BFFB7B18461037BD4680BD80B549
:10CBE00084B000AF786039600023FB733B689B889A
:10CBF000BB733B681B7803F06003402B07D0402BCE
:10CC000000F24581002B0CD0202B40F040817B6846
:10CC1000D3F8B8329B683968786898470346FB7345
:10CC20003AE13B685B78032B07D0032B00F32981A3
:10CC3000002B7FD0012B3CD023E17B6893F89C3202
:10CC4000DBB2022B02D0032B16D02CE0BB7B002BD7
:10CC50000DD0BB7B802B0AD0BB7B19467868F5F7DB
:10CC600039FC80217868F5F735FC00BF20E0396891
:10CC7000786800F06FFC1BE03B685B88002B0ED1EE
:10CC8000BB7B002B0BD0BB7B802B08D03B68DB88A9
:10CC9000002B04D1BB7B19467868F5F71BFC78683C
:10CCA00000F023FD04E03968786800F053FC00BF11
:10CCB000ECE07B6893F89C32DBB2022B02D0032BB2
:10CCC00016D030E0BB7B002B0DD0BB7B802B0AD075
:10CCD000BB7B19467868F5F7FDFB80217868F5F78E
:10CCE000F9FB00BF25E03968786800F033FC20E0EC
:10CCF0003B685B88002B1BD1BB7B03F07F03002BC1
:10CD000004D0BB7B19467868F5F703FC786800F01F
:10CD1000ECFC7B68D3F8B8329B6839687868984730
:10CD20000346FB7304E03968786800F013FC00E008
:10CD300000BFABE07B6893F89C32DBB2022B02D0E1
:10CD4000032B32D097E0BB7B002B07D0BB7B802B23
:10CD500004D03968786800F0FDFB91E097F90E3057
:10CD6000002B0BDABB7B03F07F0213469B001344BE
:10CD70009B0010337A68134404330BE0BB7B03F051
:10CD80007F0213469B0013449B0003F5A8737A6847
:10CD900013440433BB60BB6800221A60BB680222E4
:10CDA0001946786800F047FC6AE097F90E30002BCE
:10CDB00011DABB7B03F00F02796813469B00134422
:10CDC0009B000B4424331B88002B17D139687868EB
:10CDD00000F0C0FB54E0BB7B03F00F027968134600
:10CDE0009B0013449B000B4403F5B2731B88002B7C
:10CDF00004D13968786800F0ADFB41E097F90E3056
:10CE0000002B0BDABB7B03F07F0213469B0013441D
:10CE10009B0010337A68134404330BE0BB7B03F0B0
:10CE20007F0213469B0013449B0003F5A8737A68A6
:10CE300013440433BB60BB7B002B02D0BB7B802B35
:10CE400003D1BB6800221A600EE0BB7B19467868EC
:10CE5000F5F77EFB0346002B03D0BB6801221A6066
:10CE600002E0BB6800221A60BB680222194678689B
:10CE700000F0E1FB04E03968786800F06BFB00BF6C
:10CE800004E03968786800F065FB00BF04E03968A9
:10CE9000786800F05FFB00BFFB7B18461037BD468B
:10CEA00080BD000080B584B000AF78603960002399
:10CEB0003B810023FB600023FB723B685B881B0AFD
:10CEC0009BB2013B0E2B00F2528101A252F823F0DB
:10CED00041CF010859CF010899CF01086FD101084E
:10CEE0006FD101080FD101083BD101086FD10108B2
:10CEF0006FD101086FD101086FD101086FD101080E
:10CF00006FD101086FD101080DCF01087B68D3F8FC
:10CF1000B432DB69002B0BD07B68D3F8B432DB6909
:10CF20007A68127C07F1080110469847F86026E1FC
:10CF30003968786800F00EFBFB7A0133FB721EE162
:10CF40007B68D3F8B4321B687A68127C07F1080159
:10CF500010469847F86012E17B681B7C002B0DD1CE
:10CF60007B68D3F8B8329B6A07F1080210469847ED
:10CF7000F860FB68013302221A7000E17B68D3F885
:10CF8000B832DB6A07F1080210469847F860FB6880
:10CF9000013302221A70F2E03B685B88DBB2052B9A
:10CFA00000F2AC8001A252F823F000BFC5CF010807
:10CFB000F9CF01082DD0010861D0010895D00108F2
:10CFC000C9D001087B68D3F8B4325B68002B0BD062
:10CFD0007B68D3F8B4325B687A68127C07F1080189
:10CFE00010469847F86091E03968786800F0B2FA26
:10CFF000FB7A0133FB7289E07B68D3F8B4329B681B
:10D00000002B0BD07B68D3F8B4329B687A68127C13
:10D0100007F1080110469847F86077E039687868AA
:10D0200000F098FAFB7A0133FB726FE07B68D3F86B
:10D03000B432DB68002B0BD07B68D3F8B432DB68EA
:10D040007A68127C07F1080110469847F8605DE0A5
:10D050003968786800F07EFAFB7A0133FB7255E09C
:10D060007B68D3F8B4321B69002B0BD07B68D3F8F4
:10D07000B4321B697A68127C07F1080110469847A0
:10D08000F86043E03968786800F064FAFB7A0133AD
:10D09000FB723BE07B68D3F8B4325B69002B0BD0AA
:10D0A0007B68D3F8B4325B697A68127C07F10801B7
:10D0B00010469847F86029E03968786800F04AFA25
:10D0C000FB7A0133FB7221E07B68D3F8B4329B69B1
:10D0D000002B0BD07B68D3F8B4329B697A68127C42
:10D0E00007F1080110469847F8600FE03968786842
:10D0F00000F030FAFB7A0133FB7207E03968786898
:10D1000000F028FAFB7A0133FB7200BF37E07B683E
:10D110001B7C002B09D17B68D3F8B8325B6B07F11D
:10D12000080210469847F86029E03968786800F0EE
:10D1300011FAFB7A0133FB7221E07B681B7C002B28
:10D140000DD17B68D3F8B8321B6B07F1080210468B
:10D150009847F860FB68013307221A700FE03968BE
:10D16000786800F0F7F9FB7A0133FB7207E0396861
:10D17000786800F0EFF9FB7A0133FB7200BFFB7AAD
:10D18000002B1ED13B68DB88002B16D03B89002B7F
:10D190000ED03B68DA883B89934228BF13469BB286
:10D1A0003B813B891A46F968786800F044FA09E047
:10D1B0003968786800F0CEF904E0786800F095FAF4
:10D1C00000E000BF1037BD4680BD00BF80B584B011
:10D1D00000AF786039603B689B88002B31D13B6899
:10D1E000DB88002B2DD13B685B887F2B29D83B68DF
:10D1F0005B88DBB203F07F03FB737B6893F89C32A0
:10D20000DBB2032B04D13968786800F0A3F91DE084
:10D210007B68FA7B83F89E22FB7B19467868F5F7DA
:10D22000C3F9786800F061FAFB7B002B04D07B68BF
:10D23000022283F89C2209E07B68012283F89C2269
:10D2400004E03968786800F085F900BF00BF103746
:10D25000BD4680BD80B584B000AF786039600023E2
:10D26000FB733B685B88DAB24C4B1A704B4B1B78F4
:10D27000012B05D93968786800F06CF9032388E040
:10D280007B6893F89C32DBB2022B02D0032B25D0B3
:10D2900071E0424B1B78002B1CD0404B1B781A4688
:10D2A0007B685A603D4B1B7819467868FFF792F906
:10D2B0000346FB73FB7B002B04D03968786800F0D1
:10D2C00049F965E0786800F010FA7B68032283F87A
:10D2D0009C225DE0786800F008FA59E02F4B1B783B
:10D2E000002B12D17B68022283F89C222B4B1B78E7
:10D2F0001A467B685A60294B1B7819467868FFF7F5
:10D3000085F9786800F0F1F942E0244B1B781A4661
:10D310007B685B689A422AD07B685B68DBB21946FF
:10D320007868FFF773F91D4B1B781A467B685A60C3
:10D330001A4B1B7819467868FFF74CF90346FB73C4
:10D34000FB7B002B0FD03968786800F003F97B680D
:10D350005B68DBB219467868FFF758F97B680222F0
:10D3600083F89C2214E0786800F0BFF910E0786838
:10D3700000F0BBF90CE03968786800F0EBF8074B77
:10D380001B7819467868FFF741F90323FB7300BF48
:10D39000FB7B18461037BD4680BD00BFE42200204D
:10D3A00080B582B000AF786039603B68DB88012BC4
:10D3B00004D03968786800F0CDF823E07B6893F8F2
:10D3C0009C32DBB2022B02DC002B03DC15E0032BCA
:10D3D0000BD012E07B6800229A607B680833012240
:10D3E0001946786800F027F90CE07B6804330122C5
:10D3F0001946786800F01FF904E03968786800F091
:10D40000A9F800BF00BF0837BD4680BD80B582B017
:10D4100000AF786039607B6893F89C32DBB2013BE7
:10D42000022B1ED83B68DB88022B04D03968786851
:10D4300000F090F81AE07B680122DA607B68D3F88C
:10D44000A432002B05D07B68DB6843F002027B68C6
:10D45000DA607B680C3302221946786800F0EBF83A
:10D4600004E03968786800F075F800BF00BF08373D
:10D47000BD4680BD80B582B000AF786039603B6842
:10D480005B88012B06D17B680122C3F8A42278684F
:10D4900000F02BF900BF0837BD4680BD80B582B0D3
:10D4A00000AF786039607B6893F89C32DBB2013B57
:10D4B000022B0BD83B685B88012B0CD17B680022C8
:10D4C000C3F8A422786800F010F904E0396878689D
:10D4D00000F040F800E000BF00BF0837BD4680BD47
:10D4E00080B584B000AF786039603B68FB60FB6852
:10D4F0001A787B681A70FB680133FB60FB681A7846
:10D500007B685A70FB680133FB60F868FFF792FA9A
:10D5100003461A467B685A80FB680133FB60FB6850
:10D520000133FB60F868FFF785FA03461A467B680B
:10D530009A80FB680133FB60FB680133FB60F8688D
:10D54000FFF778FA03461A467B68DA8000BF103787
:10D55000BD4680BD80B582B000AF78603960802163
:10D560007868F4F7B7FF00217868F4F7B3FF00BFDD
:10D570000837BD4680BD80B586B000AFF860B960A1
:10D580007A600023FB75FB68002B36D0FB683B619B
:10D59000386900F036F8034601339BB25B009AB25B
:10D5A0007B681A80FB7DBA6813447A6812781A7017
:10D5B000FB7D0133FB75FB7DBA68134403221A70AF
:10D5C000FB7D0133FB7513E0FB7DBA6813443A69B8
:10D5D00012781A703B6901333B61FB7D0133FB75A7
:10D5E000FB7DBA68134400221A70FB7D0133FB7582
:10D5F0003B691B78002BE7D100E000BF1837BD4620
:10D6000080BD80B485B000AF78600023FB737B6879
:10D61000BB6005E0FB7B0133FB73BB680133BB6080
:10D62000BB681B78002BF5D1FB7B18461437BD4631
:10D630005DF8047B704780B584B000AFF860B960D6
:10D640007A60FB680222C3F89422FB687A689A61C8
:10D65000FB687A68DA617B68BA680021F868F4F7D9
:10D66000C2FF002318461037BD4680BD80B584B088
:10D6700000AFF860B9607A607B68BA680021F8682A
:10D68000F4F7B1FF002318461037BD4680BD80B5C2
:10D6900084B000AFF860B9607A60FB680322C3F819
:10D6A0009422FB687A68C3F85821FB687A68C3F84B
:10D6B0005C217B68BA680021F868F4F7B5FF0023A5
:10D6C00018461037BD4680BD80B584B000AFF86005
:10D6D000B9607A607B68BA680021F868F4F7A4FF43
:10D6E000002318461037BD4680BD80B582B000AF1C
:10D6F00078607B680422C3F8942200230022002172
:10D700007868F4F770FF002318460837BD4680BDDF
:10D7100080B582B000AF78607B680522C3F89422A0
:10D720000023002200217868F4F77EFF00231846CA
:10D730000837BD4680BD80B584B000AF78600B4629
:10D74000FB704FF40770F4F7D9FFF860FB68002B0B
:10D7500005D17B680022C3F8BC22022366E07B6807
:10D76000FA68C3F8BC227B681B7C002B19D14FF4EC
:10D770000073022281217868F4F767FE7B6801223A
:10D780001A874FF40073022201217868F4F75DFED6
:10D790007B680122A3F878217B681022A3F84E2031
:10D7A00016E04023022281217868F4F74EFE7B6860
:10D7B00001221A874023022201217868F4F745FEEE
:10D7C0007B680122A3F878217B681022A3F84E2001
:10D7D0000823032282217868F4F737FE7B68012250
:10D7E000A3F84C207B68D3F8C0321B689847FB68CD
:10D7F0000022C3F81422FB680022C3F818227B68B9
:10D800001B7C002B09D1FB68D3F804224FF4007372
:10D8100001217868F4F708FF07E0FB68D3F80422D9
:10D82000402301217868F4F7FFFE002318461037E3
:10D83000BD4680BD80B582B000AF78600B46FB70FE
:10D8400081217868F4F727FE7B6800221A8701217E
:10D850007868F4F720FE7B680022A3F87821822103
:10D860007868F4F718FE7B680022A3F84C207B68E8
:10D870000022A3F84E207B68D3F8BC32002B0ED0D8
:10D880007B68D3F8C0325B6898477B68D3F8BC32BA
:10D890001846F4F741FF7B680022C3F8BC2200233E
:10D8A00018460837BD4680BD80B586B000AF7860A9
:10D8B00039607B68D3F8BC323B6100237B73002363
:10D8C0007B810023FB753B69002B01D10323AFE073
:10D8D0003B681B7803F06003002B3FD0202B40F007
:10D8E0009F803B68DB88002B2ED03B681B785BB2A7
:10D8F000002B16DA7B68D3F8C0329B683A68507800
:10D9000039693A68D28898473B68DB88072B28BF7B
:10D910000723FB813B69FA8919467868FFF78BFE7C
:10D9200085E03B685A783B6983F800223B68DB88D6
:10D93000DAB23B6983F8012239693B68DB881A4611
:10D940007868FFF7A4FE72E07B68D3F8C0329B686A
:10D950003A68507800223968984768E03B685B78FD
:10D960000B2B52D801A252F823F000BF9DD9010819
:10D9700019DA01080BDA01080BDA01080BDA0108E1
:10D980000BDA01080BDA01080BDA01080BDA0108DF
:10D990000BDA0108C7D90108F1D901087B6893F8AF
:10D9A0009C32DBB2032B07D107F10A03022219468E
:10D9B0007868FFF740FE32E039687868FFF7CAFD03
:10D9C0000323FB752BE07B6893F89C32DBB2032BBF
:10D9D00007D107F10D03012219467868FFF72BFEE6
:10D9E0001DE039687868FFF7B5FD0323FB7516E085
:10D9F0007B6893F89C32DBB2032B0FD039687868D0
:10DA0000FFF7A8FD0323FB7508E039687868FFF786
:10DA1000A1FD0323FB7502E000BF08E000BF06E0A4
:10DA200039687868FFF796FD0323FB7500BFFB7D1F
:10DA300018461837BD4680BD80B584B000AF786009
:10DA40000B46FB707B68D3F8C432FB607B68D3F86D
:10DA5000BC32002B01D103234FE07B68D3F8BC32EA
:10DA6000BB60FA78796813469B0013449B000B4413
:10DA700018331B68002B29D0FA78796813469B006D
:10DA800013449B000B4418331A68F978F8680B4666
:10DA90009B000B44DB00034420331B68B2FBF3F113
:10DAA00001FB03F3D31A002B10D1FA7879681346DF
:10DAB0009B0013449B000B44183300221A60F97832
:10DAC000002300227868F4F78EFD15E0BB68002281
:10DAD000C3F814227B68D3F8C0321B69002B0BD02B
:10DAE0007B68D3F8C0321B69BA68D2F80802BA68FA
:10DAF00002F50471FA789847002318461037BD469E
:10DB000080BD80B584B000AF78600B46FB707B6849
:10DB1000D3F8BC32FB607B68D3F8BC32002B01D158
:10DB2000032315E0FB7819467868F4F79EFD02465A
:10DB3000FB68C3F80C227B68D3F8C032DB68FA6854
:10DB4000D2F80402FA6802F50372114698470023DE
:10DB500018461037BD4680BD80B584B000AF7860F0
:10DB60007B68D3F8BC32FB60FB68002B01D1032338
:10DB70001AE07B68D3F8C032002B14D0FB6893F80E
:10DB80000032FF2B0FD07B68D3F8C0329B68FA6855
:10DB900092F80002F968FA6892F801229847FB6847
:10DBA000FF2283F80022002318461037BD4680BDAF
:10DBB00080B483B000AF78607B6843221A80034B47
:10DBC00018460C37BD465DF8047B70474C010020B9
:10DBD00080B483B000AF78607B6843221A80034B27
:10DBE00018460C37BD465DF8047B704708010020DD
:10DBF00080B483B000AF78607B6843221A80034B07
:10DC000018460C37BD465DF8047B70479001002034
:10DC100080B483B000AF78607B680A221A80034B1F
:10DC200018460C37BD465DF8047B7047C4000020E1
:10DC300080B483B000AF786039603B68002B01D1BD
:10DC4000032304E07B683A68C3F8C0220023184627
:10DC50000C37BD465DF8047B704780B487B000AFD9
:10DC6000F860B9607A60FB68D3F8BC327B617B698D
:10DC7000002B01D1032308E07B69BA68C3F80822AE
:10DC80007B697A68C3F81022002318461C37BD460A
:10DC90005DF8047B704780B485B000AF7860396070
:10DCA0007B68D3F8BC32FB60FB68002B01D10323F7
:10DCB00004E0FB683A68C3F80422002318461437CE
:10DCC000BD465DF8047B704780B584B000AF7860D6
:10DCD0007B68D3F8BC32BB600123FB737B68D3F84D
:10DCE000BC32002B01D103231AE0BB68D3F81432F5
:10DCF000002B14D1BB680122C3F81422BB68D3F8EF
:10DD000010227B68DA62BB68D3F80822BB68D3F8BC
:10DD1000103281217868F4F766FC0023FB73FB7BEB
:10DD200018461037BD4680BD80B584B000AF78601E
:10DD30007B68D3F8BC32FB607B68D3F8BC32002B25
:10DD400001D1032316E07B681B7C002B09D1FB6803
:10DD5000D3F804224FF4007301217868F4F764FCCF
:10DD600007E0FB68D3F80422402301217868F4F728
:10DD70005BFC002318461037BD4680BD80B586B0D9
:10DD800000AF7860144A154BD31A7B617B693B6105
:10DD9000134B1B68002B02D1114B124A1A60104B17
:10DDA0001A687B6813443A699A4207D200F07AF8FD
:10DDB00003460C221A604FF0FF3309E0084B1B6842
:10DDC000FB60074B1A687B681344054A1360FB68C5
:10DDD00018461837BD4680BD000002200004000030
:10DDE000E8220020F02200200D488546FEF76EFB59
:10DDF0000C480D490D4A002302E0D458C4500433A6
:10DE0000C4188C42F9D30A4A0A4C002301E013607B
:10DE10000432A242FBD3F2F793FDF2F7BFFEFEE716
:10DE20000000022000000020D401002078E6010854
:10DE3000D4010020EC220020FEE700000CB430B535
:10DE4000174B0C1E1D689DB008DA8B232B604FF01A
:10DE5000FF301DB0BDE8304002B070474FF4027390
:10DE6000ADF8143014BF04F1FF3323460493079335
:10DE70004FF6FF7302900690ADF81630209A21AB52
:10DE800002A92846019300F06FF8431CBCBF8B2306
:10DE90002B60002CDDD0029B00221A70D9E700BF56
:10DEA00000000020014B1868704700BF00000020F0
:10DEB0002DE9F0478E681F46BE420B6882460C462D
:10DEC00090462DD8B1F90C2012F4906F26D06569D8
:10DED000096905EB4505A3EB010905EBD5757B1C2D
:10DEE0004B446D109D4238BF1D46530527D529462A
:10DEF000F2F7B8FD064660B321694A4600F0D8FA49
:10DF0000A38923F4906343F08003A38126616561B4
:10DF10004E44A5EB09052660A5603E46BE4200D9E9
:10DF20003E4620683246414600F0A8FAA3689B1B93
:10DF3000A3602368334423600020BDE8F0872A46AD
:10DF400000F0C4FA06460028E0D121695046F2F7F5
:10DF50001DFD0C23CAF80030A38943F04003A381C0
:10DF60004FF0FF30E9E700002DE9F04F98468B892C
:10DF70001B069DB007460D46144610D50B6973B9B4
:10DF80004021F2F76FFD2860286130B90C233B6017
:10DF90004FF0FF301DB0BDE8F08F40236B610023D0
:10DFA000099320238DF82930CDF80C803023DFF839
:10DFB0009C818DF82A304FF0010923469A4613F8C8
:10DFC000012B0AB1252AF9D1BAEB040B0BD05B4621
:10DFD000224629463846FFF76BFF013000F0A78044
:10DFE000099A5A4409929AF80030002B00F09F8059
:10DFF00000234FF0FF32CDE905230AF1010A049313
:10E0000007938DF853301A935446052214F8011BD8
:10E010004E48F2F73DFC049AD8B9D00644BF2023FD
:10E020008DF85330110744BF2B238DF853309AF8E5
:10E0300000302A2B15D0079A544600204FF00A0CC6
:10E04000214611F8013B303B092B4BD9B0B1079267
:10E0500014E0A0EB080309FA03F313430493A24668
:10E06000D2E7039B191D1B680391002BBBBF5B42CA
:10E0700042F0020207930793B8BF049223782E2B35
:10E080000AD163782A2B32D1039B1A1D1B68039295
:10E0900043EAE37302340593DFF8C0A0217803223A
:10E0A0005046F2F7F5FB38B1049BA0EB0A00402282
:10E0B000824013430134049314F8011B24488DF863
:10E0C00028100622F2F7E4FB002836D0214B1BBBB8
:10E0D000039B073323F0070308330393099B33445F
:10E0E00009936AE70CFB02320C460120A8E70023E3
:10E0F0000134059319464FF00A0C204610F8012B05
:10E10000303A092A03D9002BC6D00591C4E70CFB8D
:10E11000012104460123F0E703AB00932A460E4B8E
:10E1200004A93846AFF30080421C0646D6D1AB891D
:10E130005B063FF52DAF09982CE703AB00932A4609
:10E14000054B04A9384600F079F8EDE734E60108FC
:10E150003EE6010800000000B1DE01083AE60108D1
:10E160002DE9F047164698468A680B69DDF820903D
:10E170009342B8BF1346336091F8432007460C46DC
:10E180000AB1013333602368990642BF3368023312
:10E190003360256815F0060506D104F1190AE36815
:10E1A00032689B1AAB4226DC94F843302268003B6D
:10E1B00018BF012392062BD404F14302414638468E
:10E1C000C84701301ED02368226903F00603042BE0
:10E1D00002BFE5683368ED1AA3680CBF25EAE57550
:10E1E00000259342C4BF9B1AED1800261A34B5428D
:10E1F0001AD1002008E00123524641463846C8475C
:10E20000013003D14FF0FF30BDE8F0870135C6E79C
:10E21000E1185A1C302081F84300224494F845103C
:10E2200082F843100233C7E70123224641463846AD
:10E23000C8470130E6D00136D9E700002DE9FF4795
:10E240000F7E0C9E782F914680460C469A4601F12F
:10E25000430207D8622F0AD8002F00F0D280582F2F
:10E2600000F0B98004F1420684F842703AE0A7F168
:10E270006303152BF6D801A151F823F0D5E201086C
:10E28000E9E2010865E2010865E2010865E20108CA
:10E2900065E20108E9E2010865E2010865E20108BA
:10E2A00065E2010865E20108E9E3010813E30108FA
:10E2B000A3E3010865E2010865E201080BE4010837
:10E2C00065E2010813E3010865E2010865E201085F
:10E2D000ABE3010833681A1D1B68326004F1420683
:10E2E00084F8423001239DE033682068191D3160B5
:10E2F000060601D51D6803E04506FBD5B3F90050BD
:10E30000002D03DA2D236D4284F8433059480A2347
:10E3100011E021683368080653F8045B02D449060B
:10E3200048BFADB26F2F5348336014BF0A23082390
:10E33000002184F843106668A660002EA2BF216801
:10E3400021F0040121600DB9002E4BD01646B5FB1B
:10E35000F3F103FB1157C75D06F8017D2F46BB4261
:10E360000D46F4D9082B0BD12368DF0708D52369A4
:10E3700061689942DEBF302306F8013C06F1FF36A2
:10E38000921B2261CDF800A04B4603AA21464046CD
:10E39000FFF7E6FE01304AD14FF0FF3004B0BDE890
:10E3A000F087236843F0200323603348782784F8FC
:10E3B0004570236831681F0651F8045B02D45F067C
:10E3C00048BFADB23160D90744BF43F0200323609A
:10E3D0001DB11023ACE72748E9E7236823F02003A9
:10E3E0002360F6E71646BDE7336825686169181DA6
:10E3F00030602E061B6801D5196002E06806FBD567
:10E400001980002323611646BCE733681A1D326069
:10E410001E68626800213046F2F73AFA08B1801BA4
:10E42000606063682361002384F84330AAE72369AE
:10E43000324649464046D0470130ADD023689B075D
:10E4400013D4E068039B9842B8BF1846A6E701239F
:10E45000324649464046D04701309DD00135E368F9
:10E4600003995B1AAB42F2DCEBE7002504F11906D5
:10E47000F5E700BF45E6010856E60108884210B5F9
:10E4800001EB020402D98442234607D8431EA1426D
:10E4900008D011F8012B03F8012FF8E702440146D8
:10E4A0008A4200D110BD13F8014D02F8014DF7E783
:10E4B0000A44914200F1FF3300D1704710B511F8C2
:10E4C000014B03F8014F9142F9D110BD2DE9F04104
:10E4D000804615460C4621B9BDE8F0411146F2F7D9
:10E4E000C1BA2AB9F2F752FA00242046BDE8F081F9
:10E4F00000F01AF88542064602D8B5EB500FF4D862
:10E5000029464046F2F7AEFA07460028ECD0B5425D
:10E510002A46214628BF3246FFF7CAFF2146404619
:10E52000F2F734FA3C46E0E751F8043C181F002BA0
:10E53000BCBF0B58C0187047F8B500BFF8BC08BC8A
:10E540009E467047F8B500BFF8BC08BC9E467047B1
:10E550004D61737465720943683109436832094338
:10E56000683309436834090D0A0000002530332E52
:10E570003166092530332E3166092530332E316658
:10E58000092530332E3166092530332E3166090DC9
:10E590000A00000056312E302E330000566572738B
:10E5A000696F6E3A2025730D0A00000053544D33F5
:10E5B00032205669727475616C20436F6D506F72B2
:10E5C0007400000053544D6963726F656C65637429
:10E5D000726F6E696373000043444320436F6E663D
:10E5E0006967000043444320496E74657266616345
:10E5F00065000000010002000400060008000A0097
:10E600000C00100020004000800000010101010307
:10E6100007010000080402040801010100000000D5
:10E6200000000000010203040607080900000000C2
:10E6300001020304232D302B2000686C4C0065661A
:10E640006745464700303132333435363738394143
:10E650004243444546003031323334353637383959
:08E6600061626364656600005D
:08E66800601FFF7F01000000AC
:04E670000502010896
:04E67400E1010108B7
:10E678000400002000000000F001002058020020E3
:10E68800C0020020000000000000000000000000A0
:10E698000000000000000000000000000000000072
:10E6A8000000000000000000000000000000000062
:10E6B8000000000000000000000000000000000052
:10E6C800F1270108152801087528010839280108CB
:10E6D8009D280108C1280108FD2801080000000044
:10E6E80012010002020200408304405700020102A6
:10E6F80003010000040309041A03000000000000DD
:10E708000000000000000000000000000000000001
:10E7180000000000112A0108392A0108492A0108C5
:10E72800052B0108792B01081000000001000000EA
:10E738000024F4000A060002000000400100000066
:10E7480037D7010835D80108A9D80108000000000A
:10E7580059DB010839DA010803DB01080000000071
:10E768000000000000000000D1DB0108B1DB010857
:10E77800F1DB010811DC010809024300020100C0B5
:10E7880032090400000102020100052400100105FD
:10E798002401000104240202052406000107058261
:10E7A8000308001009040100020A0000000705011F
:10E7B800020002000705810200020000090243006E
:10E7C800020100C032090400000102020100052410
:10E7D800001001052401000104240202052406009A
:10E7E800010705820308001009040100020A00005D
:10E7F80000070501024000000705810240000000F3
:10E8080009074300020104C03209040000010202A2
:10E81800010005240010010524010001042402025E
:10E8280005240600010705820308001009040100F9
:10E83800020A0000000705010240000007058102E6
:04E84800400000008C
:040000050801DDE928
:00000001FF
